:020000040800F2
:1000000000000220712F0C08F52F0C0869DB060890
:10001000F52F0C08F52F0C08F52F0C080000000038
:10002000000000000000000000000000F52F0C0898
:10003000F52F0C0800000000F52F0C08415C0508A6
:10004000F52F0C08F52F0C08F52F0C08F52F0C08D0
:10005000F52F0C08F52F0C08E93B0508ED3B0508CA
:10006000F13B0508F53B0508F93B05084546040842
:100070005546040865460408754604088946040880
:100080009D460408B1460408F52F0C08F52F0C080E
:10009000F52F0C08F52F0C08F52F0C08FD3B050873
:1000A000F52F0C08F52F0C08F52F0C0891500408BB
:1000B000A5500408B9500408CD500408AD3904080F
:1000C000A1390408DD390408D1390408F52F0C08DA
:1000D000F52F0C083D5A0408495A0408555A0408DB
:1000E000013C0508F52F0C08000000000951040828
:1000F0005951040881510408F5500408C546040804
:10010000F52F0C0839940408E1500408F52F0C0869
:10011000615A0408F52F0C08F52F0C08B5A804083F
:10012000D9460408ED4604080147040815470408A9
:1001300029470408F52F0C08F52F0C08F52F0C089B
:1001400000000000000000000000000000000000AF
:100150003D47040851470408654704086D5A0408E0
:100160000D3A0408013A0408F52F0C08F52F0C0885
:10017000F52F0C08F52F0C08F52F0C0800000000D7
:10018000F52F0C08F52F0C08795A0408855A040835
:10019000F52F0C08F52F0C08F52F0C08F52F0C087F
:1001A000F52F0C08F52F0C08F52F0C08F52F0C086F
:1001B000F52F0C08F52F0C08F52F0C08F52F0C085F
:1001C000F52F0C08F52F0C08F52F0C08F52F0C084F
:1001D000F52F0C0869940408F52F0C08F52F0C086E
:1001E000F52F0C08F52F0C08F52F0C08F52F0C082F
:1001F000F52F0C08F52F0C08F52F0C08F52F0C081F
:10020000F52F0C08F52F0C08F52F0C08F52F0C080E
:100210001D5104083151040845510408F52F0C08FC
:10022000F52F0C08F52F0C08F52F0C080000000026
:100230003D940408F52F0C0800000000F52F0C0871
:10024000F52F0C08F52F0C08F52F0C08F52F0C08CE
:10025000F52F0C08F52F0C08F52F0C08F52F0C08BE
:10026000F52F0C08F52F0C08F52F0C08F52F0C08AE
:10027000F52F0C08F52F0C08F52F0C0800000000D6
:10028000F52F0C0800000000F52F0C0800000000FE
:0802900000000000F52F0C082E
:08029800D81F0C00010000005A
:1002A00010AE0124020100000200140030AE01244F
:1002B000020200000200140050AE0124020B0000F4
:1002C0000200140070AE01240203000004001400B8
:1002D00090AE01240208000004001400B0AE012416
:1002E000010C000000017700D0AE0124010D0000D8
:1002F00000017600F0AE012401120000000176003A
:1003000010AF0124011100000001760030AF01247C
:10031000010E01000001770050AF0124011300001D
:100320000001760070AF01240115000000001E00DE
:1003300090AF0124011B000000000D00B0AF0124AC
:10034000011C000000002C00D0AF012401160000A9
:1003500000000C00F0AF01240117000000000C00A9
:1003600010B00124011D000000000E0030B0012477
:10037000011E000000001E0050B001240118000002
:1003800000000C0070B001240119000000000E00F4
:1003900090B00124011A000000000C00B0B001244C
:1003A0000120000000000C00D0B001240121000059
:1003B00000000C00F0B00124012A01000001180027
:1003C00010B10124012200000001480030B10124D5
:1003D000012300000001490050B101240124000064
:1003E00000014A0070B101240125000000014B000A
:1003F00090B101240126000000014C00B0B101249D
:100400000127000000014D00D0B1012401280000A7
:1004100000014E00F0B101240129000000014F004D
:1004200010B20124012D00000000290030B2012487
:10043000012E01000000290050B20124012F01000B
:100440000000700070B20124013100000000310092
:1004500090B201240130010000005200B0B201242A
:100460000132010000012800D0B201240133000054
:1004700000017600F0B201240134010000012800DF
:1004800010B301240137000000003C0030B3012408
:08049000013A00000000200009
:020000040804EE
:10000000836B5A6D12F0500F5A6D1AD1196842F471
:1000100000725A650A6812F0080FCA6816D012F406
:10002000406F15D1CA68920412D45A6D22F48072BE
:100030005A655A6DD1040BD45A6D42F001025A65CB
:100040007047D20604D4DB6CDB6C18479007ECD009
:10005000704700BF704700BF836B5A6D42F040028B
:100060005A659A6D42F004029A65704702685549D4
:1000700038B5554B554D564CAA4218BF9A420CBF45
:10008000012300238A4208BF43F001033031A2421A
:1000900008BF43F0010330348A4208BF43F0010334
:1000A0003031A24208BF43F0010330348A4208BF16
:1000B00043F0010301F55C71A24208BF43F0010364
:1000C00004F55C748A4208BF43F001033031A24258
:1000D00008BF43F0010330348A4208BF43F00103F4
:1000E0003031A24208BF43F0010330348A4208BFD6
:1000F00043F001033031A24208BF43F001038A42BA
:1001000008BF43F0010313B9324B9A4208D10423CC
:1001100080F83530136823F001031360002038BDE8
:100120002D4B2E4D1168AA4218BF9A422C4C21F03B
:100130000E0105F13C050CBF012300231160A24212
:1001400008BF43F0010311682834AA4208BF43F0F6
:10015000010321F00101A24208BF43F0010314345E
:100160001160A24208BF43F001031E498A4208BF42
:1001700043F0010313B91C4B9A4217D10123856D3B
:10018000D0E91714226801F01F0122F480728B401D
:1001900022606B60C36ED0E91921516033B11A68D7
:1001A000D0E91C1422F480721A604C6001210022F4
:1001B000036D80F8351080F83420002BAED09847BE
:1001C000ACE700BF4000024010000240280002409F
:1001D00058000240B80402401C5402580854025807
:1001E0003054025880540258945402580168002236
:1001F0000B6880F842205A0410B40ED50B6823F423
:1002000080430B6090F84130292B10D090F841309A
:100210002A2B24D05DF8044B70471B04F2D50B68E1
:1002200023F400430B6090F84130292BEED12822B3
:10023000212380F841200022036390F841300C68AC
:1002400003F02803282B14BF6FF0F2036FF0420372
:1002500023405DF8044B0B6080F840207047282253
:10026000222380F841200022036390F841300C687B
:1002700003F02803282B14BF6FF0F4036FF044033E
:1002800023405DF8044B0B6080F84020704700BFAE
:100290000023202210B4174C4363C462036380F828
:1002A000412080F842304B07026811D5526A436AF8
:1002B0001A70436A028D013343624AB1438D013A99
:1002C000013B02859BB24385436C43F004034364C6
:1002D0000368102490F84120002190F841201A680A
:1002E00022F0FE021A60DC615DF8044B80F84010D9
:1002F000704700BF0000FFFF70B5574B002590F816
:100300004120044680F84250283AC3624585436C38
:10031000022A41EA0301036841642FD890F8411092
:1003200090F84120282001F0280102F02802282915
:1003300014BFF6214621282A1A680CBFC9436FF062
:10034000F6010A4045491A6084F84100A06B226B0F
:10035000616318B1112A42D0212A40D0E06B18B154
:10036000122A51D0222A4FD094F84130602B4FF0FE
:1003700000032DD0236384F8403070BD90F84120F5
:1003800090F841201A6822F0FE021A609A699207DA
:1003900000D59D629A69D60703D49A6942F001029A
:1003A0009A6194F84120602A10D0202284F84120DC
:1003B0009A6995060AD59A69D00605D51022DA61A0
:1003C000626C42F0040262642022DA610021BDE71F
:1003D000202284F8403084F84120236370BD1A68DD
:1003E00051042CD490F83530012BBDD000221C4B89
:1003F000036584F8402090F83520022A24D080221A
:100400004265BDE8704018471A68120403D51A689F
:1004100022F400421A6090F83530012BA4D000225B
:100420000F4B036584F8402090F83520022AE6D16E
:10043000FFF71CFE0028A0D0E06B036DE1E71A680F
:1004400022F480421A60CDE7FFF710FE002894D016
:10045000A06B036DD5E700BF0000FFFFDD040408BB
:100460002D08040803689A69196810B4D40528D5C2
:100470000C0606D4416C11F00B0F1FD15DF8044B34
:100480007047416C4FF4807441F0010141645105A3
:10049000DC6120D5416C4FF48064920541F0080185
:1004A0004164DC61E6D5426C4FF4007142F0020217
:1004B0004264D961416C11F00B0FDFD05DF8044B41
:1004C0001AE7540502D50906E4D4D3E79405D1D53B
:1004D0000906E8D4CEE79205E5D4CBE7F8B590F865
:1004E00040300D46C16A012B00F008810123AE06A1
:1004F000044680F8403001D5900656D4EB0619D555
:10050000D70617D5638D9BB2002B40F0F98094F885
:100510004130B1F1007FDBB240F0D580282B40F0B4
:10052000D28029462046FFF7B3FE0023184684F800
:100530004030F8BD68071AD42F0701D516074AD4F2
:10054000A807F2D59307F0D5638D9BB2002B00F07E
:10055000FA80616A236811F8010B228D9862638D1D
:10056000013A6162013B22859BB26385DDE7530757
:10057000E2D5638D9BB26BB12268636A526A1A70CE
:10058000638D606A228D013B0130013A9BB260624B
:1005900022856385638D9BB2002BC6D111F5803F08
:1005A000C3D02046FFF722FEBFE72368202118684A
:1005B000E66A94F84120D961213A092A1ED8DFE879
:1005C00012F0C70015001D001D001D001D001D00BC
:1005D000F000C700150094F84130226803F02803AA
:1005E000282B00F0C5800823D3619EE794F84120B2
:1005F0001A6822F0FC021A60222222635A68894992
:1006000042F400425A605A680A405A609A69910757
:1006100001D500229A629A69D20703D49A6942F0FE
:1006200001029A6147047BD51A6822F480421A605D
:10063000A26B1AB111684A6892B262856A070BD53B
:100640005A6A25F00405636A1A70636A01336362AB
:10065000238D002B40F08580638D9BB21BB1636CB2
:1006600043F004036364EB061AD5C70618D5638DFF
:100670009BB2002B40F0AA8094F84130282B03D184
:10068000B6F1007F00F0C98094F8413016F5803F44
:100690002268DBB202D0292B00F0AD801023D36199
:1006A000002384F84230666C6363002E40F084803F
:1006B000E36A5D4DAB423DD194F84130202384F88C
:1006C0004130266331E794F841202368292A4FF00E
:1006D0001002DA617FF429AF11F5803F3FF425AFB6
:1006E0009A69960701D500229A629A69D5073FF563
:1006F00058AF9A6942F001029A6152E70220F8BDB0
:1007000023681022DA61636C43F00403636431F000
:1007100080737FF40AAF616C2046FFF7EDFD04E7BC
:1007200001048BD51A6822F400421A60E26B002A99
:1007300080D183E72046FFF759FD2023E56284F846
:1007400041302663F1E631F080737FF4EEAE28E7A6
:1007500094F841201A6822F0FA021A6021222263DA
:100760004CE7013B2385638D013B9BB2638573E7B7
:10077000E1689369022990699368D56836D1C3F31B
:10078000C21383EA104313F006032FD1A16C013189
:10079000A164A16C02297FF4C8AE0821A364D161D1
:1007A000C3E694F8412094F841201A6822F0FE0232
:1007B0001A600022226321E7616C2046FFF79CFD4E
:1007C00094F84130282B7FF4B0AEAAE623681022BB
:1007D000DA61636C43F00403636436F080737FF482
:1007E0005FAF616C2046FFF787FD59E7136823F080
:1007F000B803136099E61023D3619369980701D574
:10080000002393629369D90703D4936943F00103EA
:1008100093612046FFF7EAFC42E729462046FFF7AE
:1008200037FD3DE700E800FE0000FFFF836B9A6B99
:100830000AB100211165DA6B0AB10021116593F844
:100840004120602A05D000221A63002283F840204C
:1008500070470022202183F841101A63002283F898
:1008600040207047016870B4CC072DD5914A1369B8
:10087000926A03F03803102B00F0E180182B00F08F
:10088000D9804368B3F5803F00F00581002B00F06C
:100890005A81B3F5A02F874B1A6800F0678222F4C3
:1008A00080321A601A6822F480221A60824B41F268
:1008B000883C804C1D6804E01A68521B624500F2B7
:1008C0003F8122689603F7D58A0768D4CD0631D5D3
:1008D000784A1369926A03F03803082B00F0C0804D
:1008E000182B00F0B880C369724C002B00F05F81B8
:1008F0002268714B42F0800222601D6804E01A6891
:10090000521B022A00F21C812268D205F7D56B4BDC
:10091000026A1D6841F20303B3EB154FC0F0448235
:100920006368202A23F0F8430CBF43F0804343EA76
:10093000826363600D0713D543695E4C002B00F0A2
:100940001881626F5C4B42F0010262671D6804E02F
:100950001A68521B022A00F2F380626F9207F7D5E1
:100960008C0613D58369534C002B00F0118122684B
:10097000514B42F4805222601D6804E01A68521BF9
:10098000022A00F2DD8022689204F7D5490700F1BF
:100990008880436A002B40F0BC80002059E0454A23
:1009A0001369926A13F038032BD1424AC368126864
:1009B000520701D5002B4BD03E4C226822F0190281
:1009C0001A433D4B22601D6804E01A68521B022A3C
:1009D00000F2B68022685607F7D5384B02691D68C9
:1009E00041F20303B3EB154F6368C0F0028123F4B7
:1009F0007C33402A0CBF43F4003343EA0233636084
:100A000064E7182B00F0F180C3682A4C002B00F03B
:100A1000DD80226822F019021A43274B22601D68EC
:100A200004E01A68521B022A00F28A8022685207E8
:100A3000F7D5D2E702F00302022A7FF422AF1D4B62
:100A40001B689B037FF540AF4368002B7FF43CAFEE
:100A5000012070BC704702F00302012A7FF443AF0B
:100A6000144B1B68DC0502D5C369802BF0D1134CF5
:100A700041F20303026A2468B3EB144FC0F0BF8055
:100A8000202A00F09E810B4C636823F0F84343EA70
:100A9000826363604EE7074A136843F48033136050
:100AA00004E70749044B0A6842F480720A601C6834
:100AB0000CE000BF00440258802C00240010005CB1
:100AC000004802581A68121B642A39D80A68D505EA
:100AD000F8D58268012A00F06E81002A00F04E816C
:100AE000052A9F4A116F00F0748121F001011167FE
:100AF000116F21F0040111671D6841F28834984993
:100B000003E01A68521BA2421AD80A6F9207F8D55E
:100B10003FE793490A6902F03802182A00F0D580AD
:100B20000A68022B8F4B22F080720A606FD018681F
:100B30000A6892017FF531AF1A68121A022AF7D9B2
:100B4000032070BC7047864C41F28835854B226883
:100B500022F480322260226822F4802222601E6801
:100B600003E01A68921BAA42EAD822689203F8D4DA
:100B7000AAE6626F7B4B22F0010262671D6803E008
:100B80001A68521B022ADBD8626F9607F8D4E7E690
:100B90002268744B22F4805222601D6803E01A68B8
:100BA000521B022ACCD822689604F8D4EEE62268BA
:100BB0006C4B22F0800222601D6803E01A68521B11
:100BC000022ABDD82268D605F8D4B3E62268654B60
:100BD00022F0010222601D6803E01A68521B022AFB
:100BE000AED822685607F8D470E694077FF40CAFAD
:100BF000DBE623F0FE4343EA0263636066E6584C9B
:100C0000E36823F07C5343EA0263E36092E61C68E6
:100C100003E01A68121B022A92D80A689501F8D4D8
:100C20008C6A514A2240846A2243C46A42EA04120E
:100C30008A62D0E90D24013A013C5202240492B2A6
:100C400004F4FE042243046B013CC4F30804224371
:100C5000C46B013C240604F0FE4422430A63CA6AC2
:100C600022F00102CA624A6B846C6FF3CF0242EA3F
:100C7000C4024A63CA6A046C22F00C022243384C54
:100C8000CA62CA6A406C22F002020243CA62CA6A9D
:100C900042F48032CA62CA6A42F40032CA62CA6A44
:100CA00042F48022CA62CA6A42F00102CA620A6839
:100CB00042F080720A601968226890013FF56DAEBB
:100CC0001A68521A022AF7D93AE7012B8A6A0D6B81
:100CD0003FF4BEAE02F00303846AA3427FF4B8AED1
:100CE000C2F30512C36A9A427FF4B2AE036BC5F336
:100CF0000802013B9A427FF4ABAE436BC5F3462238
:100D0000013B9A427FF4A4AE836BC5F30642013BDC
:100D10009A427FF49DAEC36BC5F30665013B9D42CD
:100D20007FF496AE4B6B816CC3F3CC0399423FF4D6
:100D300034AE0B480B4BC26A22F00102C2621A6841
:100D400018688242FCD0064A536B6FF3CF0343EA24
:100D5000C1035363D36A43F00103D3621DE600BFAE
:100D600000440258802C00240CFCFFFF42F4802237
:100D70001A601A6842F480321A6097E5194941F204
:100D800088350A6F22F001020A670A6F22F0040216
:100D90000A671C6804E01A68121BAA423FF6D0AE2C
:100DA0000A6F9607F7D4F4E5E36823F07C5343EA2F
:100DB0000263E360BEE50B490A6F42F001020A6775
:100DC0009AE6084A536823F0F84343F0804353609F
:100DD000B0E541F004011167116F41F001011167A5
:100DE0008AE600BF00440258334B30B4996A9C6ACB
:100DF000DD6A14F47C7F5A6BC4F3051036D0C2F35D
:100E0000CC0205F0010501F0030107EE900A05FB95
:100E100002F20129B8EEE77A06EE902AFAEEE96AC4
:100E200002D0022942D019B3DFED247A87EE876A17
:100E30001B6BC3F3080307EE903AF7EE005AF8EE87
:100E4000E77A77EEA67A77EEA57A67EE867A1A4B7E
:100E50001B6BC3F34623013307EE103AF8EEC76A63
:100E600087EEA67AFCEEC77A17EE900A30BC704780
:100E70001A6892061DD51968F7EE005A104A1B6BC6
:100E8000C1F3C101C3F30803CA4007EE903A06EE6E
:100E9000102AF8EEE77AB8EEC66A77EEA66AC6EED2
:100EA000077A36EEA57A67EE877AD0E7DFED057A26
:100EB000BCE7DFED057AB9E7004402580024744A24
:100EC0000090D00320BCBE4B0024744C344A1368FD
:100ED00030B423F08063334C1360256803E023684B
:100EE0005B1B022B54D813681B01F8D4936A056866
:100EF00023F47C3343EA053393628368C568013B7E
:100F0000013D5B022D049BB205F4FE052B434568B1
:100F1000013DC5F308052B430569013D2D0605F08C
:100F2000FE452B439363D36A456923F0C0032B43EB
:100F3000D362D36A856923F020032B43D362D36A3B
:100F400023F01003D362D36BC0696FF3CF0343EA7E
:100F5000C003D363D36A43F01003D362D36AD1B121
:100F600001290CBF43F4801343F40013D3620C4AED
:100F7000136843F080631360216803E023685B1A01
:100F8000022B05D813681B01F8D5002030BC704730
:100F9000032030BC704743F40023D362E7E700BF6F
:100FA00000440258802C0024344A136830B423F0E3
:100FB0008053334C1360256803E023685B1B022BCE
:100FC00054D813689B00F8D4936A056823F07C73A7
:100FD00043EA055393628368C568013B013D5B02A8
:100FE0002D049BB205F4FE052B434568013DC5F376
:100FF00008052B430569013D2D0605F0FE452B43F1
:101000001364D36A456923F440632B43D362D36AE4
:10101000856923F400732B43D362D36A23F480736E
:10102000D362536CC0696FF3CF0343EAC0035364C8
:10103000D36A43F48073D362D36AD1B101290CBF60
:1010400043F4000343F08073D3620C4A136843F007
:1010500080531360216803E023685B1A022B05D8D4
:1010600013689B00F8D5002030BC7047032030BCCB
:10107000704743F48003D362E7E700BF004402589F
:10108000802C00242DE9F843D0E9004806462501CC
:1010900000F17C830027E0050CD5D6F85890B9F113
:1010A000040F06D8DFE819F0E00356052505E5032F
:1010B000E50301273D46A10526D5D6F85C90B9F198
:1010C000800F00F0298500F26686B9F1000F00F06C
:1010D000D684B9F1400F40F06686914B9B6A03F0CD
:1010E0000303032B00F05F86002106F10800FFF7E1
:1010F000EDFE0546002D40F0CA84894A136D23F4A5
:10110000E07343EA09031365620526D5D6F8A89073
:10111000B9F5800F00F00F8500F24986B9F1000F94
:1011200000F09784B9F5001F40F049867C4B9B6A1C
:1011300003F00303032B00F04286002106F10800B0
:10114000FFF7C4FE0546002D40F08B84744A936D72
:1011500023F4600343EA09039365230526D5D6F8F3
:10116000AC90B9F1007F00F0A28400F20186B9F1E1
:10117000000F00F0FD84B9F1807F40F00186684BDC
:101180009B6A03F00303032B00F0FA85002106F1AC
:101190000800FFF79BFE0546002D40F09884604A4A
:1011A000936D23F0E06343EA09039365A0011DD525
:1011B000D6F84C90B9F1200F00F0AE8300F20F8604
:1011C000B9F1000F08D0B9F1100F40F00C86544A65
:1011D000D36A43F40033D362002D40F07383504A46
:1011E000D36C23F0300343EA0903D364E10426D52A
:1011F000D6F86090B9F5005F00F06C8400F2E385EA
:10120000B9F1000F00F03084B9F5805F40F0E3855C
:10121000434B9B6A03F00303032B00F0DC850021A2
:1012200006F10800FFF752FE0546002D40F0248429
:101230003B4A136D23F4E04343EA09031365A20418
:1012400025D5D6F86490B9F5003F00F0878300F209
:101250008185B9F1000F10D0B9F5803F40F0848549
:101260002F4B9B6A03F00303032B00F07D850121C4
:1012700006F10800FFF72AFE0546002D40F08184A4
:10128000274A136D23F4E02343EA0903136563043B
:1012900025D5D6F8B090B9F1005F00F02C8300F2AC
:1012A0002F85B9F1000F10D0B9F1805F40F0328581
:1012B0001B4B9B6A03F00303032B00F02B850121DA
:1012C00006F10800FFF702FE0546002D40F0668497
:1012D000134A936D23F0E04343EA09039365200426
:1012E0000FD5D6F87090B9F1805F00F02482B9F183
:1012F000005F00F08085B9F1000F00F02182012726
:101300003D46E1011DD5D6F84890B9F1030F00F232
:10131000B985DFE819F00C00070034030C0000BFAA
:10132000004402583E4AD36A43F40033D362002D8E
:1013300040F0C6823A4AD36C23F0030343EA090320
:10134000D364620200F14F82E30731D5D6F87C9076
:10135000B9F1280F2AD8DFE819F00E022900290078
:10136000290029002900290029000102290029005B
:101370002900290029002900290048042900290002
:10138000290029002900290029000E02290029002E
:10139000290029002900290029000E02290029001E
:1013A000290029002900290029000E0201273D46B5
:1013B000A00724D5D6F87890B9F1050F00F254852E
:1013C000DFE819F0130006000204130013001300F5
:1013D000134B9B6A03F00303032B00F045850121A7
:1013E00006F10800FFF772FD0546002D40F0D0839E
:1013F0000B4A536D23F0070343EA09035365610762
:1014000027D5D6F89490B9F1050F00F22985DFE8C9
:1014100019F016000900CA0316001600160000BFD6
:1014200000440258B14B9B6A03F00303032B00F006
:101430001785012106F10800FFF748FD0546002D3C
:1014400040F0A483A94A936D23F0070343EA0903FC
:101450009365A20625D5D6F89090B9F1005F00F00B
:101460009F8200F23C84B9F1000F10D0B9F1805F87
:1014700040F03F849D4B9B6A03F00303032B00F075
:101480003884002106F10800FFF720FD0546002DF5
:1014900040F07583954A536D23F0E04343EA090316
:1014A0005365630625D5D6F89C90B9F5006F00F01A
:1014B000888200F23384B9F1000F10D0B9F5806F43
:1014C00040F03684894B9B6A03F00303032B00F042
:1014D0002F84002106F10800FFF7F8FC0546002DD7
:1014E00040F05A83814A936D23F4E05343EA0903A1
:1014F0009365200625D5D6F8A090B9F5804F00F069
:10150000778200F21984B9F1000F10D0B9F5005FAD
:1015100040F01C84754B9B6A03F00303032B00F01F
:101520001584002106F10800FFF7D0FC0546002DC8
:1015300040F037836D4A936D23F4604343EA090317
:10154000936521070CD5D6F88490B9F5805F00F03B
:101550007082664A536D23F4405343EA090353658E
:10156000E2060CD5D6F89890B9F5807F00F051824C
:101570005E4A936D23F4407343EA090393652303A2
:1015800023D5D6F8A490B9F5803F00F0D681B9F5FF
:10159000003F10D0B9F1000F40F0DD80534B9B6A43
:1015A00003F00303032B00F0D680494606F1080040
:1015B000FFF78CFC0546002D40F0EC824B4A936D02
:1015C00023F4403343EA0903936560030FD5D6F84B
:1015D0008890B9F5001F00F07D81B9F5401F00F03B
:1015E000F880B9F5801F00F0EF8001273D46E10348
:1015F0001FD5D6F85090B9F1000F00F04681B9F52B
:10160000803F40F08580394B9B6A03F00303032B36
:101610007ED0022106F10800FFF758FC0546002D98
:1016200040F03B81314AD36C23F4803343EA090311
:10163000D364A20070D4A3035AD43D46E70206D572
:101640002A4A716F136D23F000430B431365E000CA
:1016500007D5264AD6F8B810136923F480430B4304
:101660001361A10206D5214AF16E136D23F0807338
:101670000B431365620009D51C4B1A6922F4004222
:101680001A611A69D6F8BC100A431A61002C06DAEE
:10169000164A716DD36C23F040530B43D36423027D
:1016A00007D5124AD6F88C10536D23F440030B4330
:1016B000536518F0010F40F0028318F0020F40F05C
:1016C000DB8218F0040F40F0EA8218F0080F40F0B7
:1016D000C28218F0100F40F0AE8218F0200F40F0D8
:1016E0009982281E18BF0120BDE8F88300440258E3
:1016F000D6F88030B3F5807F00F0D18040F2E680EC
:1017000023F48072B2F5007F00F0CE80012595E7CA
:101710000127A2003D468ED5B24B9B6A03F003031E
:10172000032B06D0022106F12800FFF73DFC00281C
:1017300081D001277FE7AB4AD36A43F40033D362F9
:10174000002D40F0BB80A74A136D23F0405343EABD
:1017500009031365D5E501273D4636E7A14B9B6A92
:1017600003F00303032B3FF421AE012106F108002F
:10177000FFF7ACFB0546002D40F00682994A536DF9
:1017800023F0380343EA0903536511E6856EB5F586
:10179000001F00F0558300F2F782002D00F07A81DF
:1017A000B5F5801F40F0F4828E4B9B6A03F0030373
:1017B000032B00F0ED8202210830FFF787FB07467C
:1017C000002F00F06C8166E4864AD36A43F400334C
:1017D000D362002D78D1834A536D23F4401343EA3A
:1017E0000903536503E7804A8049136843F4807313
:1017F0001360086804E00B681B1A642B00F2F78280
:101800001368DB05F7D5002D40F04F83754BD6F8F4
:10181000B420186F504010F4407F0FD0186FD3F8E9
:1018200070C020F440704CF4803CC3F870C0D3F812
:1018300070C02CF4803CC3F870C01867B2F5807F8C
:1018400000F0248302F44073B3F5407F00F010836E
:1018500064490B6923F47C530B61624BC2F30B02A6
:10186000196F0A431A676FE55E4AD36A43F400337F
:10187000D3623D46002D40F04C815A4A136D23F04F
:10188000070343EA0903136515E4564AD36A43F490
:101890000033D362002D3FF4C5AE2F46C9E651494F
:1018A000CA6A42F40032CA62002D7FF4C7AE4D49C5
:1018B0004A6D22F4407213434B65BEE62F4620E585
:1018C0002F463EE52F4691E42F4690E6002B7FF40D
:1018D0001DAFE9E7434B9B6A03F00303032B3FF47F
:1018E00084AE012106F12800FFF75EFB0546002DBE
:1018F0003FF471AFE8E73B4B9B6A03F00303032B14
:1019000000F00882012106F12800FFF74DFB054693
:10191000002D3FF4DDAC41E1324B9B6A03F0030341
:10192000032B00F06082022106F10800FFF7CEFAD7
:101930000546002D3FF453ACC4E72A4B9B6A03F0E5
:101940000303032B3FF407AF022106F12800FFF742
:101950002BFB0546002D3FF431AE1BE1214B9B6A6A
:1019600003F00303032B00F0FF81012106F128009F
:10197000FFF71AFB0546002D3FF482AC01E1194B3D
:101980009B6A03F00303032B00F07C82022106F123
:101990000800FFF79BFA0546002D3FF4CBAC8FE71C
:1019A000104B9B6A03F00303032B00F0A28102217A
:1019B00006F12800FFF7F8FA0546002D3FF46AAD5E
:1019C000DDE0084B9B6A03F00303032B00F0B081BA
:1019D000022106F12800FFF7E7FA0546002D3FF443
:1019E00081ADD9E00044025800480258802C002400
:1019F000C24B9B6A03F00303032B00F0A781022173
:101A000006F12800FFF7D0FA0546002D3FF492AD0D
:101A1000C7E0BA4B9B6A03F00303032B07D00221F4
:101A200006F12800FFF7C0FA00283FF4A1AD012716
:101A30009EE5B24B9B6A03F00303032B07D0022100
:101A400006F12800FFF7B0FA00283FF482AD012725
:101A50007FE5AA4AD36A43F40033D362002D3FF4F2
:101A600075AB2F46FFF779BBA44AD36A43F4003322
:101A7000D362002D3FF4DCAB2F46FFF7E0BB9F4A5B
:101A8000D36A43F40033D362002D3FF436AB2F46C4
:101A9000FFF73ABB994AD36A43F40033D362974ABB
:101AA000136D23F440132B431365FFF7F3BA934BE5
:101AB0009B6A03F00303032B00F06281002106F10F
:101AC0002800FFF771FA0546002D3FF468AB2F465A
:101AD000FFF76CBB894B9B6A03F00303032B00F0F9
:101AE0007A81002106F12800FFF75EFA0546FFF72C
:101AF0009CBB824B9B6A03F00303032B3FF4D9AAE0
:101B0000002106F12800FFF74FFA0546002D3FF4AB
:101B1000B4AE2F46FFF7CFBA784B9B6A03F00303AE
:101B2000032B00F04081002106F12800FFF73CFA6A
:101B30000546FFF7DFBA714B9B6A03F00303032BE3
:101B400000F03D81002106F12800FFF72DFA05463F
:101B5000FFF7F9BA694B9B6A03F00303032B3FF4C9
:101B6000A8AA002106F10800FFF7B0F9054681E6B2
:101B7000624AD36A43F40033D362FFF70DBB2F46AA
:101B80008FE42F46FFF783BB2F4611E42F4660E416
:101B90002F4634E42F4618E52F46AAE42F46FFF7D8
:101BA0009EBB2F46CDE4554B9B6A03F00303032BEA
:101BB00000F05681012106F12800FFF7F5F90546EE
:101BC000002D3FF43FACE1E74C4B9B6A03F003036D
:101BD000032B00F04981012106F12800FFF7E4F909
:101BE0000546002D3FF404ACD2E7444B9B6A03F05A
:101BF0000303032B3FF4DAAB012106F12800FFF7C2
:101C0000D3F90546002D3FF4B9ADBDE7012518F025
:101C1000200F0DD0394B9B6A03F00303032B07D031
:101C2000022106F12800FFF7BFF900283FF459AD63
:101C30000120BDE8F883314B9B6A03F00303032BBB
:101C4000E4D0012106F12800FFF7AEF900283FF4A7
:101C500044AD0546DBE7294B9B6A03F00303032BE6
:101C600000F0DE80002106F12800FFF79DF9002832
:101C70003FF42FAD0546D4E0204B9B6A03F00303ED
:101C8000032B00F0CB80012106F10800FFF71EF9BD
:101C9000002818BF054618F0040F3FF416AD174B87
:101CA0009B6A03F00303032B00F0C880022106F1B6
:101CB0000800FFF70BF9002818BF054605E50F4B94
:101CC0009B6A03F00303032B00F0A680002106F1BA
:101CD0000800FFF7FBF8002818BF0546EDE429F0DF
:101CE0008053B3F1804F3FF4D2ABB9F1405F3FF482
:101CF000CEAB01273D46FFF7D4BB00BF00440258DE
:101D000029F08053B3F1804F3FF4DFAAB9F1405F6F
:101D10003FF4DBAA01273D46FFF7E1BA29F48063CF
:101D2000B3F5805F3FF4DBABB9F5406F3FF4D7AB61
:101D300001273D46FFF7DDBB29F40053B3F5004F03
:101D40003FF4F5ABB9F5C04F3FF4F1AB01273D4689
:101D5000FFF7F7BB29F48033B3F5802F3FF48DAA4A
:101D6000B9F5403F3FF489AA01273D46FFF78FBAF6
:101D7000B9F1407F3FF410AAB9F1806F3FF40CAA8B
:101D800001273D46FFF712BAB5F5401F3FF487AE75
:101D90000127FFF780B9B9F1C00F3FF4ABA9B9F53E
:101DA000807F3FF4A7A901273D46FFF7ADB9B9F5FC
:101DB000C00F3FF4C8A9B9F5000F3FF4C4A901272B
:101DC0003D46FFF7CAB9B9F5405F3FF42EAAB9F511
:101DD000804F3FF42AAA01273D46FFF730BAB9F1F8
:101DE000300F3FF4F9A901273D46FFF7FFB903275C
:101DF0003D46FFF7A9BA2E4B9B6A03F00303032B62
:101E00003FF47DAA012106F10800FFF75FF80546BF
:101E1000002D3FF498AC51E501254EE4012550E436
:101E2000012518F0100F08F010037FF404AF08F03C
:101E3000200853EA08033FF4FBAEEBE6012544E437
:101E40001B4B9B6A03F00303032BA1D00221283014
:101E5000FFF7AAF80746002F3FF421AEFFF71BB9A2
:101E600001273D46FFF7F5BA01273D46FFF7C7BA00
:101E70000F48104B016903EA121321F47C510B4304
:101E80000361EAE401273D46FFF75BBAD1F800E0C1
:101E900041F2883C064804E00B68A3EB0E0363455F
:101EA000A5D8036F9B07F7D5D2E42F46FFF74CBAAE
:101EB00000440258CFFFFF00836A1A0710B406D50A
:101EC0000168846B4A6822F4004222434A60DC07BE
:101ED00006D50168C46A4A6822F4003222434A6087
:101EE000990706D50168046B4A6822F480322243C0
:101EF0004A605A0706D50168446B4A6822F480227A
:101F000022434A60DC0606D50168C46B8A6822F465
:101F1000805222438A60990606D50168046C8A685B
:101F200022F4005222438A605A060AD50168446CA2
:101F30004A68B4F5801F22F4801242EA04024A6023
:101F40000BD01B0606D50268C16C536823F400232E
:101F50000B4353605DF8044B70474A68846C22F46D
:101F6000C00222434A60ECE70022836BA3F85E20A4
:101F7000704700BF124B41F2883C124A01461B6871
:101F8000A2FB03235B0A0CFB03F33BB14A6B12F089
:101F9000450F01D0920404D5013BF7D14FF000402A
:101FA00070474B6B5B0707D4486B10F0010014BF00
:101FB0000123054B8B637047042318468B637047DE
:101FC00000000024D34D6210C50020000369426860
:101FD0001F2B70B432D9A3F1200520245168AC40E6
:101FE000214229D08169087C032838D0087C022846
:101FF00001D10020087448681F2BC968046906686D
:102000004D68C4F303244079164931F8100001EB00
:10201000840100F4F0508C68F16821EA0001F1605D
:102020001149085D295821F00101295011D9A3F166
:10203000200120238B40D36070BC7047202411689E
:102040009C402142F8D08169087C0328CED194605D
:10205000F2E7202101FA03F370BC93607047D4606B
:10206000EAE700BFC87D0C08387F0C08D0E90723D9
:102070009A423CBFC1685218D01A7047D0E9092370
:1020800000699A4238BF12180138D31AC01A704733
:10209000D0E90902101AB0FA80F04009704700BF79
:1020A000016A034640694A1C405CD9688A4228BFDD
:1020B00000221A62704700BF436A826910B4D1548B
:1020C000436A416B046901330A68A34228BF0023B5
:1020D0005DF8044B42F0800243620A60704700BF23
:1020E000436BD86910F0100002D0102201201A6250
:1020F000704700BF2DE9F047046982B0C3681C40F7
:1021000046D0814688464FF0004501F1500701F165
:102110003806B4FA84F325FA03F21B3BD243144089
:10212000C9F81020B8F1000F5FD0042B2ED8DFE8DB
:1021300003F052483D320300D8F81030D9F82CA0F3
:1021400033B19B6823B11FFA8AF108F10800984760
:10215000D8F8283033B19B6823B11FFA8AF108F10F
:1021600020009847D8F8403033B19B6823B11FFA5C
:102170008AF108F138009847D8F8583033B19B6895
:1021800023B11FFA8AF108F150009847002CC0D102
:1021900002B0BDE8F087D8F8103008F10800D9F88F
:1021A00034105B689847002CB3D1F1E7D8F8283099
:1021B00008F12000D9F838105B689847002CA8D1A6
:1021C000E6E7D8F840303046D9F83C105B689847CD
:1021D000002C9ED1DCE7D8F858303846D9F84010AA
:1021E0005B689847002C94D1D2E7042B07D8DFE82E
:1021F00003F01903140F0A00D9F83C300193019B36
:10220000002C86D1C4E7D9F82C300193019BF7E765
:10221000D9F834300193019BF2E7D9F838300193B3
:10222000019BEDE7D9F840300193019BE8E700BF3F
:1022300070B5124D124A2B68A2FB03239B09013B88
:10224000B3F1807F01D3012070BD4FF0E0220D4932
:1022500000240F2853614FF0F003064681F8233025
:102260004FF0070394611361EDD801464FF0FF3042
:1022700077F0B8FC20466E6070BD00BF00000024FF
:10228000D34D621000ED00E03749024603688B42EF
:1022900033D01831591AB1FA81F1490969BB334871
:1022A000834240D01830834240D01830834236D029
:1022B000183083423DD01830834240D018308342DA
:1022C0002CD000F55670834237D029498B4233D049
:1022D00018318B4236D018318B4236D018318B42B0
:1022E00036D018318B4236D018318B4236D0183167
:1022F0008B4236D023F0FF0013E0DBB21D491E48AD
:10230000103B10B41D4CA4FB03435DF8044B01EBE0
:10231000131393F82810C2E91601704716211848C4
:10232000D1659065704710211348F9E716211248CE
:10233000F6E706211248F3E706211248F0E71021DC
:102340000F48EDE710210F48EAE716210D48E7E7AF
:1023500000210D48E4E706210B48E1E710210A4877
:10236000DEE716210848DBE710000240400002408B
:1023700028040240C87D0C0800000240ABAAAAAAAB
:10238000040002400004024004040240F0B50C4680
:10239000114602688646936913F0100C72D04FF014
:1023A000000C102338486546D36193699E065FD4BC
:1023B00045B903685B1AA3423DD893699F06F8D5D7
:1023C0002023D3614CF0040C01209369D90552D528
:1023D0004FF480715F054CF0010CD16104D54FF4CE
:1023E00080614CF0080CD1619D0504D54FF4007359
:1023F0004CF0020CD3619369990701D500239362D5
:102400009369DB0703D4936943F001039361536835
:1024100020241E4901200B4000215360DEF8443087
:102420008EF8401043EA0C03CEF844308EF8414059
:102430008EF84210F0BD57689EF842309669DBB2C4
:10244000360408D57E0406D4202B04D0536843F408
:1024500080435360016893699F06A6D403685B1AA2
:10246000192BF8D993694FF0200C01259E069FD5B2
:10247000002DA5D0A6E75E05B1D49C05B6D40028F2
:10248000B9D1F0BD6046A0E7802C002400E800FE32
:102490002DE9F04707689A46089EBB6931EA0303B5
:1024A0000CBF01230023934220D180460C461546E1
:1024B000DFF85C90324651464046FFF767FF20BB8D
:1024C000D9F80030A3EB060CD44507D9BB6934EA30
:1024D00003030CBF01230023AB420AD0BB6934EADB
:1024E00003030CBF01230023AB42E3D00020BDE86F
:1024F000F087D8F84430202288F840001343C8F809
:10250000443088F8412088F842000120BDE8F08777
:10251000802C00240C4A136903F03803102B0DD0D3
:10252000182B09D063B913689B060BD513680748AD
:10253000C3F3C103D8407047FEF756BC0448704748
:102540000448704701487047004402580090D00387
:1025500040787D0100093D00184A136903F03803F3
:10256000102B10B524D0182B09D01BBB13689B0669
:1025700022D513681248C3F3C103D84001E0FEF727
:1025800033FC0E490F4A8B698969C3F303230E4C50
:1025900001F00F0113440A4493F8301092F83030E0
:1025A00001F01F0203F01F03D0402060D84010BD8F
:1025B0000648E6E70648E4E70148E2E70044025837
:1025C0000090D003C87D0C080000002440787D01F5
:1025D00000093D00474A70B4946A956AD66A15F4BA
:1025E0007C3FC5F30533D16B5BD0C1F3CC01C6F39F
:1025F000001604F0030407EE903A06FB01F1012CEB
:10260000B8EEE77A06EE901AFAEEE96A03D0022CE9
:102610006AD0002C4AD0DFED387A87EE876A936B58
:10262000C3F3080307EE903AF7EE005AF8EEE77AA4
:1026300077EEA67A77EEA57A67EE867A2D4AB7EE20
:10264000006A936BC3F3462307EE103AB8EEC77ADD
:1026500070BC37EE067AC7EE876AFCEEE66AC0ED1C
:10266000006A936BC3F3064307EE103AB8EEC77ADD
:1026700037EE067AC7EE876AFCEEE66AC0ED016ABD
:10268000936BC3F3066306EE903AF8EEE66A76EED5
:10269000866A87EEA67AFCEEC77A17EE903A8360D8
:1026A000704770BCC0E900338360704713689B06B5
:1026B0001DD51468F7EE005A936B1049C4F3C1029C
:1026C000C3F30803D14007EE903A06EE101AF8EE75
:1026D000E77AB8EEC66A77EEA66AC6EE077A36EEF5
:1026E000A57A67EE877AA9E7DFED057A95E7DFED52
:1026F000057A92E7004402580024744A0090D003FF
:1027000020BCBE4B0024744C474A70B4946A956A4E
:10271000D66A15F07C7FC5F30553516C5BD0C1F3CD
:10272000CC01C6F3002604F0030407EE903A06FB42
:1027300001F1012CB8EEE77A06EE901AFAEEE96A9A
:1027400003D0022C6AD0002C4AD0DFED387A87EE15
:10275000876A136CC3F3080307EE903AF7EE005A4A
:10276000F8EEE77A77EEA67A77EEA57A67EE867AC4
:102770002D4AB7EE006A136CC3F3462307EE103AF6
:10278000B8EEC77A70BC37EE067AC7EE876AFCEE01
:10279000E66AC0ED006A136CC3F3064307EE103A15
:1027A000B8EEC77A37EE067AC7EE876AFCEEE66ABD
:1027B000C0ED016A136CC3F3066306EE903AF8EEBF
:1027C000E66A76EE866A87EEA67AFCEEC77A17EEA0
:1027D000903A8360704770BCC0E9003383607047F3
:1027E00013689B061DD51468F7EE005A136C104948
:1027F000C4F3C102C3F30803D14007EE903A06EEDA
:10280000101AF8EEE77AB8EEC66A77EEA66AC6EE58
:10281000077A36EEA57A67EE877AA9E7DFED057AC3
:1028200095E7DFED057A92E7004402580024744AE8
:102830000090D00320BCBE4B0024744C0269836816
:1028400070B5044605681343C069626986B029689B
:102850001343AC4A03430A40616A1343E2682B60A6
:102860006B6823F440531343A2696B60A64B9D42EF
:1028700000F06681236AAE681A43A44B33401A43C2
:10288000AA60EB6A23F00F030B43EB62A04B9D425F
:1028900028D0A04B9D421AD09F4B9D4217D09F4BF2
:1028A0009D4214D09E4B9D4211D09E4B9D4219D00B
:1028B0009D4B9D420BD09D4B9D4208D00120002393
:1028C0004FF001126367A266A36706B070BD984B14
:1028D0005B6D03F00703052BF0D8DFE803F09F7F63
:1028E0008A925F79924B5B6D03F03803282BE5D811
:1028F00001A252F823F000BFA52A0408BD2804084D
:10290000BD280408BD280408BD280408BD28040803
:10291000BD280408BD280408DD290408BD280408D2
:10292000BD280408BD280408BD280408BD280408E3
:10293000BD280408BD280408F3290408BD2804089C
:10294000BD280408BD280408BD280408BD280408C3
:10295000BD280408BD280408032A0408BD2804086B
:10296000BD280408BD280408BD280408BD280408A3
:10297000BD280408BD2804089D290408BD280408B2
:10298000BD280408BD280408BD280408BD28040883
:10299000BD280408BD280408D1290408B0F5004F5B
:1029A000644853D0644B626803EB4103B3F8403092
:1029B000B0FBF3F000EB52004FF6EF73B0FBF2F018
:1029C000A0F110029A423FF679AFE860002076E766
:1029D000B0F5004F3AD04FF40040E3E7B0F5004FB8
:1029E0002DD003A8FFF7F6FD04980028EED0616A09
:1029F000D8E7B0F5004F71D06846FFF785FE019823
:102A0000F3E7B0F5004F5ED0494B1A68920639D50E
:102A10001B684A48C3F3C103D840C3E7B0F5004F71
:102A200032D0FFF799FD424A434BD269C2F30212FA
:102A3000134493F8303003F01F03D840D5E703A8C0
:102A4000FFF7C8FD04980028C0D0616A3A4B62685D
:102A500003EB41034FF6EF71B3F84030B0FBF3F0F6
:102A6000530803EB4003B3FBF2F3A3F110028A42D5
:102A70003FF624AF23F00F02C3F3420392B2134395
:102A8000EB60A3E72D488DE7FFF766FD284A2A4B48
:102A9000D269C2F30212134493F8303003F01F03DB
:102AA000D840D0E7B0F5004F1DD0FFF755FD204AC4
:102AB000214BD269C2F30222134493F8303003F061
:102AC0001F03D84091E71A4B1A68900640F1A58081
:102AD0001B681A48C3F3C103D840B7E76846FFF73D
:102AE00013FE0198AFE7FFF737FD114A124BD26989
:102AF000C2F30222134493F8303003F01F03D8408E
:102B0000A1E700BFF369FFCF000C0058FFF4FF11ED
:102B1000001001400044004000480040004C0040CC
:102B2000005000400014014000780040007C00404C
:102B30000044025800093D00C87D0C080090D003F5
:102B4000A868374B03401343364AAB60EB6A23F067
:102B50000F030B43EB62936D03F00703052B3FF666
:102B6000ADAEDFE803F0413C3303524F2D4B1A6802
:102B700095064CD42C482D4B656803EB410305EBBF
:102B80004501B3F84020B0FBF2F399423FF696AE10
:102B9000B3EB053F3FF692AE0023194680F0CEF925
:102BA0002A460902030241EA1061680818184FF02A
:102BB000000341F1000180F0C1F91D4BA0F5407206
:102BC0009A423FF67BAE1B4BD860FFE66846FFF7A4
:102BD0009BFD019800283FF4F9AE616ACBE703A89A
:102BE000FFF7F8FC0498F5E7FFF7B6FC0D4A0F4B2A
:102BF000126AC2F30212134493F8303003F01F0339
:102C0000D840E7E74FF40040B5E70B48B3E71B684F
:102C10000548C3F3C103D840ADE7034816E700BF3A
:102C2000FFF4FF11004402580090D003C87D0C0847
:102C3000FFFC0F00000C005800093D00474A70B42B
:102C4000946A956AD66A15F47C7FC5F30513516BB7
:102C50005BD0C1F3CC0106F0010604F0030407EEDB
:102C6000903A06FB01F1012CB8EEE77A06EE901AD5
:102C7000FAEEE96A4ED0022C6DD0002C4DD0DFED7B
:102C8000387A87EE876A136BC3F3080307EE903A2E
:102C9000F7EE005AF8EEE77A77EEA67A77EEA57AA5
:102CA00067EE867A2D4AB7EE006A136BC3F34623AC
:102CB00007EE103AB8EEC77A70BC37EE067AC7EE68
:102CC000876AFCEEE66AC0ED006A136BC3F3064345
:102CD00007EE103AB8EEC77A37EE067AC7EE876A83
:102CE000FCEEE66AC0ED016A136BC3F3066306EE01
:102CF000903AF8EEE66A76EE866A87EEA67AFCEE01
:102D0000C77A17EE903A8360704770BCC0E9003311
:102D100083607047DFED137AB3E713689B06AED587
:102D20001468F7EE005A136B0F49C4F3C102C3F3E2
:102D30000803D14007EE903A06EE101AF8EEE77A53
:102D4000B8EEC66A77EEA66AC6EE077A36EEA57AC0
:102D500067EE877AA6E7DFED057A92E7004402582E
:102D60000024744C0024744A0090D00320BCBE4B55
:102D7000F0B5354AB0F1804F344DA0EB0202036844
:102D8000A0EB050E4C69B2FA82F28F68BEFA8EFE95
:102D90000E684FEA52124FEA5E1E1FD0F2B9DFF8FA
:102DA000B8C0604537D00CF5806C604533D00CF569
:102DB000806C604512D0BEF1000F0FD1244D254A22
:102DC000904218BFA8422AD002F58062904226D0D5
:102DD00023F08003C76286621C4314E04D6823F031
:102DE0007003D1F80CC02B43C762866223F4407392
:102DF00043EA0C0323F080031C4312B9BEF1000F19
:102E000016D00B6903630368012243F004030360D7
:102E100042610460F0BD23F070034A681343CA683E
:102E200023F44073C7621343866223F080031C437C
:102E3000074A084B984218BF9042E2D003F58063DE
:102E40009842DED0DFE700BF0000014000040140EF
:102E5000004001400044014000040040026810B4FA
:102E600052E8003F23F4907342E800310029F7D183
:102E7000144C02F1080353E8003F234002F1080C10
:102E80004CE800310029F4D1C36E012B08D0002397
:102E900020225DF8044BC0F88C204367C36670475E
:102EA00052E8003F23F0100342E800310029EED041
:102EB00052E8003F23F0100342E800310029EFD12F
:102EC000E5E700BFFEFFFFEF436BDA69F0B5970659
:102ED00083B0044642D5586AE36AC0B2002B00F0C2
:102EE0009580216B9847636B1A681D4622F48072A7
:102EF0001A609A6822F001029A609A6942F0080208
:102F00009A61DA69D6072DD4DA69900701D50222D1
:102F10001A62DA69510701D504221A62DA691207C6
:102F200001D508221A62DA69170612D5D4F8BC2036
:102F3000212A0ED0D4E909128A4273D0A169895C92
:102F40000132C9B299622169B2FBF1F001FB102292
:102F5000A262DA69560608D403B0F0BDDA691D46EC
:102F6000D607D1D501221A62CEE7DA6940F60F0CF6
:102F70001E6804F1340012EA0C0F996836D0B24F83
:102F80000F4040F0BB80DFF8CCC216EA0C0F40F0D7
:102F90006381D4F8A050012D4CD0D50202D54F0248
:102FA00000F16781150606D501F4000106F08005E1
:102FB0000D4340F043815106CED57206CCD553E87F
:102FC000002F22F0400243E8002141B1626B52E839
:102FD000003F23F0400342E800310029F7D12022CE
:102FE0000023C4F8BC20C4F8AC30B5E79506D0D5B2
:102FF00006F0200501F080573D43CAD0D4F8A83030
:10300000002BA9D003B0BDE8F0401847E36962691E
:10301000D054E369E2680133B3FBF2F102FB1133F0
:10302000E36160E70022A4F88A201A6822F0800297
:103030001A608EE7D706B0D5F506AED51022B4F8E3
:1030400090501A629A68570640F11D81D4F8B40076
:1030500001684A6892B2002A00F05081AA4280F0CA
:103060004D81C169A4F89220B1F5807F40D053E82A
:10307000002F22F4807243E8002141B1626B52E8D4
:10308000001F21F4807142E80015002DF7D103F1F3
:10309000080252E8002F22F0010203F1080545E87A
:1030A00000210029F3D103F1080252E8002F22F099
:1030B000400203F1080545E800210029F3D1202250
:1030C000C4F8C020C4F8A01053E8002F22F010026A
:1030D00043E80026002EF7D15C490D6840B190F816
:1030E0003530022B00F01381802380F83460436573
:1030F0000223C4F8A430B4F892302DE712F0010F87
:103100000CD016F4807F09D04FF0010CC3F820C01A
:10311000D4F8C4C04CF0010CC4F8C4C012F0020FC3
:103120007BD112F0040F0CD011F0010F09D04FF039
:10313000040CC3F820C0D4F8C4C04CF0020CC4F88E
:10314000C4C012F0080F0CD006F0200C5CEA070C8B
:1031500007D008271F62D4F8C47047F00807C4F8E6
:10316000C47017050AD5770108D54FF400671F62B0
:10317000D4F8C43043F02003C4F8C430D4F8C430C9
:10318000002B3FF4E9AE92060CD506F0200601F0C4
:1031900080510E4306D0D4F8A8301BB10190984757
:1031A000656B0198D4F8C420AB6802F0280203F0E4
:1031B0004003134361D0FFF751FEAB685B067FF518
:1031C000CBAE05F1080353E8003F23F0400305F1BF
:1031D000080141E8003262B1626B02F1080353E872
:1031E000003F23F0400302F1080040E800310029CD
:1031F000F3D1D4F8B40000283FF4AEAE90F83520F7
:10320000134B022A03653BD1FCF730FF00283FF443
:10321000A3AED4F8B400036DF4E611F0010F90D022
:103220004FF0020C12F0040FC3F820C0D4F8C4C051
:103230004CF0040CC4F8C4C083D078E7D4F8AC30A8
:10324000002B7FF4DFAE87E601000010802C002405
:10325000691F04082001000412F0010F3FF471AF50
:1032600016F4807F7FF450AF12F0020F7FF469AF45
:1032700057E74FF480121A626EE6C4F8C4306BE66A
:1032800080224265BEE6B4F89220B4F8921092B261
:1032900089B2AA423FF460AE00293FF45DAE53E824
:1032A000002F22F4907243E8002141B1626B52E892
:1032B000001F21F4907142E800100028F7D19548D2
:1032C00003F1080252E8002F024003F1080545E827
:1032D00000210029F4D12022C4F8A810C4F8C0208D
:1032E000C4F8A01053E8002F22F0100243E8002198
:1032F0000029F7D10223C4F8A4302DE6AA427FF4B6
:103300002BAEC369B3F5807F7FF426AEF2E7036886
:10331000814A824E824FB34218BF934206F118068B
:103320000CBF01220022B34208BF42F0010218364E
:10333000B34208BF42F001021836B34208BF42F060
:1033400001021836B34208BF42F0010206F5567674
:10335000B34208BF42F001021836B34208BF42F040
:1033600001021836B34208BF42F001021836B342D8
:1033700008BF42F001021836B34208BF42F0010212
:103380001836B34208BF42F001021836B34208BFF4
:1033900042F00102A6F59266BB4218BFB34207F5A0
:1033A00092670CBF01260026BB4208BF42F0010213
:1033B00056EA020779D0D3F800C02CF01E0CC3F8EF
:1033C00000C0D3F814C02CF0800CC3F814C0D0F89F
:1033D00060C076BBD0F860C0DCF8006026F4807670
:1033E000CCF800601A6822F001021A6003E00A6853
:1033F000521B052A24D81A68D607F8D4D0E91651EA
:1034000001F01F012FB33F238B40AB60C36ED0E9A7
:103410001921516033B11A68016F22F480721A6069
:10342000436F4B600122002380F8352080F8343050
:103430005EE6DCF8002022F48072CCF80020D1E7B0
:10344000202103220023416580F8343080F83520A4
:103450004EE6344A344EB34218BF934206F1140686
:103460000CBF01220022B34208BF42F00102143611
:10347000B34208BF42F001021436B34208BF42F023
:1034800001021436B34208BF42F00102012606FAD7
:1034900001F1696025498B4208BF42F00102002A10
:1034A000B4D1234A9342B1D0BCE71E4EDFF878C0B6
:1034B000634518BFB3420CF1140C0CBF0126002663
:1034C000634508BF46F001060CF1140C634508BFC4
:1034D00046F001060CF1140C634508BF46F00106E6
:1034E0000CF1140C634508BF46F00106D3F800C088
:1034F0002CF00E0CC3F800C0DFF830C0634508BFE5
:1035000046F00106002E7FF465AF094EB3423FF44A
:1035100061AF67E7FEFFFFEF400002405800024046
:1035200028000240085402581C5402588054025883
:10353000945402584B4B10B41B684B4CA4FB0343F0
:103540005B0A03FB02F25AB18446531E4748DCF87B
:103550003420013B024201D0920406D55C1CF6D116
:103560004FF000405DF8044B7047DCF834305C07E6
:1035700041D4DCF83430D80709D43D4BCCF838308E
:10358000DCF81030DBB2994205D00120EAE70123D4
:10359000CCF83830F9E7DCF8143036481840002809
:1035A000E0D0002B2CDB5A002DD49C002DD4D90068
:1035B0002DD41A012ED45C012FD4D90130D41A0293
:1035C00031D45C0232D499023CD4DA0237D45C03A1
:1035D00032D499032DD4DA0340D41C043BD45904CB
:1035E00036D49A0431D413F0080F0CBF4FF4803056
:1035F0004FF40000B6E704231846CCF83830B1E7A2
:103600004FF00070AEE74020ACE78020AAE74FF40F
:103610008070A7E74FF40070A4E74FF48060A1E743
:103620004FF400609EE74FF480509BE74FF400504A
:1036300098E74FF4802095E74FF4003092E74FF47D
:1036400000408FE74FF480408CE74FF4800089E71B
:103650004FF4001086E74FF4801083E74FF400200A
:1036600080E700BF00000024D34D62104500200019
:10367000C500200008E0FFFD82B00023019302E0B6
:103680000369002B09DB019B01330193019BB3F11B
:10369000706FF5D9032002B070478901002341F013
:1036A00020010193016103E0036913F0200307D0B7
:1036B000019B01330193019BB3F1706FF4D9E9E7EA
:1036C000184602B0704700BF82B00023019302E0A9
:1036D0000369002B09DB019B01330193019BB3F1CB
:1036E000706FF5D9032002B07047002210230192B9
:1036F000036103E0036913F0100307D0019B01335A
:103700000193019BB3F1706FF4D9EBE7184602B057
:10371000704700BF82B00023019302E00369002BD1
:1037200009DB019B01330193019BB3F1706FF5D964
:10373000032002B0704700230193036943F00103A3
:10374000036103E0036913F0010307D0019B013318
:103750000193019BB3F1706FF4D9E9E71846E8E7EC
:103760002DE9F843056807460C46C5F31009B9F181
:10377000000F35D1844B4FF6FF72B3F8803093427F
:103780004FD0002B4DD0814A02EA432808F100684F
:10379000454534BF4FF001084FF002087C4B9D4275
:1037A00006D903F500339D4200F2C4804FF00109B1
:1037B000784E337E012B0FD00123B8F1010F337601
:1037C0004FF00003F36132D0022076F0B7F9002801
:1037D00000F09180002333764FF0FF30BDE8F8838E
:1037E0006C4E337E012B49D00123337605F17843AB
:1037F000B3F5801F46D3A5F10163B3F5801F3DD219
:1038000000230220F36176F099F900286DD1624A15
:103810004FF00208D2F80C3143EA0803C2F80C3129
:103820003DE0B5F1016F63D3052012F039FF40464A
:1038300076F084F90028CDD14046DFF85C81D8F8D5
:103840000C3023F4E663C8F80C30D8F80C3043EAA7
:10385000092343F0A403C8F80C3076F06FF9D8F8C8
:103860000C204E4B1340C8F80C300028B2D105F1A3
:1038700078430122B3F5801F327603D36FF0010045
:10388000BDE8F88300230120F36176F057F960BBAF
:10389000414A4FF00108D36843F00203D360BFF3FD
:1038A0006F8FBFF34F8F04F1200254F8043B944212
:1038B00045F8043BF9D1BFF36F8FBFF34F8F4046FC
:1038C00076F03CF9B8F1010F334A2ED0D2F80C3122
:1038D00023F00203C2F80C31002333760028CDD147
:1038E0003B6820333B60BDE8F88300233376C5E7AF
:1038F0004FF0010852E7DFF8A0800220D8F80C3121
:1039000023F4E663C8F80C31D8F80C3143EA0923F4
:1039100043F0A403C8F80C3176F010F9D8F80C2164
:103920001E4B1340C8F80C319FE7D36823F0020305
:10393000D360D1E703F500339D4211D903F500337D
:103940009D4210D903F500339D4206D903F500339B
:103950009D420BD84FF005092AE74FF0040927E7ED
:103960004FF0020924E74FF0030921E703F5003384
:103970009D4206D9B5F1016FBFF456AF4FF007096C
:1039800016E74FF0060913E700E8F11F00FE1F00DD
:10399000FFFF0108802C002400200052FBF8FFFFED
:1039A0000148FCF75FBD00BFA42C0024074810B4F9
:1039B000436A846D99691A6824B1234624305DF8FE
:1039C000044B18475DF8044B704700BF802C00245F
:1039D0000148FCF747BD00BFFC2C0024074810B489
:1039E000C36FD0F8B04099691A6824B123467C307F
:1039F0005DF8044B18475DF8044B7047802C002499
:103A00000148FCF72FBD00BF542D0024084810B416
:103A1000D0F8D430D0F8084199691A6824B1234607
:103A2000D4305DF8044B18475DF8044B704700BF75
:103A3000802C00242DE9F04FDFF8409300EB400587
:103A400083B0430009EB85050093AB680193002B1D
:103A500000F051818046E88975F0FCFB287B10F06E
:103A600077F90446687B10F073F908F10103074603
:103A7000DBB2002C00F0648140F60C12A1882372A6
:103A8000E2802268002800F04F81037240F60C2388
:103A9000C38091613B68BA889A611121204609264A
:103AA00010F012F91121384610F00EF96525002C9E
:103AB00000F024812268A38811690B4200F01E8166
:103AC0001B04936112F00EF905468B4612F00AF9B9
:103AD000401B61EB0B01052871F10001F6D314B115
:103AE0002368A2889A6112F0FDF805468B4612F011
:103AF000F9F8401B61EB0B01052871F10001F6D3C9
:103B0000013ED3D11CB1A38822681B04936112F03B
:103B1000E9F805460E4612F0E5F8401B61EB060198
:103B2000052871F10001F6D31FB1BB883A681B0468
:103B3000936112F0D7F805460E4612F0D3F8401BF9
:103B400061EB0601052871F10001F6D314B1236879
:103B5000A2889A6112F0C6F805460E4612F0C2F825
:103B6000401B61EB0601052871F10001F6D317B186
:103B70003B68BA889A61009B20463E21434409EB8A
:103B80008303DC7C224610F0C1F8224638463E21F1
:103B900010F0BCF8734C5823019A03FB08435A6297
:103BA000714B9A4200F0BB80FEF7D6FC6F4BDA698E
:103BB000C2F302126E4B134493F8303003F01F032C
:103BC000D840009B434409EB83031B7C022B00F08D
:103BD000B280032B00F0AA80012B14BF4FF4C871F0
:103BE0004FF4487175F0C4FB03465822002102FBD4
:103BF0000842D1629362C2E90D11C2E9101101219C
:103C0000116392F8651001F0FF00002900F0A08018
:103C1000582123F0706224264FF4004701FB08412D
:103C200054484B6A81F865601D6825F001051D60E8
:103C30001A619A6822F400429A609F605A6822F4DE
:103C400000625A605A681043CA6B58601202D86802
:103C500020F40040D860DA6000221A60186840F052
:103C60000100186020208A6681F865004A6581F8A5
:103C7000662091F865002028C5B217D191F864003C
:103C8000012813D081F86560186820F001001860E1
:103C9000186820F48050186018681860186840F0A0
:103CA0000100186081F8655081F86420009B0221B2
:103CB0000126314F434409EB830999F812502846F5
:103CC00075F090FF05F01F036A0999F8115006FA84
:103CD00003F30221284647F8223075F083FF58236A
:103CE00003FB084405F01F036D0906FA03F347F8C8
:103CF000253084F8206003B0BDE8F08F013D2AD064
:103D000011F0F0FF83468A4611F0ECFFB0EB0B0098
:103D100061EB0A01052871F10001F5D3C7E6FEF752
:103D20001BFC124B1A6A43E79161B6E6C82175F095
:103D30001FFB034659E7642175F01AFB034654E75D
:103D400000283FF4AAAE037240F60C23C380A1E61C
:103D500082F864005CE7002C3FF4B4AEA3882268CC
:103D6000AEE600BF802C0024001C0058004402581E
:103D7000C87D0C080080000200E100E00000002483
:103D80002DE9F04F441C85B017469DF83C202CD0FF
:103D90005824DFF890831E46054600FB04F408EB28
:103DA000040393F82090B9F1000F1ED04444490059
:103DB000FF2F04F12404039100D0E6B9002A40F05B
:103DC000C180582303FB058393F86520202A03D183
:103DD000AEB94FF400729A66B8F82831284601331C
:103DE0009BB2A8F82831FFF725FE4FF0000948469E
:103DF00005B0BDE8F08F93F86530202BECD14FF083
:103E0000580A0AFB058A9AF86430012BE4D0012293
:103E1000D8F800B019234FF400418AF864202046F6
:103E2000CDF800B0FEF734FB0028D5D10E9BDAF8B0
:103E30002410CAF848302123B44A8AF86530402358
:103E4000CAF858008AF86630CAF868002046AAF80E
:103E50004E604B681340039A1343AD4A1A434A60BD
:103E6000594675F03DFE0246002840F0F380DAF82E
:103E70002430802120469F620A23CDF800B0FEF74F
:103E800007FB002840F0E680BAF84E309BB2FF2BCB
:103E900040F20C81DAF82410FF239E48AAF84C3037
:103EA0004B689D4A0340039803431A434A605826CF
:103EB000DDF80CA05F46039506FB058605E0B6F825
:103EC0004E309BB2002B00F006813946204675F03B
:103ED00007FE002840F0E880B16C756A11F8012BEC
:103EE000B6F84C30AA62B164013BB6F84E109BB2F2
:103EF0000139A6F84C3089B2A6F84E10B6F84E102B
:103F000089B2002BDBD10029D9D002460A238021B7
:103F100020460097FEF7BCFAFF22002840F0C4803C
:103F2000B6F84E309BB2934240F29B80716AA6F87D
:103F30004C204B68774A1340774A43EA0A031A43F6
:103F40004A60BCE74FF0580A0AFB058A9AF86530C8
:103F5000202B7FF441AF9AF86430012B3FF43CAF43
:103F60000122D8F8007019234FF400418AF8642028
:103F700020460097FEF78CFA00287FF42DAF0E9BA9
:103F8000CAF85800CAF8483021238AF8653010234F
:103F90008AF86630CAF86800AAF84E60BAF84E305F
:103FA0009BB2FF2B00F2C080BAF84E309BB2AAF849
:103FB0004C30002B40F0E980DAF8241053484B686D
:103FC000564A0340039803431A434A605826AA46B8
:103FD00006FB0586B6F84E3039469BB2002B00F042
:103FE000CC80204675F07CFD002872D1B16C756ADA
:103FF00011F8012BB6F84C30AA62B164013BB6F857
:104000004E109BB20139A6F84C3089B2A6F84E107A
:10401000B6F84E1089B2002BDCD10029DAD0024666
:104020000A23802120460097FEF732FAFF2200285B
:104030004FD1B6F84E309BB2934223D9716AA6F89D
:104040004C204B68334A1340039A1343324A1A43B5
:104050004A60BFE75823002203FB058383F86420EE
:10406000BAE6B6F84E30726A9BB22A485168A6F892
:104070004C30DBB201404AEA03430B4343F0007388
:1040800053601CE7B6F84E30716A9BB2039A214820
:10409000A6F84C30DBB242EA03434A6802401343BD
:1040A00043F000734B6095E7039D95E6BAF84E30F8
:1040B000DAF824109BB2039A1648AAF84C30DBB207
:1040C00042EA03434A680240134343F000734B60E3
:1040D000EDE6554680E639462046039D75F0D2FC54
:1040E00000287FF479AE736A20210D4CD9615A689B
:1040F00022405A605823002286F8651003FB05838E
:1041000086F8660083F8642071E600BF009800FC22
:1041100000200101009C00FC0000FF0100200002C3
:1041200000E800FE802C0024FF234FF47F00FE22D5
:104130004FF08076AAF84C30039BDDF838E01E4340
:1041400058231EF801AB03FB0583DFF850C0596A02
:10415000C1F828A0A3F84C20B3F84E20C3F848E0DB
:10416000013A92B2A3F84E204B6803EA0C033343A2
:10417000034343F400534B6028E72046554675F04F
:1041800081FC00287FF428AEADE7013B4FF00076BC
:104190009AB2501CC0B20004CEE700BF009800FCE9
:1041A0002DE9F04F441C85B099469DF83C3000F055
:1041B00096805825C44C064600FB05F504EB050B1C
:1041C0009BF820A0BAF1000F00F089802544FF2A57
:1041D00090464FEA410705F1240540F08680002B08
:1041E00000F083809BF86530202B6FD19BF8643002
:1041F000012B6BD00122D4F8008019234FF4004129
:104200008BF864202846CDF80080FEF741F900289D
:104210005CD10E9BCBF85800CBF8483022238BF8AA
:10422000653010238BF86630CBF86800ABF84E9001
:10423000BBF84E309BB2FF2B00F21681BBF84E301C
:10424000DBF824109BB2A1484A68ABF84C30DBB2D3
:10425000024047EA034313439D4A1A434A604FF022
:10426000580909FB0649B9F84E309BB2002B00F003
:104270008681D9F824309A69520700F13381424689
:104280000A212846FEF782F8002840F0FA80D9F883
:1042900024309A69910640F1FE809A699A6912F079
:1042A000100200F0F680102220218A4DDA610422EB
:1042B000C9F86820D9615A682A405A6089F865109F
:1042C00089F8640089F8660022689B69B4F828318F
:1042D000304601339BB2A4F82831FFF7ABFB4FF017
:1042E000000A504605B0BDE8F08F4FF0580B0BFBAD
:1042F000064B9BF86530202BE8D10E9B002B00F07D
:10430000AC80B9F1000F00F0A8809BF86430012B5D
:10431000DCD0236801224FF4004128468BF864204A
:10432000039300931923FEF7B3F80028CED122237C
:10433000DBF824100E9A8BF865304023CBF8482028
:104340008BF86630CBF86800ABF84E90DFF87C91C4
:104350004A68CBF85800284602EA09023A4342F478
:1043600090324A60039975F0BBFB0246002840F08A
:104370003281402328461946DBF82430C3F82880D0
:10438000039B00930A23FEF783F8002840F0238163
:10439000BBF84E309BB2FF2B40F22481DBF8241097
:1043A000FF234D4AABF84C304B6803EA09033B430B
:1043B0001A434A604FF05808B946039F08FB064865
:1043C00005E0B8F84E309BB2002B00F01D810A23A7
:1043D0000022042128460097FEF75AF800287FF4AF
:1043E00075AFD8F82430596AD8F848301970B8F841
:1043F0004E10D8F848300139013389B2C8F8483036
:10440000B8F84C30A8F84E10013BB8F84E109BB2EB
:1044100089B2A8F84C300029D3D0002BD1D1024664
:104420000A23802128460097FEF732F8FF22002851
:104430007FF44CAFB8F84E309BB2934240F2B98053
:10444000D8F82410A8F84C204B68244A1340244A7A
:1044500043EA09031A434A60B3E758234FF4007252
:1044600003FB06439A6631E7DBF82410FF23174865
:10447000ABF84C304B68184A03403B431A434A6040
:10448000EDE6582303FB06435B6A9A6922689B6941
:104490001CE7C9F868202268A2EB08020A2A7FF606
:1044A000EAAE9A6912F004027FF4E5AE582101FBEE
:1044B0000641886E81F86420202240F02000886642
:1044C00081F865209B6901E7802C0024009800FC9E
:1044D0000024000200E800FE0024FF01009C00FC14
:1044E0000000FF015A6AD9F848301A70B9F84E3006
:1044F000D9F84820013B01329BB2C9F84820A9F8FD
:104500004E30B9F84C30B9F84E20013B92B29BB214
:10451000A9F84C30002A3FF4A6AE002B7FF4A3AEDE
:104520000A23002280212846CDF80080FDF7B0FF45
:1045300000287FF4CBAEB9F84E309BB2FF2B0CD9DC
:10454000D9F82410FF233B48A9F84C304B683A4A6D
:1045500003403B431A434A6085E6B9F84E30D9F828
:1045600024109BB233484A68A9F84C30DBB20240B1
:1045700047EA0343134343F000734B6073E641463D
:10458000284675F07FFA00287FF4A0AED9F82430D1
:1045900020212A4DD9615A682A405A6089F865104D
:1045A00089F866005822002302FB064484F8643030
:1045B00097E6B8F84E30D8F824209BB21D485168D1
:1045C000A8F84C30DBB2014049EA03430B4343F007
:1045D00000735360F5E65823002203FB064383F87B
:1045E000642073E6BBF84E30DBF824109BB24A68B7
:1045F000ABF84C30DBB202EA090247EA034313434B
:104600000F4A1A434A60D5E60399284675F03AFAEC
:10461000034600287FF45AAED8F824202020074D06
:10462000D06151682940516088F8650088F866308B
:10463000B8E700BF009C00FC0000FF0100E800FE9E
:10464000002400020248836B0BB12C3018477047DE
:10465000000000240248836D0BB14C3018477047AE
:10466000000000240248836F0BB16C30184770477C
:10467000000000240348D0F898300BB18C30184764
:10468000704700BF000000240348D0F8B8300BB1D9
:10469000AC301847704700BF000000240348D0F832
:1046A000D8300BB1CC301847704700BF0000002451
:1046B0000348D0F8F8300BB1EC301847704700BF12
:1046C000000000240348D0F8183113B100F58670BB
:1046D00018477047000000240348D0F8383113B160
:1046E00000F5967018477047000000240348D0F882
:1046F000583113B100F5A670184770470000002428
:104700000348D0F8783113B100F5B67018477047F8
:10471000000000240348D0F8983113B100F5C670AA
:1047200018477047000000240348D0F8B83113B18F
:1047300000F5D67018477047000000240348D0F8F1
:10474000D83113B100F5E670184770470000002417
:104750000348D0F8F83113B100F5F67018477047E8
:10476000000000240348D0F8183213B100F503709C
:10477000184770470000002410B41C464368844664
:104780006FF30F0323434360036843F001030360A7
:10479000036843F400730360002C3AD040F2E93020
:1047A000DCF814309B0748D5002A49D012F8013BA9
:1047B00040F2E9308CF82030DCF81430DB0720D4EC
:1047C0000138F9D1214B9C450CD0A3F578439C4589
:1047D00038D003F580639C4536D003F578439C457B
:1047E0000BD103201A4A00EB400002EBC002B2F8E2
:1047F000403201339BB2A2F8403200205DF8044BF6
:1048000070479CF83000C0B209B101F8010B013CBF
:10481000C4D1DCF814301B07FBD5DCF818300120BC
:104820005DF8044B43F01003CCF81830DCF800308E
:1048300023F00103CCF8003070470138B0D1C1E754
:10484000FF23B5E70120CDE70220CBE70030014090
:10485000000000242DE9F84300242C4E8046036814
:1048600056F83450AB4209D001340E2CF8D1284A06
:104870000021052009F030FF002019E0254B03EB53
:104880008409D9F82C71AFB198F8051000204B1CA1
:1048900001EB410203EB430307EBC202DB00C2F86A
:1048A0000C80C2E90400F854182303FB017008309F
:1048B000BDE8F8830721682009F096FF0146C9F892
:1048C0002C01F0B13946682282F0D4FFD9F82C11BE
:1048D00006EBC4043B4689600C6009628963096584
:1048E00056F83320954205D001330E2BF8D14F6096
:1048F0000F46C9E7084F4C2202FB03774F600F4673
:10490000C2E7064A052009F0E7FEB5E7207E0C085D
:1049100094280D08802C0024E42D0024BC280D08C8
:10492000F0B54468A37913F002025FD002224FF081
:10493000080C036864795B689B48204493F83C400A
:10494000012C90F8C80050D0012483F83C40142872
:1049500048D8DFE810F01500470047004700840002
:104960004700470047003B01470047004700BB00A6
:10497000470047004700F2004700470047004D004E
:1049800018688A4C056A8A4E25F00205B04242EA50
:104990000502056A25F0010505624768856904EA94
:1049A000050444F0600407D0824DA84204D005F508
:1049B0007055A84240F04D8122F0080247F440773C
:1049C0004CEA020222F00402476084614163026201
:1049D000826942F008028261826922F004028261E7
:1049E00082698261002283F83C20F0BD9446A0E7F2
:1049F00018686F4E046AB04224F4001444EA02526C
:104A0000046A24F4801404626B4C4568476D04EA20
:104A1000070444F4C0440ED006F58066B0420AD0C4
:104A2000664F06F58046B04218BFB84203D006F57F
:104A30008066B04201D145F4802545604465C1657A
:104A40000262426D42F400624265426D22F480626D
:104A50004265426D4265002283F83C20C5E7186834
:104A6000574C056A524E25F02005B04245EA021522
:104A7000026A22F0100202624768826904EA0204B4
:104A800044F4C04400F0DE804A4A904200F0DA80EC
:104A90004A4E4C4A904218BFB04203D002F58062A1
:104AA000904201D147F440674760846181630562A9
:104AB000826942F400628261826922F480628261CA
:104AC00082698261002283F83C208EE71868384EA4
:104AD000046AB04224F4005444EA0232046A24F422
:104AE00080540462364C4568C76904EA070444F4FC
:104AF000C0440ED006F58066B0420AD02F4F06F5AE
:104B00008046B04218BFB84203D006F58066B04276
:104B100001D145F480454560C46101640262C26907
:104B200042F40062C261C26922F48062C261C26959
:104B3000C261002283F83C2057E718681C4E046AC3
:104B4000B04224F4003444EA0242046A24F480347B
:104B500004621D4C4568476D04EA070444F0600494
:104B60000ED006F58066B0420AD0144F06F5804696
:104B7000B04218BFB84203D006F58066B04201D1FA
:104B800045F480354560446581650262426D42F0BE
:104B900008024265426D22F004024265426D4265A0
:104BA000002283F83C2020E7C87D0C088CFFFEFF24
:104BB0000000014000040140FF8FFFFE0040014063
:104BC000FF8CFFFE004401408FFFFEFF1868264C5B
:104BD000056A264E25F4007EB0424EEA0225026A9E
:104BE00022F4807202624768C26904EA020444F057
:104BF000600420D01E4A90421DD01E4E1E4A904294
:104C000018BFB04203D002F58062904201D147F450
:104C100040574760C461C1630562C26942F008023F
:104C2000C261C26922F00402C261C269C26100228B
:104C300083F83C20D9E625F4006E4EEA0C2E2EF4C3
:104C40008065E4E725F0800545EA0C1525F0400570
:104C500028E705F58065A8423FF4AEAE05F580650E
:104C6000A8427FF4B1AEA7E68CFFFEFF0000014032
:104C70000004014000400140004401404268537973
:104C8000032B0FD8DFE803F00B0805021068403053
:104C9000704710683C3070471068383070471068B3
:104CA0003430704700207047D0E90002064B51793C
:104CB00092790B44406893F8C810530701D57CF0F3
:104CC00039BF7CF0B3BF00BFC87D0C084268C36821
:104CD00012695B68C2F30322F0B53B4D05EB82021B
:104CE0009668EFF31182102484F312884468374FDA
:104CF00094F805C0D0F80CE035F81CC025680CF419
:104D0000F05CEC6824EA0C0417F806C0EC60DEF8EE
:104D1000105053F80C401F2D24F0010443F80C40B0
:104D200042D9203D2024DEF804C0AC40CCF80C4031
:104D3000D2B282F3118817F806C042F2107203EB68
:104D40000C0EDEF80040E40702D500BF013AF8D1AE
:104D500053F80C2012F0010223D1DEF8044045691B
:104D60006FF30F0421434468CEF8041061790329DE
:104D700005D8DFE801F02326022022683C32CEF875
:104D80000C500121CEF8082053F80C2042F01002FC
:104D900043F80C2053F80C200A4343F80C2001740C
:104DA000F0BD00230374F0BD2024DEF804C0AC4045
:104DB000CCF80840BCE722684032E0E72268343291
:104DC000DDE722683832DAE7C87D0C08387F0C0846
:104DD00003681A7E012A2ED0002293F83010012990
:104DE00009D093F8481001290ED093F860100129DA
:104DF0001BD02ABB7047022142F4806283F8301036
:104E000093F84810012904D1022142F4006283F88A
:104E1000481093F86010012907D01B6800211B6817
:104E20005962D9680A43DA607047022142F480521D
:104E300083F86010F1E702214FF400721976CCE795
:104E40004FF40072E9E700BF08B5204B98420ED03E
:104E500003F5806398420AD01D4A03F580439842C7
:104E600018BF904203D003F5806398421BD1FDF731
:104E700073FB1849184BCA69C969C2F30222C1F30E
:104E800002211A4492F8302002F01F02D040114A49
:104E90001269C2F3C03241EAC202134493F8CC3023
:104EA00003FB00F008BDFDF757FB0A490A4BCA692E
:104EB000C969C2F3021CC1F3021103EB0C0292F8A0
:104EC000302002F01F02D040E1E700BF00000140A7
:104ED0000040014000440258C87D0C0870B50E46E1
:104EE00005EE102AD0E90031013E1A680868B6B212
:104EF0005C681568FFF7A8FF07EE900AB8EE455A00
:104F00009FED5D7AF8EE677A87EE850A30EE070A44
:104F100080F006FB23680138AB4280B268D0C4E958
:104F2000005000238022E660A360A261C4E904333C
:104F300094F83D3003F0FF02002B78D00223211DAE
:104F4000284684F83D30FDF713FF4C4A0123B5F1A4
:104F5000804FA5EB020284F84830B2FA82F284F85E
:104F60003E3084F83F304FEA521284F8403084F8E3
:104F7000413084F8423084F8433084F8443084F877
:104F8000453084F8463084F8473084F83D3034D0DA
:104F90009ABB3B4B9D420CD003F580639D4208D0E9
:104FA00003F580639D4245D003F578439D4241D08F
:104FB00070BD94F83C30012BFAD00222314B012114
:104FC00084F83D20A8680340AB6084F83D1084F865
:104FD0003D206B68A96823F0700321F08001012255
:104FE0006B600023A96084F83D2084F83C3070BDDC
:104FF000636883423AD0606093E794F83C30012BB9
:10500000D6D002211F4B002084F83D10A9680B4028
:105010000121AB6084F83D10022384F83D306B68B9
:10502000A9680AB90028D6D023F47003D3E784F81E
:105030003C2083E794F83C30012BB9D00221114B7E
:10504000114884F83D10A968281A0B40B0FA80F086
:105050000121AB600023400984F83D1084F83C3006
:105060000A4B9D42D8D00028D6D170BDE368B34228
:105070007FF457AF70BD00BF0AD7233C000001404A
:10508000000400408800CEFF00040140000C0040F6
:10509000024B0348D3F82C11FDF72CB8802C0024C8
:1050A00000000140034B4FF08040D3F83011FDF772
:1050B00021B800BF802C0024024B0348D3F83411E0
:1050C000FDF718B8802C002400040040024B034870
:1050D000D3F83811FDF70EB8802C002400080040EA
:1050E000024B0348D3F83C11FDF704B8802C002490
:1050F000000C0040024B0348D3F84811FCF7FABFFC
:10510000802C002400040140024B0348D3F85811BE
:10511000FCF7F0BF802C002400180040024B03482D
:10512000D3F86411FCF7E6BF802C00240040014056
:10513000024B0348D3F86811FCF7DCBF802C002435
:1051400000440140024B0348D3F86C11FCF7D2BF76
:10515000802C00240048014010B5064C0648D4F8C5
:105160004811FCF7C7FFD4F85C110448BDE81040B3
:10517000FCF7C0BF802C002400040140001C00404C
:1051800010B5064C0648D4F84811FCF7B3FFD4F824
:1051900060110448BDE81040FCF7ACBF802C00242F
:1051A0000004014000200040BFF34F8F0549064B2B
:1051B000CA6802F4E0621343CB60BFF34F8F00BFB5
:1051C000FDE700BF00ED00E00400FA05002101202A
:1051D00008B50FF08FF872B6FFF7E6FF2DE9F04340
:1051E000BFB0BFF35F8F964C0023626A22F4803217
:1051F0006262C4F894309DF843109DF844C00906DB
:105200009DF842200F9841EA0C7141EAC2419DF895
:10521000452041EA82419DF8462041EA42419DF8FD
:10522000472041EA02419DF8412041EA02219DF8D0
:10523000402041EA4201C4F898300133D4F8A0205C
:10524000112B22F00102C4F8A020C4F89C00C4F87D
:10525000A010F0D10523C4F89430636A43F480337E
:105260006362BFF34F8FBFF36F8F7648764A7749FB
:10527000121A82F0E1F9764B5A6D012A00F0CA80C9
:10528000D4F888100022734B012041F47001C4F857
:10529000881018601A61196841F080011960196856
:1052A00001431960196841F480311960196841F4AB
:1052B000805119609A61DA611A629A62DA621A633D
:1052C0005A639A63DA631A645A64196821F4802174
:1052D00019601A664FF000635F49C1F80801A360C6
:1052E0007CF03CFF5D4AD36813F0040FD3687FD194
:1052F0005B4B0021594A0591D96A21F00101D9621D
:10530000DB6A03F001030593936943F4404393611F
:10531000936903F440430593059B93699804FCD576
:105320004422002110A84F4C82F0A4FA4E4B42F2C6
:105330000302A4F1100519684FF44040484BB2EB4A
:10534000114F4FF00C024FF4C07108BF2C46A270F1
:105350000022E0600792A180D96A404A21F0010151
:10536000D962DB6A03F001030793936903439361F6
:10537000936903400793079B93699904FCD5354BC8
:105380004FF4403539480321D3F8E02042F0800241
:10539000C3F8E020D3F8E03003F080030693002345
:1053A000069A85610D9ACDE9001201227CF084FDF8
:1053B00001204FF4803102234FF4C0721793CDE9DE
:1053C0000E010C21E079CDE91831A379217A1C90E6
:1053D0000EA81D91CDE91A2304220023CDE91E2336
:1053E000FBF740FA032800F0C281002844D0FEE712
:1053F00023F007031E4C43F00203D360216805E04D
:1054000023685B1AB3F57A7F3FF672AF53689D0449
:10541000F6D56DE70F4A002016495865D2F8F430EA
:1054200043F00203C2F8F430D2F8F43003F0020380
:105430000E930E9B0B6883F308884B689847FEE732
:1054400000ED00E00000000018390000CCA60D08B7
:1054500000400058004402580080005100480258A3
:10546000000400589C0200240010005C001C02583C
:10547000802C00240098F01F754B1A6812F00E0F54
:105480000BD11A6822F00F0242F002021A601B6868
:1054900003F00F03022B40F06C816E4A936903F016
:1054A00070033F2B05D8936923F0700343F040034A
:1054B0009361684AD36903F070033F2B05D8D36921
:1054C00023F0700343F04003D361624AD36903F4CD
:1054D000E063B3F5806F05D2D36923F4E06343F44E
:1054E0008063D3615B4A136A03F070033F2B05D8D6
:1054F000136A23F0700343F040031362554B9A691B
:10550000120705D49A6922F00F0242F008029A614C
:10551000504A936923F47063936113689B0130D5FB
:10552000136941F288314C4C23F0070343F0030325
:105530001361206804E023681B1A8B4200F2AD81DE
:10554000136903F03803182BF5D1936903F00F03A7
:10555000082B05D9936923F00F0343F008039361E7
:105560003B4A136803F00F03022B0BD9136823F097
:105570000F0343F002031360136803F00F03022BC1
:1055800000D0FEE7334A936903F07003402B05D93E
:10559000936923F0700343F0400393612D4AD3696C
:1055A00003F07003402B05D9D36923F0700343F057
:1055B0004003D361274AD36903F4E063B3F5806FF6
:1055C00005D9D36923F4E06343F48063D361214AAE
:1055D000136A03F07003402B00F2CC801D4EFCF7E1
:1055E00099FF1E4DB269B369C2F303221C4B1344E9
:1055F00093F8303003F01F0320FA03F368682B6040
:10560000FCF716FE002840F04981102315901790F2
:105610000EA80E93FBF726F9002840F0A780336808
:10562000104A43F080033360D6F8F43043F00203AD
:10563000C6F8F430D6F8F43003F002030493049B68
:10564000136A43F001031362074B216810E000BFA7
:105650000020005200440258802C00240000002446
:10566000C87D0C080004005880380100013B7ED042
:1056700022689142FAD0226823689B1A0A2BFBD930
:1056800000214FF48020A94C4FF44013002600273E
:1056900030934FF00208CDE90E010EA8FBF7F2FCA3
:1056A000D4F8EC30A24941F2030243F002030EA801
:1056B000C4F8EC30D4F8EC3003F002030393039BFE
:1056C000D4F8943043F00203C4F89430D4F8943002
:1056D00023F00203C4F894300B689649B2EB134FE1
:1056E000954B964A28BF0A465A601A6822F47C52A3
:1056F00042F400521A601A6842F060021A600322F3
:105700000023CDE92C67CDE90E23FBF7BBFC4FF45A
:10571000E04200230EA83A96CDE92667CDE90E2394
:10572000FBF7B0FC182200230EA82F963496CDE983
:105730000E23FBF7A7FC4FF480334FF4803217960B
:10574000229300230EA8CDE90E230D224FF4D0732F
:10575000CDE91566CDE9102303260423CDE9128691
:105760001493FBF78FFC074658B1FEE7FEE7FFF7FF
:105770002DFD06E7136A23F0700343F04003136224
:105780002CE7D4F8E03042464FF4807143F0010337
:10579000C4F8E030D4F8E03003F001030993099B2A
:1057A0000346CDE9006066487CF086FB23694246EB
:1057B000644823F0FE7343F088732361D4F8E0302B
:1057C00043F00403C4F8E030D4F8E03003F00403FD
:1057D00008933B4608994FF40071CDE900677CF0CF
:1057E0006BFB236923F07E4343F0FC432361FCF70A
:1057F00091FE2860BFF35F8F534C3E46534D4FF0F0
:105800000108636A23F480336362C4F8947028E06B
:10581000002A41D02F686B7A103515F8061C1B063C
:1058200043EA017343EA420315F8052C43EA824335
:1058300015F8042C43EA424315F8032CC4F8986089
:10584000013643EA0243D4F8A020032E43F00103BB
:1058500022F00102C4F8A020C4F89C70C4F8A03063
:105860001DD06B682A7A002BD2D02F68002AD2D1A3
:1058700027F01F02A3EB0209B9F1200F38BF4FF048
:105880002009484681F060FE421E08FA02F189456F
:1058900008BF0246D2B2BEE7FEE772E671E6052314
:1058A000C4F89430636A43F480336362BFF34F8F6C
:1058B000BFF36F8FBFF34F8FBFF36F8F0022C4F81A
:1058C0005022BFF34F8FBFF36F8F636943F40033F0
:1058D0006361BFF34F8FBFF36F8FC4F88420BFF3B2
:1058E0004F8FD4F8804043F6E0761749C4F34E3228
:1058F000C4F3C904520102EA0605234645EA83704F
:10590000013BC1F86002F9D2203A12F1200FF2D126
:10591000BFF34F8F4B6943F480334B61BFF34F8F1D
:10592000BFF36F8F3FB0BDE8F08300BF0044025863
:105930000010005C7FBB2200008400407FBB22304F
:10594000000002580008025800ED00E0AC020024FC
:105950002DE9F843374E984606EB8003D3F8DC4038
:10596000002C65D004F1D203FC360546B4F8D2020F
:10597000A36104F5E97366601746E3614FF4807331
:10598000261DE160C4E904332368C4F8CC30A36366
:1059900000284AD194F8D1000EF0DAF918F0080F77
:1059A00094F8D09034D1BA0723D4FB0711D4052141
:1059B00094F8D60274F016F994F8D63201221E49F2
:1059C00003F01F005B09824041F823203046BDE808
:1059D000F883013548460EF0BBF9EDB218B140F23C
:1059E00006630572C38094F8D42202210EF08EF96A
:1059F000DDE76B1CDBB218B1037240F20653C380C3
:105A000094F8D52202210EF081F9FB07CFD5E0E70B
:105A10000135EDB218B140F206730572C38094F8F7
:105A2000D52202210EF072F9C1E773F013FCB1E741
:105A30002646CBE7C87D0C0800E100E00148FDF7F1
:105A400043BA00BFE00200240148FDF73DBA00BFA1
:105A5000B80500240148FDF737BA00BF90080024BC
:105A60000148FDF731BA00BF680B00240148FDF77B
:105A70002BBA00BF400E00240148FDF725BA00BF35
:105A8000181100240148FDF71FBA00BFF0130024CD
:105A9000F8B52422456B00238168C0F8BC20044679
:105AA0002A6800F13407C66D22F001022A602B60DB
:105AB0006B60AB6090F806E0C0F8C43080F8B83096
:105AC000C0F8BC30C364C0F8C0304365C0F8A03033
:105AD000C0F8A4304FEA8E23816303F48053C3637C
:105AE0004FEA0E3303F4005303644FEA0E2303F42A
:105AF000806343644379D80703F0020253D4002A39
:105B00006FD1A264574B03F1200C53F8042F22B13C
:105B10001068D4F8C81088426FD09C45F5D11EF0AB
:105B2000080FD4F8BC3077D0002B00F097802423E6
:105B3000C4F8BC302B6823F001032B60002E40F02A
:105B400089803846FCF77AFE012812D06B68384607
:105B500023F490436B60AB6823F02203AB60AB6827
:105B600043F00803AB602B6843F001032B607BF02C
:105B700081FF6279D1070DD5D4F8C830196841F496
:105B800080711960996841F001019960196841F0CC
:105B900020011960930705D5D4F8C820136843F095
:105BA00080031360F8BD0423A36482B10C231EF0AC
:105BB000010FA364A6D04FF4803346F0020663665B
:105BC00046F001064FF40033E66523669AE71EF0BF
:105BD000010F97D046F002064FF48033E665636606
:105BE00090E708231EF0010FA3648BD046F0010656
:105BF0004FF40033E665236684E792F8D732002B32
:105C00008DD04FF4004346F008061EF0080FE366FF
:105C1000E665D4F8BC3087D1CBB12423C4F8BC30BE
:105C20002B6823F001032B606EB93846FCF706FEA3
:105C300001289ED06B68384623F490436B60AB68B4
:105C400023F02A038EE73846FCF736F9EDE784F8AF
:105C5000B830E2E73846FCF72FF972E784F8B8303D
:105C600065E700BFA07E0C08816011E741710FE776
:105C700081710DE72DE9F843434D3C20434C05F578
:105C80009872B5F83631C4F88C25A4F89835B5F873
:105C90003A21B5F83E31A4F89A25A4F890350EF0D3
:105CA00057F8074642200EF053F8064638200EF00B
:105CB0004FF881461FB10D23FB8000233B721EB1BC
:105CC0000D23F38000233372B9F1000F05D00D23AB
:105CD000A9F80630002389F80830B5F84231392098
:105CE000A4F89235B5F84631A4F89435B5F84A31A0
:105CF000A4F896350EF02CF880463A200EF028F8DD
:105D000005463B200EF024F80446B8F1000F05D0FC
:105D10000D23A8F80630002388F808301DB10D23A4
:105D2000EB8000232B721CB10D23E3800023237230
:105D300048460DF0BDFF012148460DF0C5FF404625
:105D40000DF0B6FF28460DF0B3FF20460DF0B0FF72
:105D5000404601210DF0B8FF284601210DF0B4FFA7
:105D6000012120460DF0B0FF38460DF0A1FF30466E
:105D70000DF09EFF384601210DF0A6FF30460121AF
:105D8000BDE8F8430DF0A0BFC87D0C08802C0024AE
:105D900038B5134D41F20D13124941F28832D5F84E
:105DA000E005D5F89C450004A060E068014020466D
:105DB0000B430D21E360FDF7BDFB38B1D5F8D025CD
:105DC000034600201343C5F8D03538BD606900F4A0
:105DD000F050A0F50060B0FA80F0400938BD00BF77
:105DE000802C0024C0E0FEFF2DE9F04FA74D7C225F
:105DF00000219BB005F29C5081F03CFD4FF48031B6
:105E0000D5F88C4595F8CC352268C5F8A0154FF427
:105E10000031C5F89C25C5F8AC150221C5F8B015B0
:105E2000002B00F088800422994B85F8CC25DA6C91
:105E30001B68D6030DD5180100F1D98001224FF05F
:105E4000006385F8CC25C5F8D03501201BB0BDE82E
:105E5000F08F9C01F2D50AAB18460193FCF7EEFED9
:105E60000B990029EAD0D5F89C450A0A894B666847
:105E7000A3FB0232884B894F33401009B94243EAF1
:105E800012136360236843F00303236040F2F98038
:105E90004300834AB1FBF3F3B2FBF3F22968023209
:105EA0002B685B1A9A42FBD800237E4A0493A360B6
:105EB0007D4BE16817680B4043F48053E3607B4BF4
:105EC000A3FB073741F288337F0A03FB07F73B4602
:105ED000002B00F0CB80626B013B1106F8D5744BB0
:105EE000714AA3634FF4D573A360E3681A4041F28B
:105EF00008131343E3604FB13B46626B12F0450F4A
:105F000002D0920440F1DC80013BF6D10023C5F8B9
:105F1000D835A360644BE268134043F48053E360D8
:105F20003B46002B00F0A280626B013B1106F8D5C6
:105F30005F4BA363E3E05F4B9A425FD05E4B9A42B4
:105F400000F00F8195F898050DF002FF834695F853
:105F50009A050DF0FDFE824695F890050DF0F8FECD
:105F6000814695F892050DF0F3FE804695F894056C
:105F70000DF0EEFE074695F896050DF0E9FE95F852
:105F8000992506460E2158460DF0C0FE504695F85C
:105F90009B250E210DF0BAFE484695F891250E215D
:105FA0000DF0B4FE404695F893250E210DF0AEFE9F
:105FB00095F8952538460E210DF0A8FE0E2195F88E
:105FC000972530460DF0A2FE0221B4F9040073F0CB
:105FD00009FEB4F90430002BFFF625AF03F01F00D3
:105FE00001225B093549824041F823201BE70AABB7
:105FF00018460193FCF7EEFA0C9932E7244BD3F8DC
:10600000D42022F48032C3F8D420D3F8D42042F430
:106010008032C3F8D420D3F8D42002F48032039223
:10602000039ADA6F42F48032DA67DA6F22F4803250
:10603000DA6787E72A684FEA134EA2EB0902734634
:10604000824213D8002B40F03181C4F808E0E368A5
:1060500003EA0A030B43E3603B46626B12F0450F11
:1060600002D0920440F1F080013BF6D14FF00040A5
:10607000012385F8CC35D5F8D0350343C5F8D035A4
:10608000E3E6074AB2FBF1F2296808E7802C002416
:1060900000440258598B4F01002CC0FFFF340C0004
:1060A0001021010000000024C0E0FEFFD34D62106B
:1060B000C5002000007000520024024800E100E00A
:1060C000636B5B0700F16F83636BDE0769D4636BFF
:1060D000580601D54023A3630123704A3721204687
:1060E000C5F8D8350023A360E3681A4041F237139E
:1060F000134341F28832E360FDF71CFA70BB049A47
:106100004FF6FE739A4200F23982DFF890A1DFF871
:106110009881634E002241F2371337212046A26056
:10612000E26802EA0A02134341F28832E360FDF7B3
:1061300001FA00289CD1C4F8088041F22913E268D2
:1061400002EA0A021343E36047B13B46626B12F076
:10615000450F01D0920427D5013BF7D14FF0805075
:1061600086E7504BD3F8DC2022F40072C3F8DC2021
:10617000D3F8DC2042F40072C3F8DC20D3F8DC2032
:1061800002F400720292029AD3F8842042F4007260
:10619000C3F88420D3F8842022F40072C3F884204A
:1061A000D0E60123A36397E7636B5B0758D4A6632C
:1061B0006269049B002A03F101030493049B03DB3F
:1061C0004FF6FE718B42A5D904994FF6FE739942A2
:1061D00000F21782500040F1D4814FF00108D5F849
:1061E0000090C5F8D4852368990700F0C481002386
:1061F000DFF8A8A02046A36041F20233E26802EA79
:106200000A021343E360FBF7B5FE00287FF430AFCA
:10621000636941F20311C5F80836A369C5F80C3665
:10622000E369C5F81036236AC5F81436A060E36840
:1062300003EA0A030B43E360002F3FF417AFDFF8D4
:1062400060C041F2873007E7636B5B0722D4636B62
:10625000DE071CD42369DBB2032B06D0012007E73D
:1062600004234FF08050A36302E7C4F838C0636989
:1062700013F4604F3FF4DEAE590400F19D8213F435
:10628000004F0CBF4FF480304FF48050F0E60123F4
:10629000A363E3E704231846A363E9E6C0E0FEFF37
:1062A000C500200000440258000010C14FEA0E490A
:1062B000C5F8E0E5D44A2046C4F80890E3681A40DF
:1062C00041F209331343E360FBF754FE00287FF4E7
:1062D000CFAE6269C5F8F825A369C5F8FC35E76952
:1062E000C5F80076216AC5F80416D4F818C04FEA3C
:1062F0001C5CC5F8DCC54FEA927C8DF828C0C2F35F
:10630000836C8DF829C0C2F3016C8DF82AC0C2F3EA
:10631000074C8DF82BC0C2F3072CD2B28DF82CC0DD
:106320008DF82D201A0DADF82E20C3F303428DF801
:106330003020C3F3C0328DF83120C3F380328DF8A2
:106340003220C3F340328DF83320C3F300328DF88E
:1063500034208DF83500B8F1000F00F01F811B04C8
:1063600003F47C1343EA17430E934FF40073C5F80C
:10637000E8350E9B01339B02C5F8E435C5F8EC35D2
:10638000C7F380334FF4007A20468DF84130C7F3CD
:10639000C61307F07F07C5F8F0A58DF84230CB0F84
:1063A0008DF8437001278DF84430C1F341738DF8A7
:1063B0004530C1F382638DF84630C1F383538DF8C5
:1063C0004730C1F340538DF8483000238DF84930F1
:1063D000C1F300438DF84A30C1F3C0338DF84B3020
:1063E000C1F380338DF84C30C1F340338DF84D301C
:1063F000C1F300338DF84E30C1F381238DF84F3057
:10640000C1F30123C1F346018DF8503041F2071367
:106410008DF8511007218DF85270C4F80890DFF8FC
:10642000E891E26802EA0902134341F28832E3602C
:10643000FDF780F800287FF41BAEC4F808A041F2F5
:10644000101BE36841F288321021204603EA090359
:1064500043EA0B03E360FDF76DF8002840F09480F9
:1064600095F8CC35032B3FF4F0AC2F6863699A01A3
:106470007ED44FF0400A41F2883210212046C4F801
:1064800008A0E36803EA090343EA0B03E360FDF7AE
:1064900051F8002843D1D5F8E035372120461B04B8
:1064A000A36041F23713E26802EA0902134341F2A2
:1064B0008832E360FDF73EF888BB4FF0FF330D21D3
:1064C0006362C4F828A0E36A23F0FF0343F0630388
:1064D000E36241F20D13A0602046E26802EA09027D
:1064E000134341F28832E360FDF724F8B8B9019E06
:1064F00004E02B68DB1B013300F08A80636B13F42C
:10650000957F636B40F087801B04F2D506F1200273
:10651000D4F8803046F8043BB242F9D1E9E7D5F827
:10652000D035C5F8D035394B0122A363D5F8D03525
:1065300018434FF40073C5F8D005204685F8CC25E4
:10654000A36041F21013E1682F4A0A40102113435F
:1065500041F28832E360FCF7EDFF00283FF475ACB0
:106560002A4A0123A263C5F8D00585F8CC356CE42E
:106570004FF40060D7E74FF0806079E5049A9A42C3
:106580003FD84FF000082AE6204BA363D5F8D0355A
:106590000343C5F8D03585F8CC7556E440F6FC7257
:1065A00002EA830343EA97730E93C7F3C2638DF83D
:1065B0003C30C7F302638DF83D30C7F342538DF88A
:1065C0003E30C7F382438DF83F30C7F3C2338DF8B6
:1065D000403001230E9A9DF840001A4400F0070055
:1065E000023082409DF8300000F00F00C5F8E4252D
:1065F0008340C5F8E8355B0A02FB03F3C5F8EC35C8
:10660000BEE64FF0807033E5C0E0FEFFFF0FE01FF5
:106610004FF0004087E7180700F1C880636B9907C7
:1066200000F1C880636B9A0608D5C1E0D4F88020D9
:106630002B6846F8042BDB1B0133E9D0636BDB04CA
:10664000F4D40A9B5E4AA263C3F381128DF814202E
:10665000C3F340128DF815201A0A22F0FF0242EA15
:106660001362DDE90B1392B209BAADF81620DAB263
:1066700006918DF81C20C3F307229DF83B108DF87E
:106680001D20C3F303521B0C8DF81E200D9A23F01E
:10669000FF03D0B203432046ADF82030C2F3852378
:1066A0008DF82230C2F301238DF82330C2F3031397
:1066B00002F00F028DF824304FF400738DF825207E
:1066C0008DF826101021A3603E4AE3681A4041F27B
:1066D0001013134341F28832E360FCF72BFF0028CC
:1066E0007FF43EAF9DF82430B8F1010F9DF82520CE
:1066F000DBB2D2B205D1134314BF4FF400784FF48C
:106700008078D5F8A805C5F8F48573F0BDF80028A1
:106710007FF49BAB2C6803E02B681B1B013330D04C
:1067200073F090F80428F7D100230121D5F8E4256F
:10673000C5F8D035C5F8C83585F8CC15002A3FF422
:1067400084AB4FF4804073F09FF800287FF47DAB5A
:10675000D5F8D435F3B1012B7FF477AB02201A4C76
:1067600085F81806A4F124030FCB84E80F00A4F1E8
:10677000140310340FCB84E80F0000201BB0BDE8D9
:10678000F08F4FF000420123C5F8D02585F8CC35B5
:10679000FFF75BBBD5F8D835002BE0D0012B7FF499
:1067A00054AB1846DBE70423A36395E40820BAE65C
:1067B0002020B8E60220B6E64FF4005058E400BFAF
:1067C0003A0F0018C0E0FEFF9C320024C74BD3F8FC
:1067D0001C16D3F8202670B58C0F93F81856100E9F
:1067E000C2F3072C83F84846C1F383640001012DEE
:1067F00083F84946C1F3016483F84A46C1F307446C
:1068000083F84B46C1F30724C9B283F84C46C2F360
:10681000035483F84D16A3F84E06C2F3C030B3F804
:106820004E1689B241EA0401C2F30344A3F84E169E
:10683000C2F3403183F85046C2F3803483F85106E6
:106840004FF0000083F8524683F85316C2F300312C
:1068500083F85416D3F8241683F8550640F2EF80D7
:10686000022D00F0C3802A204FEA4C0C83F86146C9
:10687000C1F3C01201F07F010CF07E0C83F862C6F8
:106880004FF0010C93F862461443D3F8282683F89E
:106890006246D40F83F86316910D83F86446C2F301
:1068A000417401F00C01C2F3815583F86546C2F3CF
:1068B000826483F8664683F8671693F86716D3F800
:1068C0002C46294383F86716C2F3405183F86816B3
:1068D000002183F86916C2F3004183F86A16C2F3F7
:1068E000C03183F86B16C2F3803183F86C16C2F3A3
:1068F000403183F86D16C2F3003183F86E16C2F38F
:10690000812183F86F16C2F30121C2F3460283F896
:106910007016C4F3074183F87126220E090283F82A
:1069200072C683F87426C4F30722A3F876162406E9
:10693000B3F8761689B21143A3F87616D3F8301659
:10694000C3F878460C0ED3F8782642EA0442C3F81E
:1069500078260A0AD3F8784602F47F422243C1F32C
:106960000724C9B2C3F87826D3F87856D3F834266A
:106970002C43C3F8784683F87C16110E83F87D16F5
:10698000110C0906C3F880161102D3F880460A4696
:1069900001F47F01214392B2D3F83846C3F8801640
:1069A000D3F880160A43C3F88026C4F30352D3F801
:1069B000801641EA1461C3F8801693F884161143D7
:1069C000C4F3072283F88416210A01F47061A3F846
:1069D0008616B3F8861689B21143C4F34602A3F8AB
:1069E000861683F8882683F889C670BD1204C1F321
:1069F000072C0D0E02F47C12C3F85826C1F307428F
:106A0000D3F8584644EA0524C3F85846D3F8584604
:106A100022434FF40074C3F85826D3F85826C3F81D
:106A20009846013240F10004A40244EA92549202D2
:106A3000C3F89446C1F38034C3F8902614E74FEAB4
:106A40008C2CC1F3C26594000CF44062C1F3072C96
:106A500004F47F74C3F85826D3F858261443CA0B9D
:106A6000C3F8584602F00602D3F8584644EA917437
:106A7000C3F85846C1F3026483F85C56012583F8D5
:106A80005D46C1F3425483F85E46C1F3824483F805
:106A90005F46C1F3C03483F8602693F86026224332
:106AA00083F86026D3F8584693F8602693F850662A
:106AB000023205FA02F2B540D617A2FB052EC3F842
:106AC000985605FB06EE04FB0EEE0134A2FB0424EF
:106AD000A644520AC1F3803442EACE52C3F890264B
:106AE0004FEA5E22C3F89426BEE600BF802C002445
:106AF000024B01F001011970704700BFC416002459
:106B0000704700BF704700BF704700BF012070474B
:106B1000034B18685B68C01AC0F30B00704700BFD6
:106B200040330024074B93F8A422012A01D100200E
:106B3000704793F8A432032BF9D1034B1878C0B2F5
:106B4000704700BF40330024C4160024012380F89E
:106B500049307047EFF31182702383F3128808499C
:106B6000D2B2D1E9B93182F31188581E8B42A0EB21
:106B700001008CBF0023012300EB0330704700BFEE
:106B80004033002470B5D0F8D442D0F8C86200EB8E
:106B9000840EDEF8C05245B301F00F040A4604EB40
:106BA000840C00EB8C0CDCF818306BB9DEF8C432C6
:106BB00000211B69C5F8141223B105F50471D5F83D
:106BC00008029847002070BD04EBC40406EB84065D
:106BD000F469B3FBF4F604FB1633002BE6D11A4636
:106BE000CCF818307AF068FEECE7032070BD00BFE7
:106BF000D0F8D42200EB820210B5D2F8C042ACB17A
:106C000001F00F03D0F8C802D2F8C42204F50371D2
:106C100003EBC303D26800EB8303D4F80402D3F878
:106C20006832C4F80C329047002010BD032010BD1C
:106C3000D0F8D43200EB830010B5D0F8C04284B154
:106C4000D0F8C4325BB194F80002FF2807D09B68EB
:106C5000214694F801229847FF2384F8003200204F
:106C600010BD032010BD00BF30B52B4C86462379E4
:106C7000E5889D4242D91846043419461A4602E076
:106C8000954246D921780C440A44617892B205298C
:106C9000F6D1A1788229F3D19C461A461F4903E018
:106CA000AA4234D291F800C06144624491F801C014
:106CB00092B2BCF1050FF3D191F802C0BCF1010F03
:106CC000EED1164A02E0A8421DD213781A440344BA
:106CD00092F801C098B2BCF1050FF4D19378812BE2
:106CE000F1D10CB11023A37119B100200223087156
:106CF0004B711AB1002102231171537143230748CC
:106D0000AEF8003030BD0022002CEBD1ECE70021C2
:106D1000D7E70024C0E700BFC4160024C81600242B
:106D200030B52B4C86462379E5889D4242D91846DA
:106D3000043419461A4602E0954246D921780C449B
:106D40000A44617892B20529F6D1A1788229F3D15B
:106D50009C461A461F4903E0AA4234D291F800C06B
:106D60006144624491F801C092B2BCF1050FF3D1C5
:106D700091F802C0BCF1010FEED1164A02E0A84220
:106D80001DD213781A44034492F801C098B2BCF1A2
:106D9000050FF4D19378812BF1D10CB11023A3719D
:106DA00019B10020402348710B711AB10021402312
:106DB0005171137143230748AEF8003030BD0022F3
:106DC000002CEBD1ECE70021D7E70024C0E700BF9F
:106DD000C4160024C8160024A2E700BF03460A22F6
:106DE00001481A80704700BF0C170024064B4FF073
:106DF000120C064AA3F11400526DA1F800C0022A39
:106E000018BF1846704700BF2C17002400400058D8
:106E1000042301480B807047401700241D48D0F818
:106E20000038D0F8082830B59B184FF01A040C80B1
:106E300001D1194830BD184A0024D0F8040802F1E5
:106E4000100511464FEA137EB3F1204FCC7001F1CB
:106E500002010EF1370C38BF0EF1300C8D424FEAB3
:106E6000031381F800C0EDD102F108050024010FE1
:106E7000B0F1204FD47402F1020201F1370338BFA0
:106E800001F1300395424FEA00101374EFD102482C
:106E900030BD00BF00E0F11F441700241223014859
:106EA0000B8070471817002400207047212808B570
:106EB00028D0222818D0202814D199B1072A11D11E
:106EC000184A0868184BB1F804C0D2F8EC22897946
:106ED000C3F89C00A3F8A0C083F8A21012B1014629
:106EE00000209047002008BD0029FBD0022AF9D1DC
:106EF0000C4AD2F8F032002BF4D00988D2F8F40210
:106F00009847EFE70029EDD0072AEBD1064B002088
:106F1000D3F89C200A60B3F8A0208A8093F8A230AE
:106F20008B7108BD40330024C41600240020704734
:106F3000034B93F81C03003818BF0120704700BFB3
:106F400040330024034B93F81C03032894BF002014
:106F50000120704740330024004870476036002409
:106F6000164B002030B493F82A4014B1DD698D42ED
:106F700005D0013010330828F5D130BC7047104BD4
:106F8000BAB1D3F8681301EB40218A4201D1022C37
:106F900008D093F8082512B9012283F808250122A8
:106FA00083F8512303EB0013012283F87A2330BCCA
:106FB000704703EB001383F87A23DEE79036002452
:106FC0004033002430B40023194C04F5547084F885
:106FD000F43303E001331030082B1CD0C5698D4217
:106FE000F8D190F82AC0BCF1030FF3D1AAB1D4F8BC
:106FF000681301EB43218A4208D094F8082512B99E
:10700000012284F80825012284F8512304EB03149B
:10701000012384F87A3330BC7047D4F8F02304EBB2
:1070200003130421013283F87A13C4F8F023F2E742
:1070300040330024C0B1836823B10F4B072283F88B
:10704000522370470C4A042192F8500382F86433AB
:10705000032882F85213C2E9D73314BF4FF4807368
:107060008023C2E9D5337047034B012283F80825FA
:1070700083F85123704700BF40330024244910B5E2
:10708000B1F8A64091F8A4C0644531D96346A43153
:10709000E646624603E0944238D991F800E0714434
:1070A000724491F801E092B2BEF1050FF3D191F86C
:1070B00002E0BEF1810FEED1164A03E0A3421BD2DB
:1070C00092F800C06244634492F801C09BB2BCF1E4
:1070D000050FF3D192F802C0BCF1010FEED119B146
:1070E000002402230C714B71002102231171537192
:1070F00020230380074810BD0029F9D00223002275
:107100004B7120230A710380024810BD0021D3E790
:10711000C416002468170024244910B5B1F8A6400D
:1071200091F8A4C0644531D96346A431E64662466D
:1071300003E0944238D991F800E07144724491F828
:1071400001E092B2BEF1050FF3D191F802E0BEF179
:10715000810FEED1164A03E0A3421BD292F800C081
:107160006244634492F801C09BB2BCF1050FF3D1B5
:1071700092F802C0BCF1010FEED119B100244023F6
:107180004C710B7100214023517113712023038036
:10719000074810BD0029F9D0402300220B7120239D
:1071A0004A710380024810BD0021D3E7C4160024B1
:1071B00068170024244910B5B1F8A64091F8A4C07E
:1071C000644531D96346A431E646624603E0944201
:1071D00038D991F800E07144724491F801E092B21C
:1071E000BEF1050FF3D191F802E0BEF1810FEED1AF
:1071F000164A03E0A3421BD292F800C062446344E3
:1072000092F801C09BB2BCF1050FF3D192F802C015
:10721000BCF1010FEED119B1002440234C710B7168
:10722000002140235171137120230380074810BDB2
:107230000029F9D0402300220B7120234A710380DA
:10724000024810BD0021D3E7C416002468170024AB
:1072500003460A2201481A80704700BF881700249D
:1072600038B5D0F8D432B03350F823507DB195F80A
:107270001C32044623B9D5F818320BB16B7A8BB1A6
:10728000812120467AF092F96B7A022B00D038BD2A
:10729000204681217AF08AF920460121BDE8384054
:1072A0007AF084B901217AF081F920468121BDE884
:1072B00038407AF07BB900BFD0F8D42200EB8202CC
:1072C0002DE9F041D2F8C0420646002C4ED0B4F869
:1072D000643204F11007D4F870520846D2F8C42280
:1072E000394603FB05F5D2F81080B5F5007FD4F8D8
:1072F0006C2228BF4FF40075B5FBF3F39BB2C04777
:1073000000281BDB2B463A46812130467AF0D4FA1E
:10731000B4F86422B5FBF2F2D4E99B1311449B1A32
:10732000D4F83822521BC4E99B13C4F8382213B195
:107330000020BDE8F08103232372F9E7D6F8D432A8
:10734000B03356F823208AB192F861320424112018
:1073500003F148010133DBB202F8314002EBC10115
:10736000A342888008BF002382F861324FF0FF30CB
:10737000DFE700BF38B5084BD3F8783553B1DB6988
:1073800014460D4698474FF40073026800202A60A7
:10739000238038BD1B68FFDE4033002408B5064B50
:1073A000D3F8783523B11B699847013840B208BD3E
:1073B0004FF0FF3008BD00BF40330024002070476D
:1073C00000207047174A10B51368506851681B1A9F
:1073D000C3F30B03002BF7D0B1F5805F0AD04B1C31
:1073E0001148C3F30B03445C536092F87C354BB9EE
:1073F000204610BD01230C49536092F87C350C786F
:10740000002BF5D05368116803F6FF735B1AC3F3C2
:107410000B03802BECD9002382F87C3572F0A8FF97
:10742000204610BD40330024145500242DE9F843B4
:107430001B4E07460D683468C4F58058454516D87C
:107440002A46254417483946C5F30B05204480F0E9
:10745000F3F83560736803F6FF735B1BC3F30B032C
:10746000802B16D972F084FF0020BDE8F883DFF886
:1074700034900146424609EB0400A4F5805480F0A4
:10748000DBF807EB0801254448462A4680F0D4F88B
:10749000DFE70123032086F87C35BDE8F88300BFD1
:1074A00040330024145500242DE9F0410121044605
:1074B0004FF4077080F0DAF8054600286CD0D4F855
:1074C000D46204EB8606C6F8C002237CC4F8BC0272
:1074D000002B40D0402302228121204679F05EFF1C
:1074E0000121402302222046218779F057FF4FF0E7
:1074F00001080823032282212046A4F8788179F02C
:107500004DFF294B0027E364D6F8C432C5F8047256
:107510001B689847D5F80402C5F81472C5F81872AC
:1075200000283ED0227CD4F8C83222BBC3F88C227B
:107530004FF400749A7903F51E71C3F88402012A8E
:10754000A3F87882C3F8884223D018687AF0A4F8A8
:107550000020BDE8F08120464FF400730222812113
:1075600079F01CFF01214FF400730222204621878D
:1075700079F014FFBBE79A79402403F51E71C3F834
:107580008C72012AC3F88402A3F87882C3F8884277
:10759000DBD1C3F89402D8E7D4F8D432B03344F83E
:1075A00023000220BDE8F08101001000D0F8D432A1
:1075B000B03370B550F823402CB30026124B05466B
:1075C00084F83C12C4F8303204F50C7226720D2394
:1075D000812104F504747AF06FF9D5F8C8321F22BE
:1075E0000121C3F88C62A3F8781203F51E711868A4
:1075F000C3E9A1429A79012A08BFC3F89442BDE8C1
:1076000070407AF049B870BD55534253D0F8D42237
:1076100000EB82022DE9F041D2F8C0420646002C70
:1076200067D0B4F8643204F11007D4F870520846F9
:10763000D2F8C422394603FB05F5D2F81480B5F51B
:10764000007FD4F86C2228BF4FF40075B5FBF3F32C
:107650009BB2C047002834DBD4F83802B4F8642267
:10766000401BB5FBF2F5D4E99B13C4F8380229445A
:107670005B1BC4E99B13FBB1D6F8C80202FB03F302
:1076800001220021B3F5007FC0F88472A0F87822AF
:10769000827928BF4FF40073C0F88C1200F51E7178
:1076A000012AC0F8883208BFC0F89472006879F0E7
:1076B000F3FF0020BDE8F08119463046FFF776FF62
:1076C000F7E7D6F8D432B03356F823208AB192F8CF
:1076D00061320424032003F148010133DBB202F8D4
:1076E000314002EBC101A342888008BF002382F829
:1076F00061324FF0FF30DDE7D0F8D43200EB830386
:107700002DE9F043D3F8C04283B0002C00F0B780DD
:107710001646127805460F465A2A5FD85A2A00F2B2
:107720009B80DFE812F04601990099005A01990008
:107730009900990099009900990099009900990081
:10774000990099009900990099008E01990099007B
:1077500099009900990099009900AC01CD01990018
:1077600099003D0199009900990099001002990033
:10777000360299009900FA0099005E02990099007A
:1077800099009900E10199009900990099009900E8
:107790009900990099009900990099009900990021
:1077A0009900990099009900990099009900990011
:1077B0009900990099009900990099009900990001
:1077C00099009900990099009900990099009900F1
:1077D00099009900990099009900F001A82A53D0C6
:1077E000AA2A00F064829E2A36D1D3F8C432084611
:1077F00004F5197204F51A715B6898470146002870
:1078000040F0098394F86232022B00F00483D6F82A
:107810000A301ABAE2601BB104F1100080F02AF8B5
:10782000D4F868320022013B190E61F30702190CEB
:1078300061F30F22190A61F31742B4F8641263F37B
:107840001F624BBA6383002362612383D6F80A3038
:107850001BBAE360002014E094F86122052620257D
:107860000221531C4832DBB204F8326004EBC20040
:10787000042B858008BF0023617284F861324FF0C9
:10788000FF3003B0BDE8F08394F80880B8F1000F32
:107890007DD194F91C22002A80F2058394F862229B
:1078A000022A00F08083D3F8C43208469B689847C8
:1078B000002840F0DE82D6F80230D5F8D4121BBA88
:1078C000B031C4F86C32D6F8062055F8211012BA3F
:1078D000C4F870220029D2D01344D1F86802834240
:1078E00000F24783B4F8643202FB03F3D4F81822A1
:1078F0009A424AD091F861320524202003F14802CF
:107900000133DBB201F8324001EBC202042B90805C
:1079100008BF002381F86132B1E794F80880B8F11C
:10792000000F34D194F91C22002A80F2BC8294F812
:107930006222022A00F03783D3F8C43238469B68AB
:107940009847002840F09582D6F80220D5F8D41246
:1079500012BAB031C4F86C22B6F8073055F82110CD
:107960005BBA9BB2C4F87032002988D01A44D1F8AF
:107970006862B24200F27383B4F8642202FB03F33C
:10798000D4F818229A4240F0E182022323724FF485
:10799000007339462846E36003B0BDE8F0438BE44A
:1079A000337900229B1AE26018BF012384F8623207
:1079B00050E7D4F81822002A40F0398294F8621275
:1079C000022900F04683D3F8C43238469B689847B2
:1079D000002840F0D382E0603CE7D4F81832002B56
:1079E00000F025827021002294F8603221740C216D
:1079F000C4F81520E17594F86112C4F81120994279
:107A0000C4F81920C4F81D2084F8212011D004EBFB
:107A1000C30191F84012A17404EBC3010133B1F822
:107A20004412DBB2A183042B14BF84F8603284F8C3
:107A300060221223E36032799A4298BF1346E360D2
:107A400008E7D4F81822002A00F0F1817278D207F2
:107A500040F1B181B378002B00F0CF81802B40F052
:107A6000E0810821CC4A04F1180304F11000E16020
:107A700012F8011D03F8011D8342F9D1EAE6D3F89B
:107A8000C4323846DB689847002840F07481327968
:107A9000042A134628BF0423E360002A3FF4DAAE29
:107AA000013BBD4A04F1100099B201F111030A44EF
:107AB000234412F8011903F8011D8342F9D1C9E6E4
:107AC00094F862223379012A03F0030300F06A81FB
:107AD000012B00F06C81022B00F06A81032B00F077
:107AE00066810023E360B5E6737813F0020340F08B
:107AF0009881D4E99B210A44D4F868128A4200F2A2
:107B0000E581E360A6E6D3F8C4323846DB689847DF
:107B1000002840F03881337A082B194628BF082105
:107B2000E160002B3FF496AE9C4A01F1100304F192
:107B300010000A4454FA83F312F8011D03F8011DE2
:107B40009842F9D186E6D3F8C4320DF102023846E4
:107B500001A95B689847002840F06F8194F8623271
:107B6000022B00F06A81BDF802200821206152BA80
:107B7000019BA061013B62830C22E174E375190E45
:107B8000E2601A0C1B0A217562750222A375227627
:107B900077E6D3F8C43204F51972384604F51A7141
:107BA0005B689847002840F0368194F86232022BD7
:107BB00000F03181D4F868320822A082013BE260F3
:107BC000190E1A0C61F30700190A62F30F20B4F8BA
:107BD000642261F3174052BA63F31F60E2822061AE
:107BE00038E694F80890B9F1000F40F00081D4F81D
:107BF0001822002A00F08A8194F91C22002AC0F27F
:107C00001582D3F8C43238469B68984780460028CE
:107C100040F0F181D5F8D432384605EB8303D3F830
:107C2000C432DB6898470146002840F08281D6F8CC
:107C30000220D5F8D40212BAB030C4F86C22B6F8DB
:107C4000073055F820005BBA9BB2C4F870320028A8
:107C50003FF415AE1A44D0F86862B24200F2C68111
:107C6000B4F8642202FB03F3D4F81822934240F0E4
:107C7000EC80B3F5007F4FF0010004F1100428BF41
:107C80004FF4007304F8080C1A46D5F8C832C3F84C
:107C900088229A79C3F88C1203F51E718242C3F8C8
:107CA0008442A3F8780262D1C3F894425FE0227A5A
:107CB000002A40F09C80D4F81812002900F083813B
:107CC00094F91C120029C0F22181D3F8C43238463D
:107CD0009B689847D5F8D432002840F05A8105EBCC
:107CE00083033846D3F8C432DB689847002840F055
:107CF000F280D6F80230D5F8D4121BBAB031C4F8ED
:107D00006C32D6F8062055F8211012BAC4F8702249
:107D100000293FF4B4AD1344D1F86802834200F265
:107D20002881B4F8643202FB03F3D4F8182293429A
:107D30007FF4E0ADB3F5007F4FF0010104F11000D6
:107D400028BF4FF40073217200241A46D5F8C832B8
:107D5000C3F888229A79A3F8781203F51E71012AD4
:107D6000C3F88402C3F88C4208BFC3F894021868B1
:107D700079F092FC6EE50A4A92F8E23063F07F03F4
:107D800082F8E23083E6064A92F8E73063F07F0338
:107D900082F8E730BFE600BFA4170024A81700242C
:107DA000C4160024022B3CD0012B7FF497AE002395
:107DB00084F8623295E6D3F8C43207EBC701327912
:107DC000D86900EB810003790533934228BF13463D
:107DD000E360002B3FF43EAD03F110020344224464
:107DE00013F8011D834202F8011DF9D132E539462D
:107DF000284603B0BDE8F04308E406219A4A04F19E
:107E0000160304F11000E16012F8011D03F8011DD2
:107E10008342F9D11EE53A220221284679F0F0F892
:107E20002DE524220521284679F0EAF827E52022CD
:107E30000521284679F0E4F821E528463A22022176
:107E400079F0DEF84FF0FF301BE590F86132052540
:107E5000202403F148020133DBB200F8325000EB7A
:107E6000C202042B948014BF80F8613280F8611242
:107E700005E5D5F8D432B03355F82320002A3FF475
:107E8000FEAC92F8613202243A2003F1480101333A
:107E9000DBB202F8314002EBC101042B888075D0BF
:107EA00082F86132EBE494F861320520202103F17D
:107EB00048020133DBB204F8320004EBC202042BA7
:107EC00091807FF4DAAC84F86182D8E42122052124
:107ED00079F096F8D3E4D5F8D432B03355F82320AE
:107EE0008AB192F861320225272003F1480101335B
:107EF000DBB202F8315002EBC101042B888008BFCD
:107F0000002382F8613205232372B8E494F86132C9
:107F10000525202003F148010133DBB204F831507C
:107F200004EBC101042B88807FF4A7AC84F86122A4
:107F3000A5E4D5F8D432B03355F82320002A3FF415
:107F40009EAC92F86132022427209EE791F86132BC
:107F50000525202403F148020133DBB201F8325039
:107F600001EBC202042B94807FF4D4AC81F861024F
:107F700085E491F8613205242120BFE43A220221F0
:107F8000284679F03DF80523237278E482F861826F
:107F900075E4B03355F82320002AB4D092F861324A
:107FA00002253A20A1E794F8613203F14801013338
:107FB000DBB204F8312004EBC1013A22042B8A80A1
:107FC0007FF45BAC7FE794F861320525202003F154
:107FD00048020133DBB204F8325004EBC202042B36
:107FE00090807FF44AAC84F8611248E490F86132E2
:107FF000052521242DE7D5F8D432B03355F82320B8
:10800000002A3FF43CAC92F8613202243A2003F19A
:1080100048010133DBB202F8314002EBC101042B0D
:1080200088807FF43DAF82F8619228E494F8613251
:108030000520202103F148020133DBB204F83200AD
:1080400004EBC202042B91807FF417AC84F8619298
:1080500015E43A2278F0D4FF052323720FE491F857
:1080600061320525212475E79A170024D0F8D4320F
:10807000B03350F82330CBB110B51A7A022A07D0AA
:10808000033A012A02D80021FFF790FA002010BD20
:1080900003F21F2293F81D120446FFF72DFB002860
:1080A000F4DA01212046FFF781FAEFE7002070475C
:1080B000D0F8D432B03370B550F8235025B12B7AB4
:1080C000044683B1012B01D0002070BD05F21F22B0
:1080D00095F81D12FFF710FB0028F5DA0121204664
:1080E000FFF764FAF0E7D5E98523C5F83832D0F810
:1080F000C832C5F83422D3F88C321F2B04D12F4B51
:10810000D5F810229A421AD095F861324FF0050C3A
:108110002021204603F148020133DBB205F832C0CA
:1081200005EBC202042B91804FF0020208BF00232E
:108130006A7285F86132FFF793F8002070BD95F8F8
:108140001D120129E0D895F81E32013B0F2BDBD818
:1081500005F21F22FFF7D0FA00282B7A22DB013B21
:10816000022BB1D9EE681EB3D4F8D432B03354F830
:1081700023100029A8D02046D1F83842D1F818326F
:1081800005F11002A41BB342C1F838424FF00004BD
:1081900028BF334681F83C4204240C72812179F0D7
:1081A0008BFB91E7052B99D02046FFF759F88BE719
:1081B00031462046FFF7FAF986E700BF55534243A0
:1081C000F8B5D0F8C85240F20112044695F894343C
:1081D0002A87012B3ED001260027286832463146E7
:1081E00085F8946479F0E8FB27873A463146286899
:1081F000A5F8786285F8946479F0DEFB4FF481731A
:10820000A4F8787132460221286885F89464A5F8AC
:108210005C3079F0D1FB85F89474D4F8D432002521
:1082200004EB8303E564D3F8C0228AB1D3F8C432E7
:108230005B689847D4F8D432B03354F823007FF009
:1082400039FAD4F8D432B03344F82350C4F8BC52CD
:108250000020F8BD00224FF481710287A5F8783222
:10826000A0F87821A5F85C10D7E700BFF8B5D0F8E2
:10827000C85201260446002295F89434A5F8786285
:10828000B34227D03146286885F89464002779F0F6
:1082900093FB40F20113A4F8787132463146286806
:1082A00085F894642B8779F087FB85F89474D4F86B
:1082B000D4320025B033258754F8230040B17FF035
:1082C000F9F9D4F8D432B03344F82350C4F8BC528E
:1082D0000020F8BD40F20113A0F878212B87E6E7D3
:1082E000D0F8D43200EB8303F0B5002683B0D3F886
:1082F000C0728DF80560ADF806605FB191F800C0FE
:1083000004460D461CF060022FD0202A05D02046DE
:1083100079F088F9032003B0F0BDCA884878002AB4
:1083200042D01CF0800F00F08380D3F8C43239466D
:108330009B689847EA8802234FF48071072AC4F8A3
:10834000943228BF0722D4F8C832C4E906225A6200
:108350009A79998203F11401012A1F629E6200D169
:108360001F63186879F098F922E04B780B2BCED870
:1083700001A252F823F000BFB5830408B1830408BA
:108380000F8304080F8304080F8304080F83040875
:108390000F8304080F8304080F8304080F83040865
:1083A000F5830408EB830408D3F8C4329B6898472C
:1083B0000020B0E790F89C32032BA8D10222D0F81D
:1083C000C8320020C4F8942203F11401C4E9062243
:1083D0000DF106049862C3E908424FF480729A8254
:1083E0009A79012ABDD11C63BBE790F89C32032B1C
:1083F000DED08CE790F89C32032B88D10122022139
:10840000D0F8C832C0F8941203F11401C0E9062272
:108410000DF10500C3E908024FF4807200209A8232
:108420009A799862012A9CD10DF10500186398E7AA
:10843000402A4FF0030387F8000228BF402287F844
:108440000122C4F89432D4F8C832C4F85821C4F8D0
:108450005C2103F51571C3F864229A79C3F8607240
:10846000012AC3F86862A3F8546208BFC3F87072A7
:1084700077E700BF08B520B9044870F0BDFE044896
:1084800008BD044870F0B8FE014808BDD8280D08A2
:10849000C0380024FC280D08024808B570F0ACFE76
:1084A000014808BD20290D08C0380024024808B53D
:1084B00070F0A2FE014808BD28290D08C03800242C
:1084C000024808B570F098FE014808BD34290D082F
:1084D000C038002408B520B9044870F08DFE044867
:1084E00008BD044870F088FE014808BD44290D0805
:1084F000C038002464290D08024808B570F07CFEDD
:10850000014808BD84290D08C0380024024808B578
:1085100070F072FE014808BD90290D08C038002493
:108520005A4B00215A4A1B685A48A2FB032330B514
:10853000DB0C594C83B0013BC4F89016C4F8881684
:1085400042F20F7194F8BD26C4F88006C4F88C1668
:10855000C4F88436002A00F0938002254F494D4824
:1085600084F8BD56FAF704FC01234D4A0621372052
:1085700084F8C83684F8BE3684F8BF3684F8C0362E
:1085800084F8C13684F8C23684F8C33684F8C43619
:1085900084F8C53684F8C63684F8C73684F8BD3604
:1085A000D2F8E83043F02003C2F8E830D2F8E830DF
:1085B00003F020030193019B71F014FB394B4FF43E
:1085C00000025A6094F8BD36012B3BD1D4F88026C6
:1085D000354B3648B2F1804F18BF9A4284F8BD56E9
:1085E000D1680CBF0123002341F00101824208BF82
:1085F00043F0010300F58060D160824208BF43F080
:10860000010300F580602A49824208BF43F001035C
:1086100000F57840824208BF43F001038A4208BF58
:1086200043F0010313B9234B9A4207D19168224BBF
:108630000B40062B06D0B3F5803F03D0136843F000
:1086400001031360D4F8DC3204EB8303D3F8C8329F
:1086500043B11A4800211A4AC3F80802C3F810129D
:10866000C3F8042200252560C4F8F0526560C4F800
:10867000EC5284F87C5571F07BFE284603B030BD87
:1086800002F0FF0084F8BC0667E700BF000000248A
:1086900083DE1B430014004040330024C43900240F
:1086A0000044025800E100E00000014000040040E6
:1086B000001800400040014007000100144500245C
:1086C0000C3A00242DE9F84F2C4E8B46D6F8C422E4
:1086D000D6F80C8705E0D6F80C37A3EB0803322B4D
:1086E00044D8D2F81472002FF5D1BBF1000F3ED060
:1086F00000F1FF3A4FF07009D6F8E8321AF8012F6E
:108700001F49CA540133C3F30B03C6F8E832EFF331
:10871000118289F31288D2B2D6E9B93182F3118875
:108720008B42A3EB01038CBF0022012203EB023337
:10873000012B1FD1D6F80C37A3EB0803322B16D828
:108740000DF0D0FA04460D460DF0CCFA001B61EB9B
:108750000501B0F57A7F71F10001F5D3EFF31182D5
:1087600089F31288D6E9B931D2B2D7E70027384663
:10877000BDE8F88F0137BB45BED1F8E74033002490
:1087800014450024F8B5104D95F8A432012B00D102
:10879000F8BD95F8A432032BFAD10C4B1B78002BB3
:1087A000F6D00F461446D5F80C6708E0FFF78AFFAD
:1087B000D5F80C37241A07449B1B322BE8D8002C21
:1087C00021463846F2DCF8BD40330024C4160024AC
:1087D000F8B590F848305D1C0344EDB280F848507D
:1087E00083F8341090F8493053B1132D07D9002382
:1087F00080F84830104F97F8A432012B05D1F8BD0E
:1088000080F84830002DF5D1F8BD97F8A432032B3D
:10881000F5D1D7F80C6700F1340429462046FFF75C
:1088200051FFD7F80C372D1A04449B1B322BE6D886
:10883000002DF2D1F8BD00BF40330024F8B500236D
:1088400090F84850A0F8483005B9F8BD0D4F97F89A
:10885000A432012BF9D097F8A432032BF5D1D7F825
:108860000C6700F1340429462046FFF72BFFD7F8A8
:108870000C372D1A04449B1B322BE6D8002DF2D165
:10888000F8BD00BF40330024F8B51F4FD7F8342A95
:10889000B7F8381AD7F8783591614BB39B69984788
:1088A00030B30026D7F8783513B11B69984790B9D3
:1088B000B6F57A7F25D00DF015FA013604460D463F
:1088C0000DF010FA001B61EB0501B0F57A7F71F134
:1088D0000001F5D3E6E7B6F57A7F4FF0FF3018BF19
:1088E0000020B7F8383AD7F8342A1B049361F8BD52
:1088F000064B03F1EC02D3F8EC30C7F87825984723
:10890000CFE74FF0FF30ECE740330024C4160024DB
:108910002DE9F84F344E90469A46B6F8442AD6F8D8
:10892000404A1304A361BAF1000F50D0C8EBC853FA
:10893000C24406F52E6901EB432B41F28937D6F884
:1089400078255AB100235468494640461A46A04744
:10895000A8B9D6F878350BB11B699847013F3AD0D2
:108960000DF0C0F904460D460DF0BCF9001B61EB9B
:108970000501B0F57A7F71F10001F5D3DFE741F22F
:108980008937D6F8783513B11B69984780B9013F0C
:1089900021D00DF0A7F904460D460DF0A3F9001BF8
:1089A00061EB0501B0F57A7F71F10001F5D3E8E7DD
:1089B0000BEB482008F101084FF4007249467EF0A5
:1089C0003BFED045B9D1D6F8404AB6F8442A00203B
:1089D000A261BDE8F88FD6F8403A4FF0FF30B6F804
:1089E000442A9A61BDE8F88F403300242DE9F84FFE
:1089F000364E90469A46B6F8442AD6F8404A1304B2
:108A0000A361BAF1000F54D0C8EBC853C24406F5B5
:108A10002E6901EB432B4FF400720BEB48214846C3
:108A20007EF00AFED6F878250AB341F28937002392
:108A3000D468494640461A46A047D6F87835B8B1BA
:108A40000BB11B699847013F37D00DF04BF9044635
:108A50000D460DF047F9001B61EB0501B0F57A7F7B
:108A600071F10001F5D3D6F87825002ADFD1002373
:108A700041F2893713B11B69984790B9013F1CD067
:108A80000DF030F904460D460DF02CF9001B61EB9A
:108A90000501B0F57A7F71F10001F5D3D6F878358C
:108AA000E8E708F10108D045B5D1D6F8404AB6F854
:108AB000442A0020A261BDE8F88FD6F8403A4FF072
:108AC000FF30B6F8442A9A61BDE8F88F403300249D
:108AD00010B5104CD4F8483323B119689A880B6943
:108AE0001A420AD0FDF780F938B994F810330133EF
:108AF000DBB2072B84F8103303D9002384F81C332E
:108B000010BDD4F80C270123C4F80C2384F81C33BF
:108B100010BD00BF4033002410B50D4CD4F84833CD
:108B200023B119689A880B691A420CD0FDF75CF9D9
:108B300048B9D4F80C270123A4F81003C4F80C2377
:108B400084F81C3310BD002384F81C3310BD00BF13
:108B50004033002470B5174D0021174E6B6C2C6804
:108B60001B04C6F81813154A0D21A3602046E368BC
:108B70001A4041F20D13134341F28832E360FAF7D1
:108B8000D9FC58B16B6B03436B63D6F80C270923F0
:108B90000020C6F80C2386F81C3370BD636903F40B
:108BA000F053B3F5006FF0D10423022086F81C3394
:108BB00070BD00BF1C32002440330024C0E0FEFF23
:108BC00070B50D4D04460E4695F81C33042B0BD0A2
:108BD000082B07D1D5F8143383420AD0FFF7BAFF28
:108BE000022801D0012070BD0823C5E9C54685F8DB
:108BF0001C33022070BD00BF4033002470B58A4C86
:108C000094F81C536B1E082B1ED8DFE803F0796C18
:108C10007D1D4F05361D2700844B5B6A002B6DD1EF
:108C20000722D4F80C37D4F8045384F81C23C4F872
:108C30000C33002D62D0D4F808330120D4E9BE21D2
:108C4000A84794F81C536B1EDBB2022B4FD9042D9E
:108C500018BF082D0CBF0120002070BDFDF798F84B
:108C6000002840F0D680D4F80C33D4F80C27FA331F
:108C70009342ECD2FFF72CFFC2E7FDF789F80028FA
:108C8000F1D0D4F818330022012B84F8102340F2DD
:108C9000C480D4F81423013B08210132C4F81833EE
:108CA00084F81C13C4F81423012070BD5F4B1E6AA6
:108CB000002E6DD1FDF76CF8002871D00423D4F894
:108CC000045384F8106384F81C33002DECD0D4F8DE
:108CD00008333046D4F8F822D4F8FC12A84794F8A8
:108CE0001C536B1EB0E770F0ADFD042867D0D4F8BC
:108CF0000C37D4F80C239B1AC82B7FD8002070BDEA
:108D0000022384F81C337BE7FDF760FD0028EED1D9
:108D1000474B0421C4F8180393F82C2084F81C1343
:108D2000D88D196B84F82623090E1A6BA4F8240336
:108D3000120C84F82713196B186B84F82823090A7E
:108D400084F82A0393F8340093F8352084F8291323
:108D5000120984F82B0393F8350084F83023996BBB
:108D600000F00F00DD8FDA8FC4F82C13D98FC2F317
:108D70000B1384F8310343EA152301F00F0203F0CB
:108D80000F0384F8342303F5FA63A4F8323337E78A
:108D9000D4F80C33D4F80C2764339342BFF457AFA4
:108DA000FFF796FED4F80453002D3FF429AF0022BC
:108DB000D4F80833D4F8FC121046A84720E7FDF792
:108DC00005FD002893D11B4B1B78002BA3F1020358
:108DD000B3FA83F308BF01255B0984F8125384F8C2
:108DE0001333FDF7F3FC00287FF444AF104B03224C
:108DF0009B6C84F81C23C4F8203301E7FFF768FE5E
:108E000094F81C03042818BF08280CBF0120002078
:108E100070BD042384F81C3346E7FAD1FFF79AFEAD
:108E200094F81C536B1E0FE7403300249C3200243F
:108E3000C8320024983200242DE9F0415C4C0D46E4
:108E40000646904694F81C131F4604290ED00829A4
:108E500040F08180D4F81433B34207D0FFF77AFE94
:108E6000022878D194F81C130429F0D10123514A27
:108E7000C4F8048384F800335362EB06C4F8087323
:108E8000C4E9BE5660D1BFF34F8F4B4A05F5007160
:108E90002B46C2F8683220338B42FAD1BFF34F8F92
:108EA000BFF36F8F002D7CD0DFF8188198F8303039
:108EB000012B49D1731CD8F8501000228B42C8F8FE
:108EC00034204BD80323D8F80070C8F81C50182160
:108ED00088F830304FF40073FA623846C8F8203012
:108EE000D8F83830354A012B4FF0FF337B624FF40E
:108EF000007318BF7602BB62FB6A23F0FF0343F0E6
:108F00009003FB62FB6843F04003FB609023BD6568
:108F100001253D65C8F82C30BE60FB681A4041F25F
:108F20001813134341F28832FB60FAF703FB68B36E
:108F3000234B0022BB63D8F834300343C8F83430E5
:108F400088F83050C8F82C2094F81133022B0CD834
:108F5000013384F811330120BDE8F081D8F83430B2
:108F600043F00073C8F83430EEE7002684F811634C
:108F7000FFF7AEFDD4F8045335B1D4F808333246C8
:108F8000D4F8FC120120A8470320E5E7FB6B06227A
:108F900084F8110343F48D7384F81C23FB63BDE84C
:108FA000F081084A536B43F000635363CCE700BF82
:108FB000403300249C32002400ED00E0C0E0FEFFBE
:108FC000FF0FE01F1C3200242DE9F84F5F4F0C46C5
:108FD0008046164697F81C131D46042908D0082918
:108FE00002D00020BDE8F88FFFF7B4FD0228F8D1C9
:108FF00014F01F016AD10122554B56489A60026253
:109000004FF40072C7F8E04C5A60002C00F09080DA
:10901000DFF84CB19BF83030012B57D108F101003B
:10902000DBF85030CBF83410984200F287800323ED
:10903000DBF800A04FF001098BF830305046DBF828
:109040003830CAF82C101121012B4FF0FF33CBE937
:109050000942CAF824304FF4007314BF4FEA482283
:109060004246CAF82830DAF82C3023F0FF0343F0E8
:109070009203CAF82C30DAF80C3043F04003CAF8F7
:109080000C308123CAF85840CAF85090CBF82C30E5
:10909000CAF80820304ADAF80C301A4041F21113AD
:1090A000134341F28832CAF80C30FAF743FA034608
:1090B00030B32A4ACAF83820DBF8342013430022A0
:1090C000CBF834308BF83090CBF82C2097F8113354
:1090D000022B03D8013387F8113382E7002587F884
:1090E0001153FFF7F5FCD7F80443002C3FF479AF98
:1090F000D7F808332A46D7F8FC122846A04770E76D
:1091000087F811330522DAF83C304846C7F8046383
:1091100043F49573C7F8085387F81C23CAF83C300A
:10912000D7F80C37C7E9BE48C7F80C33BDE8F88F4D
:109130000B4A536B43F000635363C7E7DBF83430EB
:1091400043F00073CBF83430C0E700BF4033002455
:10915000204000249C320024C0E0FEFFFF0FE01FEF
:109160001C3200242DE9F04104464FF41D707EF0BE
:1091700099FA054600285BD0D4F8D47204EB87072F
:10918000C7F8C002237CC4F8BC02002B45D04023A2
:1091900002220121204678F001F9012240234FF0FC
:1091A00001082046A4F8782181210222002678F0C7
:1091B000F5F8A4F83880D7F8C43230462E81A5F8E7
:1091C000606285F862621B689847D4F8C84294F8D8
:1091D00094342768434508D03846FAF775FA414673
:1091E0003846FAF749FA84F8946405F504751F22A5
:1091F0000023384604F51E71C4F88C320123C4E9FB
:10920000A152A279A4F878329A4208BFC4F89452C5
:1092100078F042FA0020BDE8F0814FF4007302229A
:109220000121204678F0BAF801224FF40073B6E726
:10923000D4F8D4320220B03344F82350EBE700BF17
:10924000F0B5002383B0ADF80630D0F8D43200EB8F
:109250008303D3F8C0524DB10A78044612F060007F
:1092600036D0202805D0204678F0DCF9032003B062
:10927000F0BD4878FE2849D0FF28F4D14B88002B58
:10928000F1D1CE88002EEED11006ECD44FF48073CD
:1092900081212B8105F50475D4F8C842204678F069
:1092A000B1FD2046012178F0ADFD1F22012304F518
:1092B0001E712068C4F88452A4F87832C4E9A2264A
:1092C000A2799A4208BFC4F8945278F0E5F946E0D2
:1092D0004B780B2BC7D801A252F823F063930408F4
:1092E000D3930408679204086792040867920408FD
:1092F000679204086792040867920408679204085A
:10930000679204089B930408539304084E88002E28
:10931000A9D1CF88012FA6D11206A4D5D3F8C43283
:109320009B699847022328604FF48071C4F89432F7
:10933000D4F8C832C4E906779A79998203F1140106
:10934000012A5F621D629E6241D0186878F0A4F91C
:1093500005E094F89C32032B85D18B786B6000205C
:1093600085E794F89C32032B7FF47DAF0222D4F87A
:10937000C8320020C4F8942203F11401C4E9062283
:109380000DF106049862C3E908424FF480729A8294
:109390009A79012AD9D11C63D7E794F89C32032B20
:1093A0007FF461AFD4F8C8320122022104350020D5
:1093B000C4F894124FF48071C4E90622C3E908523C
:1093C0009A79998203F11401012A9862BDD11D6333
:1093D000BBE794F89C32032BC1D14B88002BBED144
:1093E000D4F8C8628F8896F89434012B0AD00123F0
:1093F0003906306886F8943410D4FAF765F90023FA
:1094000086F894346B7A022B0DD03A06A7D5012B3F
:10941000A5D001212046FEF7C9F8A0E707F00F010B
:10942000FAF72AF9EBE72046812178F0BFF801210D
:10943000204678F0BBF892E770F060B870F05EB844
:1094400010B51C200AF084FC044611210AF03CFCF3
:1094500020460AF033FCC8200CF072FC2046BDE820
:1094600010400AF025BC00BF2DE9F04FDFF804B32F
:109470008BB0DBF8ECACDAF8143013F0010902D051
:109480000BB0BDE8F08FDAF81420DAF818301A4281
:10949000F6D0DAF808380AF50062C3F30D2301921A
:1094A0000BF58052C2F8C031DAF81430DAF818201F
:1094B00013409D0705D5DAF8143003F00203CAF80B
:1094C0001430DAF81430DAF818201340DC061BD513
:1094D000DAF8183023F01003CAF81830DAF8203020
:1094E00003F4F01203F00F01B2F5802F00F067854E
:1094F000B2F5402F00F03E83CDF800A0009A9369AA
:1095000043F01003936101E0CDF800A0009A536985
:1095100092691340180300F1AC82009A5369926972
:1095200013405F0300F1E081009B5A699B691A4276
:1095300000F1F180009A5369926913401B0509D527
:10954000019B9B68DF0700F18285009A536903F451
:109550000063536100994B698A6913401E0119D554
:109560004B690A4603F000634B61804991F8B831BA
:10957000002B00F0D8827D4BD3F8CC3193F89C229D
:10958000042A04D093F89C22D2B283F89D220422AC
:1095900083F89C22009A536992691340DD0400F11C
:1095A0005381009A5369926913409C0400F1E4804E
:1095B000009A536992691340190700F1C980009914
:1095C0004B698A6913401A0600F181804B698A69E8
:1095D0001340DB022AD59BF8F08CB8F1010F20D99B
:1095E000634B0293029E0AF51267012504E00135E0
:1095F00020372436454514D096F83C303A68012B84
:10960000F5D1002AF3DA65F07F0086F83B30C0B26E
:1096100070F0F4FDEBE7009A536992691340DA02A7
:1096200004D5009A536903F480135361009A536977
:10963000926913409F0232D59BF8F07C012F29D903
:109640000AF532624A4B012003E0B84203F12403D9
:1096500020D093F87C120130146820320129F4D113
:10966000002CF2DA414DD5F8C05185EA1445EE07D9
:10967000EBD483F87B12DAF8181041F08001CAF8B5
:109680001810DAF814100D06DFD4019A536843F469
:1096900000735360009A536903F400135361009AF6
:1096A0005369926913405C0000F1C88000994B69CE
:1096B0008A69134058077FF5E3AE4C68610700F1F3
:1096C000D784DBF8EC3C5A6814435C60D8E6DAF8DF
:1096D00018309BF8F07C23F08003012FCAF8183073
:1096E00099D9234B01251E46029303E00135243608
:1096F000BD4207D096F87B32012BF7D1E8B270F06B
:109700007DFDF3E7009B5A699B691340DB028DD511
:109710009BF8F08C66E7019A536823F001035360CD
:10972000124B93F8B831012B00F011820F4BD3F894
:10973000CC3193F89C22042A04D193F89D22D2B212
:1097400083F89C22009A536903F000435361F1E6C9
:10975000064BD3F8CC0190F89C32032B00F0FC812F
:10976000009A536903F00803536128E7404300243B
:109770002C40002440330024009AD2F800396FF3C3
:109780000A03C2F80039D2F8043843F48073C2F8EF
:109790000438D2F80838980700F1018213F0060F58
:1097A0000CBF00230F238BF8F33CF8F7D5FE9BF892
:1097B000F36C022E00F082844FF410530099003EA7
:1097C000CA6818BF012622F47052CA60B34AD2F8A0
:1097D000CC51CA681343CB600123002185F89C3229
:1097E000D5F8B8326960C5F8A41285F8A012C5F89A
:1097F00094121BB15B680BB12846984700224024A5
:10980000012740231146284677F0C8FD2346002251
:1098100080212846C5F86041A5F8647177F0BEFD47
:109820009E4BDBF8EC2CD3F8CC31AF842C621E7449
:109830005369009203F400535361B9E6009A5369E7
:1098400003F08043536131E7019A10210098536877
:1098500023F001035360F9F70FFF9BF8F00CE0B120
:109860000AF510634FF67F31996009F101091A6812
:109870002033814522F4001243F8202CC3F8E8116C
:10988000D3F8E02122F40012C3F8E021D3F8E0215C
:1098900042F00062C3F8E021E6D1019AD36943F0B7
:1098A0000113D3619BF8FB3C002B00F04581019A2A
:1098B000D2F8843043F00B03C2F88430536C43F089
:1098C0000B035364DAF80038009C23F4FE63744AF7
:1098D0002046CAF800389BF8F21C77F0E1FD636976
:1098E00003F4805363615CE6009AD2F81878D2F8EA
:1098F0001C381F40BFB2002F3FF416AE694D0AF569
:1099000010614FF00008CDF80CA013468A4644467B
:109910000295CDF8109008E07F0804F1010405F1EC
:1099200024050AF1200A00F03C81FE07F4D5D3F8A3
:10993000102804F00F01D3F834684FEA4419CE40E0
:10994000F601F6B2164303F5106202EB4412926878
:109950001640E2B2F007009222D50120019A00FAE7
:1099600001F1526B22EA010201994A639BF8F21C51
:109970004A4A8142CAF80800D2F8CC8100F08883B4
:109980002B6A0593002C40F00883D8F89432022B00
:1099900000F0FC8398F8A03213B1002388F8A032BD
:1099A000320702D50823CAF80830F30602D510237F
:1099B000CAF80830700602D54023CAF80830B1074B
:1099C00000F117813206DBF8EC3CA5D5D5E9090694
:1099D0008642A1D8811BEA6903F5106E8A42CE4403
:1099E00028BF0A46DEF81810033289B2B1EB920F95
:1099F00031D39BF8F28C03F5805C009442460CEB6B
:109A0000043C98461346B04240F2A383811BEA69A6
:109A1000914228BF11462A6A01F103094FEA9909C8
:109A200073B98CB20334A4080AD002EB840452F850
:109A3000040BA242CCF80000F9D12A6AD5E9090644
:109A40000A440E442A62DEF81820AE6292B29145B2
:109A5000D9D9009C4346B0423FF65EAF04F00F02F6
:109A600001219140D3F8342822EA0102C3F83428B6
:109A700052E70098D0F81838D0F81C2813401F0C73
:109A80003FF44BAD074B0AF53066CDF80CA04FF014
:109A900000089A460293CDF814900DE0404300244C
:109AA000C84400242C4000247F0808F1010806F176
:109AB00020060AF1240A78D017F00109F4D05FFAE1
:109AC00088F300F530624FEA4815009302EB481323
:109AD0009C68D0F814180C40E1076CD4210700F101
:109AE0009480E50601D51023B360A0070FD5039B32
:109AF0005B69190604D5019A536843F48063536087
:109B00009AF85732012B00F027830223B360A20694
:109B100001D52023B360A30402D54FF40053B360F2
:109B2000DBF8EC0CC0E7012381F8B831536DC3F3C7
:109B30008303C1F8BC312DE5019942F22B034A6938
:109B400013434B610B6943F00B030B61BAE600232F
:109B5000B64A82F8B831F5E5D0F8B832002B3FF4B8
:109B6000FFADDB69002B3FF4FBAD9847DBF8EC3C25
:109B70000093F5E501EBC101C3F30A13AB4C0BEB0A
:109B800081020AF58051D2F8540F03440868C4F8E2
:109B900088010968C2F8543FC4F88C11ACE4022370
:109BA00001E6DDE903A90093BEE4DDF80CA0DDF8D1
:109BB00014900090B1E40121B1609BF8F21CD0F840
:109BC00040E00129D3F808C000F0B38298498E45DF
:109BD00000F0AA83DBF8503F58EA030300F05984F1
:109BE000924BDAF860220099D3F8CC0177F08AFE24
:109BF00074E721460398F9F73FFDEB7D012B00F058
:109C0000C7830223CAF80830DCE6DBF8EC2C082313
:109C1000B36002F53063126C2B4410460492854AFF
:109C20009968904204D90A0402D54FF400429A6020
:109C30007E4AD2F8CC5192F8883105F2AA2085F8F4
:109C4000AA3292F889E1079085F8ABE2B2F88A115E
:109C5000A5F8AC1206910121B2F88CC1A5F8AEC2EC
:109C6000B2F88E21C5F8941203F01F01A5F8B022B6
:109C70000129C5F8982200F0B182022900F013836F
:109C8000002940F0EA8203F06003202B00F0F78304
:109C9000402B00F0F483A3B9BEF1090F11D8DFE81F
:109CA0001EF0F400CD001000E400100081006700F9
:109CB000100041002500D5F8B4325B69002B40F05C
:109CC000D485284677F0AEFC5A4B049A9A427FF628
:109CD00008AF9BF8F21C01297FF403AF029BDBF86D
:109CE000EC0C03F29C4277F0DBFBFAE69DF818904F
:109CF000514BB9F1010F83F8D890E2D895F89C2226
:109D0000D1B2022A069100F01785032900F0E984F8
:109D1000284677F087FCD5F8B832494628465B6874
:109D20009847D1E7012ACCD195F89C120229CBB2F1
:109D300000F2B884002BC4D0D5F8C83200212846E0
:109D40004FF0020C40F8081FC5F894C2C5E906227E
:109D5000C3E9092118624FF4807203F114019A8259
:109D60009A79012A08BF1863186877F095FCABE769
:109D7000069B00221B0AADF82620013B062BA0D82B
:109D800001A252F823F000BF6D9F0408519F040800
:109D9000279F0408C39C0408C39C0408C59E0408AC
:109DA0007F9F040852EA0C0C8BD1069B7F2B88D82E
:109DB00095F89C32032B84D00698D5F8C8325FFA08
:109DC00080F985F89E9293F89424012A12D01A689B
:109DD0004FF0000C83F81190D2F8001821F4FE61C6
:109DE000C2F80018D2F8001841EA0011C2F80018B1
:109DF00083F894C40422002003F11401C5F89422CE
:109E00004FF48072A8619A829A799862012AC3E914
:109E1000080008BF1863186877F03EFCB9F1000F1E
:109E200040F08584012385F89C324DE740430024AF
:109E30000A31544F0A30544F3844002495F89C326C
:109E4000013B022B3FF63DAF069B012B7FF43CAF5D
:109E50000020D5F8C832C5F8A402A8610422C5F8CC
:109E600094229862C3E9080075E7069B012B00F075
:109E70007A84069B022B7FF424AF4FEA1C2CD5F882
:109E8000C832002085F8A0C2E7E795F89C32013B74
:109E9000022B3FF616AF022A7FF413AFD5F8A43297
:109EA0002846002B18BF4FF0030940F80C9FD5F847
:109EB000C832C5F89422C5E90622C3E90802002287
:109EC0009A6248E72B7C002B7FF4FBAED5F8B832C2
:109ED0000DF126005B6B98470346B5F8B0020028E9
:109EE00000F04484BDF82620002A3FF4EAAE824206
:109EF0004FF0020128BF0246D5F8C802C5F89412F7
:109F000000F11401C5E90622C0E90832002282628C
:109F10004FF4807282828279012A08BF036300684D
:109F200077F0BAFBD0E69DF8180005283FF6C9AED9
:109F300001A353F820F000BFA3A8040895A80408C3
:109F400087A8040879A80408B79C04085FA8040837
:109F50002A7CD5F8B832002A40F07E849B6A0DF145
:109F600026009847022203464270B6E7D5F8B4327D
:109F70000DF12601287C1B6898470346ADE72B7C32
:109F8000002B7FF49EAED5F8B8320DF126001B6B86
:109F900098470722034642709FE798F89C32032BAC
:109FA0007FF4FEACD8F8B8325B69002B3FF4F8AC14
:109FB000002240460099C8F8D4229847F0E447F6BA
:109FC000F07213423FF498AA01EBC102C3F3881464
:109FD0004FEA131CC3F301130BEB8202CE00D2F83D
:109FE0004C7F002C00F008830AF5805E0022384682
:109FF0000132DEF80050944240F8045BF8D107EBE0
:10A000008404002B00F0EC810AF58052234415688B
:10A01000002225FA02F0083204F8010B9C42F8D124
:10A0200073180BEB8303D3F84C7FDBF8EC3C009305
:10A030007318CCF30A0C0BEB83036744D3F8542F4B
:10A04000C3F84C7F6244C3F8542FFFF757BABC4B98
:10A05000D3F8CC3193F89C22042A04D093F89C22A4
:10A06000D2B283F89D22042283F89C22FFF76DBAB6
:10A07000B34B0122D3F8CC01D0F8B83280F89C223F
:10A08000002B3FF41EAB5B6801799847FFF719BBC3
:10A09000D5E9070202442A62002C7FF47EAFDBF888
:10A0A0000C0DDBF8102D0590002A7FF46EAC1846DD
:10A0B000029B03F29C4277F0F3F966E4A14BA24ABB
:10A0C0000344934240F27D81A04BA14A0344934252
:10A0D00040F282819F4BA04A0344934240F238826F
:10A0E0009E4B9F4A03449342C0F06E829D4B9E4A12
:10A0F0000344934240F296829C4B9D4A0344934210
:10A10000C0F094829B4B9C4A03449342FFF454ABAF
:10A110009A4B9B4A03449342C0F0DF82994B9A4A80
:10A12000034493422CBF4FF4C0534FF4E053FFF766
:10A1300045BB1CF0080F00F04881944A96457FF615
:10A14000CDAC1CF4004F3FF4C9AC4FF400429A6010
:10A15000C4E4009C434681E400238AF85732784BDC
:10A16000D3F8CC01D0F8D432AE3350F82330002BE2
:10A170003FF4CBAC90F89C22032A7FF4C6AC5B6A18
:10A18000002B3FF4C2AC00999847BEE4D8E90732EF
:10A19000934200F2288100F09A8198F89C32032BB8
:10A1A00000F0CA818021404677F000FA05230020A4
:10A1B000C8F89432D8F8C8329A7903F51571C3F803
:10A1C0006802012AA3F85402C3E9980008BFC3F843
:10A1D0007002186877F060FAFFF7DCBB03F06002EA
:10A1E0005B0602D5402A7FF46CAD95F89C32013BAA
:10A1F000022B3FF666AD5FFA8CFCBCF1030F3FF615
:10A2000060ADD5F8B8329B68002B3FF45DAD4FF0E0
:10A21000000907992846C5F8D4929847B5F8B022A6
:10A22000002A7FF451AD00287FF44EAD0422D5F80A
:10A23000C832C5F81890C5F894224FF4807203F123
:10A240001401C3F828909A829A79012AC3E90899DF
:10A250007FF48AADC3F8309086E51B06D5F8C85266
:10A2600000F12F81002385F8553205F51573012281
:10A270004FF000099A7083F8009095F89414914279
:10A280003FF422AD286885F894245A78197806900E
:10A2900077F052F9069805F29C42A97977F000F917
:10A2A00085F8949410E503F06003202B00F07E8184
:10A2B000402B00F07B81002B7FF403ADBEF1010F3A
:10A2C0005FFA8CF100F04881BEF1030F00F080814D
:10A2D000BEF1000F7FF4F5AC95F89C32022BDAB298
:10A2E00000F0A881032A7FF4ECAC01F00F031422E4
:10A2F0001CF0800F02FB035340F0B681B3F86431C9
:10A30000002B3FF4DEAC02FB015202F5AA700029DB
:10A3100040F0318200230360D5F8C8320222C5F82C
:10A320009422C5E90622C8E51CF4004F7FF40DAF66
:10A330001CF0200F3FF454AC20229A6050E400BF80
:10A3400040430024405327FFFF340C00401E1BFFF6
:10A350003F420F0000DC0BFF7F4F1200808CF9FEA4
:10A3600020D6130060B6E5FE5FE3160000D3CEFEF4
:10A3700040771B00C05BB3FEC091210000CA91FE74
:10A3800020753800E05459FEE09C41000A30544FDB
:10A390000023EB75C14BD3F8CC01D0F8D432AE33E7
:10A3A00050F82330002B3FF42CAC90F89C22032A69
:10A3B0007FF427AC1B6A002B3FF423AC009998472D
:10A3C0001FE44FF47053FFF7F9B91CF0200F37D09A
:10A3D00020229A60FFF782BB4FF46053FFF7EEB97B
:10A3E000CDF800A024E69A1AD8F8C832C8E90622A7
:10A3F0005A6203F11401059A1A6200229A624FF41C
:10A4000080729A829A79012A01D105981863186896
:10A41000CDE9050377F040F9069B00209A7903F512
:10A420001571C3F86802012AA3F85402C3E9980021
:10A4300008BFC3F87002059877F02EF9FFF7AABAA3
:10A44000974A964503D91CF4004F7FF47EAE1A69F3
:10A45000DAF87432C2F312029B1ACAF86832B8F101
:10A46000000F7FF4BDABDBF8502F002A00F0D28044
:10A47000DBF84C2F1A44CBF84C2FFFF7B1BBD5F8C3
:10A48000D43228460799AE3355F823309B68984755
:10A490001AE4016C824B994203D91368002BFFF632
:10A4A0009FAB00231361136943F400231361136905
:10A4B00043F018031361136943F0C0431361FFF7BE
:10A4C0008FBB4FF001036B7505F11403CFE6D8F88D
:10A4D000182093423FF661AED8F898329A42BFF402
:10A4E0005CAED8F8C83200204FF48072C8F818006B
:10A4F00003F114019A829A799862012AC3E908004B
:10A5000008BF18631868CDE9050377F0C5F8069B06
:10A510004FF0000C059803F51571C8F898C29A79A8
:10A52000C3F868C2012AA3F854C2C3E998CC7FF4E7
:10A5300051AEC3F870C24DE6D8F8B832DB68002BD4
:10A540003FF430AE00224046C8F8D422984729E6AE
:10A550004FF45053FFF732B995F89C32022BDAB220
:10A560004CD0032A7FF4ADAB069B002B7FF4ACAB41
:10A570004806D5F8C89240F00A810422002309F168
:10A580001401D9F80000C5F894224FF48072AB6131
:10A59000A9F8142099F80620C9F82830012AC9E939
:10A5A000083308BFC9F8303077F076F8D5F8B832FC
:10A5B00000229B68C5F8D422002B3FF485AB079995
:10A5C00028469847FFF780BB4FF44053FFF7F6B893
:10A5D00095F89C32022B5FFA83FC0FD0BCF1030F7D
:10A5E0007FF46FAB480603D0069B134300F0CB808B
:10A5F000D5F8C832002030E43C4602E54B06284638
:10A600003FF460AB76F0D2FF2846802176F0CEFF93
:10A61000FFF75ABB029B012103F29C4276F040FFF8
:10A62000FFF7DEBA4FF43053FFF7C8B84FF42053AA
:10A63000FFF7C4B84A067FF444AB1CF0800FD5F88E
:10A64000C8324FF002024FF0000114BF05F11400B0
:10A6500005F5AA700160C5F89422C5E90622C3E990
:10A6600009211862FFF777BB9B8C002B3FF429ABC5
:10A6700001F07F01481C00EB800005EB8000002901
:10A680003FF448AE2422D5F8C83202FB01318A7D5E
:10A69000003A18BF0122026040E600BF4043002498
:10A6A0000A30544F032B7FF40CABD5F8C83202218B
:10A6B000C5E90622C5F8941204355A62002203F156
:10A6C00014011D629A624FF480729A829A79012A6B
:10A6D0007FF44AAB1D63FFF747BB4FF40053FFF70E
:10A6E0006DB8B9F1000F00F0AB80696801293FF443
:10A6F0007FAFD5F8B822C9B22846526890476C4B54
:10A7000093F8D810D5F8B8326960002B3FF470AFD9
:10A710001B682846984700283FF46AAF284676F021
:10A7200081FFD5F8B832297928465B68984702231B
:10A7300085F89C32FFF7C8BAB9F1000F3FF476AD47
:10A740000121D5F8B8326960002B55D01B68284626
:10A750009847002850D0284676F064FF069B85F87D
:10A760009C32FFF7B1BAC5F8A43241E7D5F8C83238
:10A77000A861FFF773BB2422D5F8C83202FB013170
:10A7800091F8562284E7284676F010FF30E701F072
:10A790000F0199F804308B42FFF4EFAE01EBC103D7
:10A7A0001CF0800F4FEA830341D103F5157300229B
:10A7B00009EB030C242303FB019383F855224FF08C
:10A7C00000038CF800108CF8023099F89434012BB7
:10A7D0003FF4D3AE0123D9F8000089F894349CF8F3
:10A7E00004309CF801209CF8001076F07FFE4FF0BA
:10A7F000000389F89434C0E60422D5F8C83200205A
:10A80000C5F894224FF48072A86103F114019A8272
:10A810009A799862012AC3E9080008BF186318688A
:10A8200076F03AFF032385F89C32FFF74DBA1433D4
:10A83000012209EB030C242303FB01935A75BEE7A5
:10A84000022349462846C5F8049085F89C32D5F87D
:10A85000B8325B689847E9E4DB6AFFF780BBD5F85C
:10A86000B4329B69002B3FF42CAA0DF12601287C01
:10A8700098470346FFF731BBD5F8B4321B69002B6C
:10A88000F3D1FFF71EBAD5F8B432DB68002BECD158
:10A89000FFF717BAD5F8B4329B68002BE5D1FFF764
:10A8A00010BAD5F8B4325B68002BDED1FFF709BAD5
:10A8B000384400242DE9F0474A4FD7F88056EE6817
:10A8C0002C69A30701D5B00736D4610701D57207FB
:10A8D0002AD4230701D530071ED4E10601D5F2069C
:10A8E00012D4E30701D5F0073BD414F4025F2BD058
:10A8F00031066CD4600601D571066ED4A20601D56E
:10A90000B30629D4BDE8F0876FF010032B61002354
:10A91000EA6987F89C36E4E76FF008032B610023AF
:10A92000EA6987F89C36D8E76FF004032B610023AF
:10A93000AA6987F89C36CCE76FF002032B610023ED
:10A94000AA6987F89C36C0E7E305D3D53706D1D589
:10A950006FF480732B61CDE76FF020032B61BDE8AE
:10A96000F0876FF001032B611F4B9D42BDD1D7E9EA
:10A97000B9839845B9D098BFA3EB0809D7F8DC3262
:10A980001A4A88BFC8F5805907EB83034244D3F8BD
:10A99000C832002BA9D0D3F814A2C3F80822C3F8F8
:10A9A0001092BAF1000FA0D10121C8441048C3F899
:10A9B00014124B468121C7F8349076F07DFFB8F52C
:10A9C000805F14BF43465346C7F8E4328DE76FF407
:10A9D0000253E2052B618DD5BAE76FF040032B617E
:10A9E0008CE700BF403300240014004014450024CD
:10A9F0004833002402784368022A11D00D490269C5
:10AA0000D1F86C05023A184010B4400AD1F86445F8
:10AA1000D1F8601504FB02005DF8044B0844704750
:10AA2000044AD2F85815D2F8542502EB410202EB41
:10AA300053207047403300242DE9F04F83B002F0DB
:10AA40000207854D019308B9002F6CD1D5F85C45FC
:10AA5000002C53D14FF0FF3E804C4FF0000CF146DC
:10AA6000F046F246E36994F82A60984200F0A38029
:10AA7000002E3BD0012E05EB0C1B0AD19BF87B630B
:10AA8000F30706D416F07E0F03D1F60900F0968086
:10AA9000E0460CF1010C1034BCF1080FE2D1BEF11C
:10AAA000000F04DAB8F1000FC0F29A80C646D5F85C
:10AAB000EC430EF1020605EB0E18013405EB061C03
:10AAC000C5F8EC430CF5547CCCF80440C8E9DB0431
:10AAD0000024CCF8084005EB061494F85A43042CE3
:10AAE00021D8DFE804F02B461C464800E6460CF16E
:10AAF000010C1034BCF1080FB4D1D0E7D5F864656F
:10AB0000D5F8603506FB0434A042A3D395F8083588
:10AB100013B9012385F80835012385F85133002046
:10AB200003B0BDE8F08F95F80835002B54D0012311
:10AB3000022085F8513303B0BDE8F08F12F0010414
:10AB4000D5F868C374D105EB0610019B4FEAE20CFF
:10AB500090F85B83032B6CF3C71880F85B8365D98F
:10AB60004FF6FF70834228BF034605EB0610A0F89E
:10AB70005833002F46D1500707D505EB061090F843
:10AB80005B3343F0010380F85B33D3060AD505EB52
:10AB9000061696F85B33C3F34502013262F34603AF
:10ABA00086F85B33D5F86833012003EB4E230B6046
:10ABB00003B0BDE8F08FC6B9E64678E7666A1034A0
:10ABC000B24588BFE1460CF1010C88BFB246BCF12A
:10ABD000080F7FF447AF62E7012385F80835A6E741
:10ABE000B9F1000F9BDBCE4661E7D5F8EC430CF1E1
:10ABF0000206E646013405EB061CC5F8EC43CCF82A
:10AC0000544368E7D5F8F003D5F8EC33013001334D
:10AC1000C5F8F00305EB0E10C5F8EC33C0F870333F
:10AC200005EB0613042083F85A03A4E723469CE7A8
:10AC3000D5F87835002B3FF472AF5C680CEB4E21F1
:10AC40000023074AA04700283FF469AF05EB06162A
:10AC5000022386F85A3362E74033002490360024FA
:10AC6000616F040870B5114D82B00E4695F85033EF
:10AC7000022B16D1020AC4B2D5F85405002301A94B
:10AC800010440322FFF7D8FE012808D195F850336D
:10AC9000019A022B0CBF22F8146042F8246002B023
:10ACA00070BDC0F3D41200F07F04E5E74033002408
:10ACB0002DE9F04F444E0D4683B0174696F85013D9
:10ACC0002B6803293ED0022961D14FEA13294FF4A2
:10ACD000807A5FFA83F8421E012A23D84FF0010BD5
:10ACE0009F421AD901288CBF00240124D6F8CC2415
:10ACF0001AB1D6F8E81499424CD0D6F8540500237E
:10AD0000092201A94844FFF797FE012823D0022811
:10AD100014D020B12B689F42E8D803202F6003B0E5
:10AD2000BDE8F08FB8F1000F13D096F8083513B9CD
:10AD3000012386F80835012386F85133022003B039
:10AD4000BDE8F08F4FF0800AC3F3D41903F07F08F9
:10AD5000C1E7D346C4E796F85013022913D003295C
:10AD6000ECD1019B53F8282022F07042B2FA82F213
:10AD70002B685209A2421FD0D8445B44D0452B60B7
:10AD80001DD20229EDD1019B33F81820EEE74FF4D4
:10AD9000807AD9E7D6F86415013A02EB41224902DC
:10ADA000B2FBF1F21344B3FBFBF20BFB12320AB11C
:10ADB0005B449B1A2B60AEE79F42B0D8ADE709F128
:10ADC00001094FF00008A6E7403300242DE9F04FB9
:10ADD000DFF884918B4685B0174699F850C309680F
:10ADE000BCF1020FD9F8545540F08280CEB24FF436
:10ADF000807305EB1125A6EB010890449844B942F5
:10AE000008F1FF38B8FBF3F84AD200F00103A84478
:10AE10006FF0404A0193BCF1030F07EB0604A8EB67
:10AE20000503284614BF4FF480728022641A03A9D8
:10AE3000944228BF1446944228BF002E14BF01221A
:10AE400000220A32FFF7F8FD01282AD199F850C3F1
:10AE5000DBF800E0BCF1020F0EF1010324D0B44294
:10AE600055D9039806EB0A02011F00EB820201EBA1
:10AE7000840142F8043F8A4203F10103F9D1DBF86F
:10AE80000030A11B19448F42CBF8001002D1019B66
:10AE9000002B48D18F4205F101054FF00006BAD8CA
:10AEA000012005B0BDE8F08FB44246D903986FF099
:10AEB0000042811E324401EB440100EB420222F8C1
:10AEC000023F914203F10103F9D1A11B71448F426A
:10AED000CBF80010DED1019B002BDBD086466FF053
:10AEE00000434FF6FF72012023442EF81320D8E7C9
:10AEF00001F07F06C1F3D413BCF1030FA6EB0108E8
:10AF00001D4414BF4FF480738023904476E7AEEB6A
:10AF1000060E0EEB04018F42CBF80010BAD1019B54
:10AF2000002BB7D003986FF040434FF0FF3223441B
:10AF300040F82320DBF80010ACE7AEEB060E0EEB7A
:10AF400004018F42CBF80010A4D1019B002BA1D0AB
:10AF5000DDF80CE0C3E700BF4033002430B5044601
:10AF6000C06983B010B9012003B030BD0D46002385
:10AF7000032201A9FFF760FD0128F5D1B4F92020D3
:10AF8000002A19DB019B012D4FEA421103EB42120B
:10AF900003D0022D1BD1E5205854A368D361237838
:10AFA000032B04D10023137753779377D377636A06
:10AFB000190C53839182D6E7064A92F8081509B90D
:10AFC00082F808050123022082F85133CCE7E368B8
:10AFD000E4E700BF403300242DE9F041044682B08D
:10AFE0000D4694F83C30042B7ED8DFE803F02B03A9
:10AFF00069493A003D4E4FF6F777DFF8F48016E0E6
:10B00000BA425BD86EF0CCF801284FF0000134D181
:10B01000206BFFF727FE01282FD1019AD6F868157B
:10B02000531E22638B4228BF0B46C6F8683596F83C
:10B03000502301A9236B032A18469AB2E0D1434555
:10B04000E0D93BE06900204601F0FE01FFF786FFF2
:10B0500001283FD1636B002B18BF022084F83C000D
:10B06000BFE794F82830042B02D1002384F828305D
:10B07000A36B0BB120469847012002B0BDE8F081D8
:10B080001A4E0021E26AD6F8E83406F2C440C6F847
:10B09000E8249B1AD6F8642502FB03F3D6F8CC24E7
:10B0A00002EB4322C6F8CC24D6F8D02402EB43228C
:10B0B000C6F8D024FFF752FF01280BD10420CDE7BA
:10B0C000626B04F130010020FFF780FE012801D1FE
:10B0D0000320C3E70228D0D194F82830042BCCD128
:10B0E000002384F82830C8E70220F5E74033002425
:10B0F000F7FFFF0F38B5044694F83430052B60D8BD
:10B10000DFE803F031251D130D0394F82830082BD8
:10B110003FD02D4B0122022083F8092538BD94F839
:10B120002830082B30D0012038BD00212046FFF701
:10B1300015FF012845D1042084F83400DCE7D4E968
:10B140000B01FFF78FFD01283BD10320F4E74FF0FF
:10B15000FF31206BFFF786FD012832D1E36A002B17
:10B16000F3D00220E8E7184D04F130010120D5F8B2
:10B170005C250232FFF79CFD012813D00238C0B2D3
:10B1800001281ED80520D7E70023012084F82830A5
:10B19000CAE700230122022084F828300A4B83F8F2
:10B1A0000925BBE7E368D5F86415226B03EB41235F
:10B1B000C5F86825C4E90332E36A002BBCD162629A
:10B1C000BAE7002038BD00BF40330024F8B504467C
:10B1D00094F83830032B4CD8DFE803F021180B0229
:10B1E00000212046FFF7BAFE431EDBB2012B41D9F6
:10B1F000F8BD0120626B04F13001FFF7E7FD012883
:10B200004FF00303F0D184F83830E1E700211E4805
:10B21000FFF7A4FE01284FF00203F4D0E4E71B4B34
:10B22000E66893F85023D3F86415032AD3F8CC5476
:10B23000D3F8E80414BF4FF480728022206102FB2F
:10B2400001F1871A0244A5EB412506EB4126E66091
:10B25000C3F8CC54D3F8D054C3F8E824A5EB41216B
:10B26000C3F8D014E36AC4E90C025BB9606201233D
:10B27000C9E7022094F82830062BB9D1002384F8BE
:10B280002830F8BD2763F2E7043800244033002457
:10B290004368C3F308020A44B2F5007F2DE9F04188
:10B2A000054682B00C4605D223446B60012002B0F3
:10B2B000BDE8F08190F91A10481C0AD0474A02EB09
:10B2C000011292F87B1321F0010182F87B13FF2217
:10B2D000AA7695F91B20511C16D0404E023206EB7F
:10B2E000021191F85B13C1F34501012944D90139D9
:10B2F00001F03F0106EB0212FF2692F85B0361F3B7
:10B30000460082F85B03EE762A78022ACCD0334ED0
:10B31000D6F86425B4EB422F4FEA42282EDCD6F84B
:10B320006C751F407A42A24228DCE2192869424526
:10B3300013D32A7E12072DD5D6F8E824411C8A4261
:10B340001ED300D100214344A4EB080868610846DD
:10B35000DB1B08EB070429616B600028A6D096F878
:10B360005023032A35D080B24FF6F77290429DD811
:10B370001A4614446C6099E70021BBE7002096E769
:10B3800096F808250ABB012386F8083586F851335C
:10B390006B68D8E701A96DF003FF0128EED16B6857
:10B3A000A4EB080428699844297868613C44A8EB18
:10B3B0000703019802291A466B602861CDD1D6F89F
:10B3C0007415B3EB412FD4D370E7012286F85123D3
:10B3D000B9E7034A90423FF669AFC9E7403300241A
:10B3E000F7FFFF0F2DE9F0474FF0010882B0044648
:10B3F00094F83830032B00F2A680DFE803F05517ED
:10B400000C020020236C84F8280003B19847022026
:10B4100002B0BDE8F0870022236C84F828200BB12D
:10B4200020469847012002B0BDE8F087237867687E
:10B43000022B03D0454BD3F86C351F40C7F34F2781
:10B440002046FFF7D7FA414E3F1A0546BFB207EB39
:10B45000050C022201A9002328461FFA8CF9FFF7E8
:10B46000EBFA01284FF400724FF00001D0D101989F
:10B470007CF000FAE3694FF4007120460BB1636879
:10B48000EBB1D6F864355A1E914547D20135FFF726
:10B49000FFFE0028DBD196F8083513B9012386F8A2
:10B4A000083586F85183D2E72046FFF723FE0128AE
:10B4B00002D0022847D1032084F8380098E7019B86
:10B4C0004FF020324FF0100E4FF02E0C42F62E6A45
:10B4D000C3F80120C3F80520A3F8092083F800C0B1
:10B4E000D4F824C0A3F820A083F80BE0C3F82220EE
:10B4F000C3F8262083F82A20E26BA3F81AC02CFA9E
:10B500000EFC5A8722FA0EF2A3F814C09A8683F82A
:10B510002BE0D6F864355A1E9145B7D3C3EBC3531D
:10B520002046590201F50071FFF7B2FE28B996F8DE
:10B53000083523B1012386F851330220BCE70123EB
:10B5400086F80835F6E7002062E700BF40330024A4
:10B55000B1F904300F2B2DE9F0410D4682B00446BD
:10B56000164634D02046FFF745FA94F91B80B8F10F
:10B57000FF3F3DD05C4F07EB0813D3F86C33984284
:10B5800012D097F80835002B70D0012387F851337B
:10B590002378022B60D02269002A75D10023012074
:10B5A000336002B0BDE8F081D7F8681301EB4821A1
:10B5B000002967D0AB88204601331BB201EB431151
:10B5C000AB803160FFF716FA28600120E9E74FF4FD
:10B5D0000071FFF75DFE002844D04FF6FF73204650
:10B5E000AB80FFF707FA94F91B80B8F1FF3FC1D198
:10B5F0002378022B3ED02269002ACFD03A4F97F809
:10B600005033032B67D093B24FF6F7718B4294BF40
:10B6100000230123002BBFD130B997F80835002B48
:10B620004CD0012387F851330023112201A9FFF7E1
:10B6300003FA012826D10199D7F86833CB1A48BFFD
:10B6400003F2FF13B3F5805F4FEA63222CD24FFA67
:10B6500082F884F81B80ABE7D7F874256368B3EBF6
:10B66000422F9BD2002002B0BDE8F081012387F871
:10B6700008358AE71C4F6368D7F87425B3EB422F6F
:10B68000CAD38BE7237884E797F85033032B19D07C
:10B6900093B24FF6F772934294BF00230123002B1D
:10B6A0007FF47CAF0020DEE797F8083513B901235B
:10B6B00087F80835012387F85133CAE7012387F853
:10B6C0000835AEE7094B9A4294BF00230123002BB3
:10B6D0007FF464AFE6E7054B9A4294BF0023012351
:10B6E000002B7FF459AF97E740330024F7FFFF0F9B
:10B6F0002DE9F047044688B094F83030042B11D877
:10B70000DFE803F0501361035A00237E9A0640F1EC
:10B71000F9800023112204A9E069FFF78DF90128BF
:10B7200000F0F08008B0BDE8F087C64D03AE04F12C
:10B730001C0705F20C59324639464846FFF708FF08
:10B74000012800F0FA800228ECD195F926355F1C1B
:10B750000AD005EB0313FF2193F87B2385F8261508
:10B7600022F0010283F87B2395F927355E1C17D060
:10B77000023305EB031292F85B23C2F34502012A60
:10B7800040F25E81013A02F03F0205EB031393F8A9
:10B790005B1362F34601FF2283F85B1385F82725CC
:10B7A000042306E0A8486EF0FFFF4FF6FF72012366
:10B7B000228484F830309FE70020E36A207008B0CC
:10B7C000BDE8F04718479F4D95F83435002BA9D1B7
:10B7D00004F11C0705F20C5803AE324639464046C8
:10B7E000FFF7B6FE012840F01881039B002B00F004
:10B7F000F1801A780AB1E52AEFD1D5F868239A1AB0
:10B8000048BF02F2FF12B2F5805F4FEA622180F07A
:10B810004C8109018D4A0A44917B04290CD0D5F84A
:10B82000EC130131C5F8EC13516004219173D5F884
:10B83000F0230132C5F8F02395F92625501C0AD0D3
:10B8400005EB021292F87B1321F0010182F87B13C1
:10B85000FF2285F8262595F92725511C17D002329D
:10B8600005EB021191F85B13C1F34501012940F288
:10B870006481013901F03F0105EB0212FF2085F8D8
:10B88000270592F85B0361F3460082F85B032022F0
:10B89000002118467BF0EEFFD4F831100346D4F8AF
:10B8A000352005A819605A6094F83B20B4F8391087
:10B8B0009A721981627E0193DA7203F06BFA019B2E
:10B8C000002800F0DB809DF816009DF817209DF8F9
:10B8D000191042EA4012BDF814004901A0F2BC70F0
:10B8E00042EA40229DF81A0041EA50019DF81800F2
:10B8F00092B241EAC02188B2D9811A821A83D882D1
:10B90000032356E720466EF04FFF2369002B00F01B
:10B910008980237E03F0F70213F00403227640F0BF
:10B920009780122A00F0AD800022E36A204684F856
:10B93000282008B0BDE8F0471847DDF80C80B8F1C2
:10B94000000F00F0BE8098F80030002B00F0B980A6
:10B9500098F80BA01AF0080F7FF4EDAE0B2204F15B
:10B96000310140467BF0CAFF00287FF4E4AE637EDD
:10B970008AEA0303DF0640F1E48095F926355E1C70
:10B980000AD005EB0313FF2193F87B2385F82615D6
:10B9900060F3000283F87B2395F92725511C3FF4BF
:10B9A000FFAE023205EB021393F85B33C3F345039A
:10B9B000012B40F20981013B03F03F0305EB02122A
:10B9C00092F85B1363F34601FF2382F85B1385F85B
:10B9D0002735E5E695F80C350922022B3FF4E0AE59
:10B9E00095F83435002B7FF4DBAE85F844354046BE
:10B9F000C5F84835C5F84C3585F84035D5F82035BB
:10BA000085F83425C5F83835D5F86835C5F83C359E
:10BA1000FFF7E8FC01283FF4E0AE02287FF482AE95
:10BA20000423C6E6237E1B077FF57EAF054B93F804
:10BA3000EC24002A7FF476AE072283F8EC2473E727
:10BA40000022A2E6403300244C380024AC36002407
:10BA50000023A5682046E66A294684F82830FFF7C7
:10BA600017FC002863D194F82830002B7FF45AAEDD
:10BA70000223C4E90B6584F8283053E644F281724E
:10BA80003BE7E06A0421626AA063204684F83C3008
:10BA900084F8281063636362C4E90B22C4E90233AB
:10BAA00008B0BDE8F0476EF07FBE95F8082512B9E2
:10BAB000012285F8082501226FF00F0185F8512336
:10BAC000A8E695F92635591C0AD005EB0313FF218A
:10BAD00093F87B2385F8261522F0010283F87B2357
:10BAE00095F927355A1C16D0023305EB031292F84C
:10BAF0005B23C2F34502012A21D9013A02F03F0239
:10BB000005EB031393F85B1362F34601FF2283F8FE
:10BB10005B1385F82725237EDB067FF541AE2C4895
:10BB20006EF042FE4FF6FF720223228441E6002EA1
:10BB30003FF4F8AD2046334641E600219CE6002262
:10BB4000DEE7B8F81420B8F81A3043EA0243D5F813
:10BB5000642563625202D8F81C30B3FBF2F102FB99
:10BB60001131A36009B113445B1AE36084F819A092
:10BB700095F926355A1C0AD005EB0313FF2193F8DB
:10BB80007B2385F8261522F0010283F87B2395F9A3
:10BB90002725531C3FF4B4AE023205EB021393F891
:10BBA0005B33C3F34503012B10D9013B03F03F0383
:10BBB00005EB021292F85B1363F34601FF2382F850
:10BBC0005B1385F827359BE60023F7E60023EFE7B4
:10BBD0004C38002410B50378044690F818C0023B96
:10BBE000012B02D91CF0060F6ED11CF0200F44D19E
:10BBF00094F91A20511C0AD03A4BFF2103EB02138F
:10BC000093F87B2322F0010283F87B23A17694F939
:10BC10001B305A1C16D03349023301EB031292F841
:10BC20005B23C2F34502012A4BD9013A02F03F02DD
:10BC300001EB031393F85B1362F34601FF2283F8D1
:10BC40005B13E2761CF0080F0ED0264991F8EC3415
:10BC5000072B06D091F80835002B3DD0012381F841
:10BC60005133002381F8EC340023E26A237084F816
:10BC7000283042B3BDE8104010471B4A0023E0695A
:10BC8000D1691032884206D00133082BB0D0D16977
:10BC900010328842F8D11349023301EB031292F8B3
:10BCA0005B23C2F34502012A1AD9013A02F03F028E
:10BCB00001EB031393F85B1362F3460183F85B1304
:10BCC00096E70022B4E710BD0121FFF747F90128EC
:10BCD000F9D194F818C088E7012381F80835BDE749
:10BCE0000022E5E7403300249036002438B51A4C92
:10BCF00094F834352BB970B190F828201AB1184651
:10BD000038BD002038BD0146442204F20C507BF0BF
:10BD100093FC012038BD04F20C550146442228460C
:10BD20007BF0A8FD94F8503303224FF6FF71022BED
:10BD30002846A4F8261518BF1346D4F8701584F8C1
:10BD40002425102284F80C35C4F8301584F82525F4
:10BD50006EF02AFDDDE700BF40330024314A4FF08A
:10BD6000FF31F8B5A2F5547C00230C4603E0013303
:10BD70001032082B14D092F82A000428F7D10CEBCB
:10BD8000031090F87B03C607F1D4651C106A01D03C
:10BD90008142ECD91C46013301461032082BEAD10E
:10BDA000002C01DA0120F8BD1F4DA61C05EB06137F
:10BDB000D5F87825B3F85813E9B927012F44D5F8F9
:10BDC0006813D5F87835D7F86C0301EB4421DBB163
:10BDD000DC680023154AA047B0B1022809D1D5F884
:10BDE000F03305EB06160122013B86F85A23C5F80D
:10BDF000F0330020F8BD05EB04132701D3F86C03E2
:10BE000012B193689847D9E7D5F8F03305EB0616D9
:10BE100003210122013B86F85A1385F8F423C5F863
:10BE2000F033E6E79036002440330024C56F040861
:10BE30002DE9F04390F8283083B00446013B082BED
:10BE40000BD8DFE803F0383C1F2305290A2E330006
:10BE50000121FFF7C1F8012802D003B0BDE8F0834B
:10BE600000222378216C84F82820002BF5D00322AF
:10BE7000E162D4E9010384F82820834238BF0346F5
:10BE80002046A36003B0BDE8F043A3E6002103B061
:10BE9000BDE8F043FFF7A0B803B0BDE8F043FFF7FB
:10BEA00095B903B0BDE8F043FFF724B903B0BDE88E
:10BEB000F043FFF797BA03B0BDE8F04318E4DFF8AA
:10BEC00034914368D9F86C65026B19461E40D9F865
:10BED000640594F800C0B5184702B5EB402F41D374
:10BEE0004FF6F778BCF1020F14D025692846002DD3
:10BEF0005AD16168A3680020E26A8B4284F8280066
:10BF000038BF0B46A360002AA7D0204603B0BDE887
:10BF1000F04310476168D9F87405B1EB402F5CD24B
:10BF20002069217E090732D5D9F8E814451CA942B9
:10BF30002AD299F80815002943D1012389F8083538
:10BF400089F85133226B636894F800C0D21B3B44DC
:10BF500032449B1B00269742194663602263C4E962
:10BF60000450BFD9BCF1020F37D02569002DC1D0D4
:10BF700099F85033032B36D0ADB24FF6F7739D428C
:10BF8000B8D811446160B5E7E0D10025DEE701A92A
:10BF90006DF006F901287FF460AF2069019D94F8E7
:10BFA00000C06368226BD1E799F8501303290ED0C3
:10BFB000A9B2414594BF002101210029B1D0616897
:10BFC000D4E7012189F8511394F800C0BEE708496D
:10BFD0008D4294BF00210121EFE7D9F87435B1EB10
:10BFE000432FCED386E7024B9D4283D8C9E700BFDB
:10BFF000F7FFFF0F40330024704700BF0079704700
:10C000000079C0F34010704700794009704700BFC5
:10C01000704700BF704700BF03685A1C0260197068
:10C02000704700BF03685A1C02601970704700BF58
:10C03000024B186803681B68184700BF206500247E
:10C040002DE9F0413A4E33787E2B03D00027384655
:10C05000BDE8F08108214FF4FC4341F221041AB2FB
:10C060005B00002A84EA42009BB2B8BF83B2013968
:10C07000F5D1B6F80140002C37D02E4A2E4DAA42F9
:10C08000E4D2052CA2F106028CBF0027012714443C
:10C09000AC4228BF47F00107002F46D141F2210EE4
:10C0A000A24214D0501E04F1FF3810F8011F0822DC
:10C0B00083EA012319B25B0000298EEA410C9BB28E
:10C0C000B8BF1FFA8CF3013AF4D14045EDD1218875
:10C0D00061B1A21DAA42BAD2052904EB0100224691
:10C0E000B5D9A842B3D20446DAE7144C671E41F230
:10C0F0002105BC4617F8012F83EA0223082219B252
:10C100005B00002985EA41009BB2B8BF83B2013AC7
:10C11000F5D16445EDD16788094AFF1A231DB7FAA6
:10C1200087F79B1B7F09938091E70F468FE700BF3E
:10C1300000000208070002080000040801000208CD
:10C140002065002490F83C20034602F0FF0012B165
:10C15000002283F83C2070474FF48053838170475E
:10C160004FF40063838170474FF40063838170470D
:10C170004FF40063838170474FF4006383817047FD
:10C18000074B10B403F11001002453F8042B824232
:10C1900008BF43F8044C8B42F7D15DF8044B70475D
:10C1A0002865002470B5374CE08C238BB4F93050EF
:10C1B0001B1AA08CB4F91EC000FB03F3B4F92E00C7
:10C1C000E66B05EBE335C00290FBF5F000EBE330E6
:10C1D000B4F92A30A0F57A6E60630EFB0EF50EFB03
:10C1E0000CFC2D134FEAEC2C05FB03F30CEBE32CBA
:10C1F000B4F9283005FB03F3B4F920501B140EFBEF
:10C2000005F503EB6533B4F91C5002330CEB850CD8
:10C21000B4F938509B10648C0CFA05FC03F500430C
:10C220000CF1020C04FB03F34CF25034A6EBAC0C03
:10C230002C41DB0B04FB0CF4002C1EDB6400B4FB74
:10C24000F3F389B11C1240F6DE3504FB04F405FB60
:10C2500004F40D4D241403FB05F504EB254404F60A
:10C26000CF6403EB24130B602AB100EB8000400085
:10C27000083000111060012070BDB4FBF3F35B00C7
:10C28000DFE700BF2065002443E3FFFF0120704784
:10C29000012070472DE9F04F734D85B00F46286C93
:10C2A000B5F844300092C3EB2014B5F948205B0088
:10C2B000B5F950E004FB04F4B5F84A80C3EBE003A1
:10C2C000CDF80CE02413B5F95260B5F9541002FB17
:10C2D00004F4B5F94620029602FB03F3A413B5F962
:10C2E0004C2004EBE3242B6EA4F5FA300193B5F94E
:10C2F0004E3080FB00EA4FEAE37B82FB002C03FB1D
:10C300000AF94FEA0C3CEC650EFB0B99A3FB0E3BC4
:10C310004CEA125C1203CB441B0A43EA0B639B18E2
:10C320004CEB2B2BA3FB08320BF5004B08FB0B2B24
:10C330004FEAEB734FEA6B0953EA6B0B00F0928004
:10C34000029E01FB0AFA019A86FB0008039EC2F5D1
:10C35000801C4A464FEA48484FEAE17948EAD0381B
:10C360000EFB09A94004A1FB0E1E4118F1444FF039
:10C3700000000CF0004E49EB08094EEA5C0E411833
:10C380004FEACC7C09EBC609BCEB010C6EEB090E45
:10C390001CEB0C084EEB0E0118EB0C084EEB0101E8
:10C3A0004FEA88104FEA811918EB000049EA9869B2
:10C3B00041EB0901890041EA9071800010EB0C000B
:10C3C0004EEB0101890041EA9071800010EB0C00F6
:10C3D0004EEB010176F062FDB5F95A304FEA613853
:10C3E00084464FEA503EB5F956204FEAE37A03FB04
:10C3F00008F94EEAC14EB5F958000EFB0A99A3FBA5
:10C400000E35A94403FB08F50EFB0955A3FB0E3EB0
:10C4100075445B0E4FEAE07E43EAC51313EB0C0351
:10C4200041EB656500FB01F10EFB0C11A0FB0C0C50
:10C430006144C00C40EA41301B1845EBE1451B0A42
:10C4400043EA056303EB02130FB11B0A3B60009B39
:10C4500023B104EB8404803424121C60012005B055
:10C46000BDE8F08F0023EFE720650024012070472E
:10C47000012070472DE9F04FC94C83B0B4F8680033
:10C48000636EB4F86A50A3EB002394F96C00009239
:10C49000A5FB03574FEAE07CA3FB0336BF0400FB78
:10C4A00006F647EA953703FB0C66AD04A0FB0303D1
:10C4B0004019334443EB0703002B02DA013843F100
:10C4C0000003DF17C4E92037002900F0158103FBC2
:10C4D00007FCD4F88850A3FB030606EB4C064FEA92
:10C4E000901E4FEAA6184EEA866E0EFB07FC03FB71
:10C4F00008CCAEFB03E81CEB080C00F14B814FEAC3
:10C500001E2E4FEA2C224EEA0C6E94F972C0019254
:10C510004FEAEC780CFB02FA0EFB08AAACFB0EC843
:10C520001AEB080A00F131814FEA5C1CB4F96F8004
:10C530004CEACA6294F971C0A8F580484FEAEC7BD6
:10C540000CFB06F900FB0B99ACFB00CBD944B4F90A
:10C550006DB04FEA8909ABF5804B49EA9C794FEA07
:10C560008B3B4FEA8C0C0BEB6A1A12EB0C0C4FEA6C
:10C57000E87B4AEB090A08FB07F903FB0B99A8FBC8
:10C58000038BD9444FEA495949EAD8294FEA485818
:10C590001CEB080C4AEB0909B9F1000FC0F2EE8060
:10C5A00094F978804FEA1C6C019A4FEAE87A08FB0C
:10C5B00002FB4CEA092C4FEA29690EFB0ABBA8FBD7
:10C5C0000E8E1BEB0E0B00F1D48094F977E04FEA4E
:10C5D000581848EACB6A0EFB06F84FEAEE7600FBE5
:10C5E0000688AEFB006EF044B4F873E04FEA08181A
:10C5F0004FEACE3E48EA167836010EEB6B1E1AEB78
:10C600000606B4F875A04EEB080EAAFB03800AFBE1
:10C610000700800540EA98204FEA885816EB080684
:10C620004EEB000EBEF1000FC0F29F80B60894F9E9
:10C630007B00ACFB05C846EA8E7616EB0C0605FBC4
:10C64000098C4FEAE07900FB07F84CEBAE0CB4F92B
:10C6500079E003FB0988A0FB0309C8444FEA0E49AF
:10C6600010EB090048EBEE78A0FB050E05FB08EE89
:10C67000BEF1000F72DB400B40EACE404FEA6E3E47
:10C68000A0FB050805FB0E8EBEF1000F5FDB400A24
:10C6900094F97C8040EACE5036184CEB6E24A5FB12
:10C6A000050E4FEAE87C00FB0CFC08FB0ECCA0FB5F
:10C6B00008081CEB080C43D4000C40EA0C404FEA7D
:10C6C0002C4CA0FB050E05FB0CE5002D34DBC0094E
:10C6D00040EA4560801944EBE514051844EB040674
:10C6E0002D1844EB0606F60046EA5576ED002D18A7
:10C6F00044EB0604240C0C60009A9AB1D91847EB5D
:10C700000700C91847EB0000C00040EA5170C9009B
:10C71000C91847EB0007002F08DB890B009B41EA93
:10C7200087411960012003B0BDE8F08F43F6FF7325
:10C73000C91847F10007F0E77F3045F10005C6E76B
:10C740004FF6FF7E10EB0E004CF1000CB4E740F208
:10C75000FF1810EB08004EF1000E98E741F6FF7845
:10C7600010EB08004EF1000E85E703364EF1000E87
:10C770005CE718F11F084BF1000B26E76FF07F48CC
:10C780001CEB080C49F100090AE71CF11F0C4AF1E7
:10C79000000AC9E61EF1FF0E4CF1000CAFE600BF27
:10C7A0002065002431B10A4BD3ED2A7AFDEEE77AF9
:10C7B000C1ED007A52B1064B9FED067AD3ED2B7A8C
:10C7C00067EE877AFDEEE77AC2ED007A01207047C6
:10C7D000206500240000C8422DE9F04F5F4D9346CC
:10C7E00085B0B5F8BE30D5F8B0001B02B5F8BCE096
:10C7F000B5F8BA40C21AB5F8B830019167EB07072F
:10C80000AEFB020C1B04B5F8B6100EFB07CCC0093A
:10C81000B5F8C060C90340EA4C604FEAEC1CC01890
:10C82000A4FB023E04FB07EE4FEA13234CF1000C7D
:10C8300043EA0E634FEA2E2E5B18A6FB021406FB9A
:10C8400007444FEAD1514EF1000E41EA4421E4156C
:10C8500011F5FA6844F10006B8F5FA6F029676F120
:10C86000000630DA01FB04F60394A1FB014A0AEB4F
:10C87000460AA6004FEA8A09361949EA9479384CE3
:10C880004AEB09094FEA560AB6084AEAC97A46EA63
:10C890008976B0EB0A0A6CEB690C9E1B50466EEB76
:10C8A000A90E3346A045029E4FF0FF34A64126DB79
:10C8B00002FB07F7A2FB022101EB4701D20F42EA7C
:10C8C0004102B8EB0208019C84B1D5F8C410A1FB69
:10C8D000033201FB0E225B0D43EAC22352151B1AE1
:10C8E00062EB0C02DB0B43EA42432360BBF1000F17
:10C8F00001D0CBF80080012005B0BDE8F08F40F6F4
:10C90000AC56039C891944F1000401FB04F4A1FB1B
:10C91000016101EB4401F4004FEAC109341B49EA0B
:10C92000567961EB090924184CEB090C2046B4191F
:10C9300041EB0109A41941EB09094FEA890949EAC8
:10C940009479A400A41B69EB0109610841EAC9714B
:10C95000591A6EEB690E0B46AAE700BF206500244A
:10C9600024FAFFFF01207047104B10B4104C1B68D5
:10C97000D4F8C8001B1AFA2B0BD811B1D4F8D43054
:10C980000B6012B1D4F8D830136001205DF8044B6D
:10C990007047D4F8CC30002223F00403104684F80A
:10C9A000D020C4F8CC305DF8044B70474C3A0024DA
:10C9B000206500242DE9F8430D46D0E900311344E9
:10C9C0008B4220D80446AE18076BCAB14FF000095D
:10C9D00000F10C0801E0AE4212D0E36A5A1C234475
:10C9E000E262202A15F8011B1973F4D14146204652
:10C9F00017B9F6F7B5FE0746AE42C4E90B97ECD17E
:10CA00003846BDE8F8834FF0FF37F9E72DE9F04FDE
:10CA10005422044600218BB09F487AF02BFF9F4A96
:10CA2000611EE01C144611F8013F5D1E052D88BFF4
:10CA30000023884244F8043BF5D102F1100311466B
:10CA400051F8040B012800F019818B42F8D11146EE
:10CA500051F8040B022800F007818B42F8D11146EF
:10CA600051F8040B032800F0F5808B42F8D152F8FE
:10CA7000041B042900F0E4809342F8D105204FF014
:10CA80001A094FF0000ADFF81082854DFFF778FB96
:10CA9000844F0620FFF774FB98F80C407CB32046C7
:10CAA00098F90D6007F054F928B1052380F8079034
:10CAB000837100230372032107F006F9002302E0CB
:10CAC00001331C2B3DD015F83320A242F8D105EBE1
:10CAD000C3035868F42106230122C8F8100001FBA3
:10CAE000067688F816309244D6F8F03088F815208B
:10CAF00086F8EC209A1888F81430C6F8F02009F16E
:10CB0000010908F10C085FFA89F9B9F1200FC3D1C6
:10CB1000BAF1000F12D0DFF88CA14FF0000BDFF854
:10CB20009C81D14699F8EC306BB90BF1010B09F1FE
:10CB3000F40908F58C78BBF1030FF3D10BB0BDE815
:10CB4000F08F0020C6E7B9F806006CF083FBB9F857
:10CB500004006CF07FFBD9F8F0304FF4403CF42136
:10CB6000012BC9F8283001FB0BA1D9F80020D4BF54
:10CB7000002301234FF0030EC9F81020C9F81C3020
:10CB80000023C9F8383089F82C30C9F83030C9F89A
:10CB9000203089F8483004930823C9E905C34FF4CD
:10CBA0008063C9F834304FF48073A9F824304FF40F
:10CBB0008053C9E90FE34B6E002B69D093689F0047
:10CBC00003D59168384B0B4093609368DE0014D412
:10CBD000364B37491B689068B3FBF1F33549013395
:10CBE000014041F0805191600493049B2BB1049B60
:10CBF000013B0493049B002BF9D19368DD001CD406
:10CC0000F423012103FB0BA30191596E41F01001A4
:10CC10005966996E41F001019966F423916803FB0E
:10CC20000BA301F00401586E00F01000014347D03F
:10CC30005A6E42F010025A6677E700230193ECE740
:10CC40001D4B342193F8302183F80C11013283F805
:10CC5000302113E71849352491F8300181F800415B
:10CC6000013081F8300102E71349312491F8300195
:10CC700081F8F440013081F83001F0E60E493024AB
:10CC800091F8300181F8E840013081F83001DEE6AA
:10CC90008B6689F8603091E7FC65002428650024E4
:10CCA0006C7F0C08D0170024C0FFFF5F0000002439
:10CCB000400D0300C0FFFF6F20650024000000301E
:10CCC000596E21F4817141F0020159669368DC07C5
:10CCD00013D4784B9A4200F0178303F580739A427D
:10CCE00000F01283744B9B68D90706D473498B6894
:10CCF00023F47C1343F440338B60714B71491B6800
:10CD0000D368194043F208030B43D36091689368DA
:10CD100001F0040103F00803194300F06182D9F81F
:10CD20001000D9F81C30012B00F05583036B23F061
:10CD30000F030363F42303FB0BA35A6E22F00302D9
:10CD400042F001025A66019A002A7FF4EEAE019A7F
:10CD5000059299F86020012A3FF4E7AE826801212C
:10CD6000940789F86010816802D4CA0700F18882AC
:10CD7000F421554A554B01FB0BA14C6E224042F069
:10CD800002024A668268134043F00043836083686E
:10CD90004F4A002BC0F2E581F4214E4B4E4C4FF42C
:10CDA000806C01FB0BA14D4803274D4D4A6E22F0CC
:10CDB000030242F001024A66D9F80820D9F80C6053
:10CDC000A24218BF9A424FF40054C9F878600CBFD1
:10CDD00001230023C9F89C70824208BF43F001037D
:10CDE0001830824208BF43F001031830824208BF66
:10CDF00043F001031830824208BF43F001031830AA
:10CE0000824208BF43F001031830824208BF43F05A
:10CE1000010300F55670824208BF43F00103183049
:10CE2000824208BF43F001031830824208BF43F03A
:10CE300001031830824208BF43F0010318308242D8
:10CE400008BF43F001031830824208BF43F00103DA
:10CE50001830824208BF43F00103002089F86000C7
:10CE6000C9F89800C9E91F00C9E928004FF400601B
:10CE7000C9E921C04FF48070C9E923404FF4003064
:10CE80004C46C9F89400286844F8742F1BB9154B18
:10CE90009A4240F0BE84F423022103FB0BA383F8E3
:10CEA000A9100021136889F8A81023F0010313606A
:10CEB0001FE000BF002002400060025800630258DB
:10CEC0000010005C03C0F0FFFDEEFFFFC0FFFE3F5F
:10CED00000F8C32510000240280002404000024034
:10CEE000802C0024B80402402B681B1A052B00F28A
:10CEF000BD811368DF07F7D4A44913680868A44903
:10CF00006FF30F001940A34BB0F1005F43EA010338
:10CF10000BD32E2E40F21F833F3E132E05D89E4882
:10CF2000F040C00701D59D4B0B4313602046536969
:10CF300023F007035361F5F7A7F9D9F8D02002F0E1
:10CF40001F013F228A408260D9F87420944B954992
:10CF5000954E8A4218BF9A4201F11801A2EB0600D1
:10CF60000CBF012300238A4208BF43F0010318319C
:10CF70008A4208BF43F0010318318A4208BF43F0D8
:10CF8000010318318A4208BF43F0010318318A4275
:10CF900008BF43F0010318318A4208BF43F0010380
:10CFA00001F556718A4208BF43F0010318318A42E5
:10CFB00008BF43F0010318318A4208BF43F0010360
:10CFC00018318A4208BF43F0010318318A4208BF72
:10CFD00043F0010318318A4208BF43F001031831BE
:10CFE0008A4208BF43F001037049511AD1F1000C85
:10CFF0004CEB010C6E498A4208BF43F001036D49B6
:10D000004642A2EB010701F1140146414CEA030339
:10D01000D7F1000EA2EB010043EA06034EEB070E28
:10D0200041424EEA0303414163480B430291634985
:10D03000571A794279410B430391111A48424841EA
:10D040005F49571A0343794279415E4FBA4214BF90
:10D05000002701270B4301D1002F3BD046EA0C06E5
:10D06000029B4EEA060E039E43EA0E031E43D3B212
:10D0700030430143394300F05D831422083B01260D
:10D08000514FB3FBF2F3514A9E401A449200D9F833
:10D090007C30C9F8DC60802BC9E9352700F00881B5
:10D0A000D9F87830D8B2013B072B10607E6000F2CF
:10D0B0000481461E002900F06885454B454903441C
:10D0C0009B0001220020B240C9E93831C9F8E820AC
:10D0D00018604A60F423012100204FFA8BFE03FB05
:10D0E0000BA30A460295C3F8C80083F8A91009F1FA
:10D0F0001003C9F85C40C9F8AC30374B04E001328A
:10D100000C33072A00F00A81597D0029F7D093F9E2
:10D110000D107145F3D1002101989D7D06912F4995
:10D12000039501EB80011869D1F8E04099F860108F
:10D1300001293FF4FAAC4FF0010189F86010D9F8E9
:10D1400010108D686F0740F10F81F42303FB0BA3D0
:10D150005A6E42F020025A664FF0000389F86030A0
:10D16000E3E4059B01330593059B9342FFF40FAE67
:10D17000F422002102FB0BA2536E23F0120343F0B2
:10D180001003536689F86010CFE400BF0010005C04
:10D190003F8010FE002D02000F030F00002D120033
:10D1A00010000240280002401C5402580854025843
:10D1B000B8040240305402586C5402585854025873
:10D1C0008054025894540258805802580096001611
:10D1D0003F96001640590258FC6500246C7F0C08ED
:10D1E000D068AA4B0340D9F8440043F00303D3604E
:10D1F000136923F001031361136923F070430343A0
:10D200001361A34B9A4277D003F580739A4273D08F
:10D21000A04B9B6813F4403F14BF01230023002B55
:10D2200000F0EA80F5F798F9D9F814300146B3F523
:10D23000003F00F01E82B3F5403F00F01E82B3F5C0
:10D24000803F00F01682944BD9F810001A6841F222
:10D250000303B3EB124FC0F0C780904B9942836831
:10D2600000F20F8123F4807383605AE5F4232022B7
:10D2700003FB0BA3C3F8C820032283F8A92054E4BE
:10D28000826802F00D02012A1DD05A6E002142F080
:10D2900010025A669A6E42F001029A66F42303FB6A
:10D2A0000BA35A6E42F010025A6689F860103CE4F3
:10D2B0000023C9F8783013607E600023C9E9383351
:10D2C000C9F8E83006E78268754B764D134043F0A5
:10D2D00002038360032303602A688368DE077FF507
:10D2E00047AD2B689B1A022BF7D98368DF07F4D56B
:10D2F000F42303FB0BA3C8E76B4B9B6813F4403F7D
:10D3000014BF012300238AE7614B68499B68896841
:10D310000B43D8073FF5F1AC6349E8E4D9F81010A6
:10D320005B4B029D9942D9F8F07052D003F580739F
:10D3300099424ED0574882688B685E073FF5F5AB3F
:10D3400099F86030012B3FF4F0AB02F01F0240F27D
:10D3500021230124D34089F86040234040F0FF801E
:10D3600089F86030FFF7E1BB00284FEA906709DBDE
:10D37000C0F31305002D40F0E6800125BD40CE69C5
:10D380002E43CE61A50901F1300604F01F0407F019
:10D390001F0705F00C054FF01F0CA7400CFA04FC0A
:10D3A000745924EA0C043C4374518D688C6805F070
:10D3B000040504F008042C4300F082808C68E60722
:10D3C00032D501990131C9B20191002189F860106B
:10D3D00095E63548AFE7026BD9F8283022F00F0206
:10D3E000013B13430363A5E4314B994242D8836860
:10D3F00023F44073836094E42E4B9A6D02F4403220
:10D40000B2F5803F00F08881B2F5003F00F06981FD
:10D41000002A7FF418AF1B681A017FF514AF07A824
:10D42000F5F7D8F807990EE7D1F8C040C0F3130517
:10D43000002824EA0504C1F8C040C2DA144CA14215
:10D4400000F01D8104F58074A14200F01881114C98
:10D45000194EA568B668F60740F11B81F423002138
:10D4600003FB0BA35A6E42F020025A6689F8601043
:10D47000FFF75BBB114B994200F22881836823F4CC
:10D48000407343F4807383604BE400BFFCBFFFFF35
:10D4900000200240006302580010005C002D3101A2
:10D4A000C0FFFF7F802C00240023024000210240A7
:10D4B00021BCBE00004402580060025841787D0142
:10D4C000C0F30454039FC50D01F1140607FA04FCD0
:10D4D000072705F00405A740745924EA070444EA25
:10D4E0000C0474519F4C246804F07044B4F1805FC4
:10D4F000CC6800D0CC680C6E850604F0F844B4EB20
:10D50000806F03D10C6E24F000440C664C6E04F066
:10D51000F844A54203D14C6E24F000444C668C6E56
:10D5200004F0F844A54203D18C6E24F000448C66CC
:10D53000CC6E04F0F844A5427FF440AFCC6E24F0EA
:10D540000044CC663AE790FAA0F50126B5FA85F5D5
:10D5500006FA05F513E7282E7FF6E7ACE3E48B68BF
:10D56000DC0733D48C68804B1C421FD18C687F4B06
:10D57000234043F001038B602C688368DB0602D0F4
:10D580007B4B994222D079480B68DE071ED48B680A
:10D59000DE0704D48B68034043F001038B602B68E3
:10D5A0001B1B022BF0D90B68DB07EDD4F42303FB24
:10D5B0000BA35A6E42F010025A669A6E42F00102B4
:10D5C0009A66002389F86030FFF7AFBAF420694B00
:10D5D00000FB0BA0446E234043F48073436612B1FA
:10D5E000634B994206D0F42303FB0BA35A6E22F43B
:10D5F00080125A66F42303FB0BA35A6E12F4805276
:10D6000000F0A8809A6E22F006029A66D9F85C00B3
:10D610000024594BD9F83C20C363584B0364584B42
:10D62000C3641C230B604B6889F8604043F010030F
:10D630004B60CB6823F003031343CB6090F8343086
:10D64000012B0CD0012380F8343090F83530012BB9
:10D6500000F02C814FF4006380F834404365D9F822
:10D660001020424B91680B4043F004039360FFF796
:10D670005CBA1B0CB1FBF3F1E5E58108E3E5414C35
:10D68000414E3B4FA568B668BF683E43F7073FF57C
:10D69000E5AE3E4F05F0E076B84200F08D803C4F9D
:10D6A000B84200F0A7803B4FB8427FF48AAE6F02C9
:10D6B0003FF587AE384881427FF483AEA16821F000
:10D6C000E071314341F48001A1607AE6334B994225
:10D6D00083682AD823F4407343F400738360FFF710
:10D6E00020BBDA6C186802F04052470701D5002AC7
:10D6F00032D02B4B1B68DE0503D5B2F1805F00F002
:10D70000D380274B1B689D037FF59DAD254BB2F160
:10D71000005F08BF194696E51B689B007FF593AD37
:10D7200007A8F4F7F1FF09998DE543F4407383608E
:10D73000FFF7F7BA1C48103B10441822A828B3FB87
:10D74000F2F300D80833194A0126194F1A449E40B3
:10D7500092009CE49A6659E71B681649C3F3C1031B
:10D76000D94070E50010005C3F000080C0FFFF7FE3
:10D7700000210240FEF0FFFF0100040855000408EC
:10D78000590004080023024000200240000084CB1E
:10D79000000052C70000B8CF0060025881F0FA02C2
:10D7A0000044025840787D01F0FBFDBF008200106C
:10D7B000800802400090D0032D023FF502AE9F4842
:10D7C00081427FF4FEAD9E499E480968B1FBF0F1AD
:10D7D000A068013120F0E0704900304340F40000BF
:10D7E000A060069102E00699013906910699002988
:10D7F000F9D1E6E5E8013FF5E4AD904881427FF4D8
:10D80000E0ADA16821F0E071314341F08071A16089
:10D81000D7E58D4B8D48824218BF9A4200F1140023
:10D820000CBF01230023824208BF43F001031430E0
:10D83000824208BF43F001031430824208BF43F024
:10D8400001031430824208BF43F0010314308242C6
:10D8500008BF43F001031BB97D4B9A4240F09B8106
:10D86000F42102207B4B01FB0BA1134481F8A9009A
:10D870001421B3FBF1F38340106842F2A0516FF31F
:10D8800010100143002089F8A80020461160C9F853
:10D89000D030F4F7F9FCD9F8D02002F01F010122B2
:10D8A0008A404260FFF750BB6B49CCE403684031CB
:10D8B0006A4A6B4DAB4218BF934205F118050CBF85
:10D8C00001220022AB4208BF42F001021835AB42F0
:10D8D00008BF42F001021835AB4208BF42F0010216
:10D8E0001835AB4208BF42F0010205F55675AB4250
:10D8F00008BF42F001021835AB4208BF42F00102F6
:10D900001835AB4208BF42F001021835AB4208BFE0
:10D9100042F001021835AB4208BF42F0010218354F
:10D92000AB4208BF42F001021835AB4208BF42F0DB
:10D9300001021835AB4208BF42F00102142505FB75
:10D9400007F7022580F83550464D4465464CAB42FA
:10D9500018BFA342856D0CBF0124002401950AB9AC
:10D96000002C37D01D6825F00105D0E919EC1D60A9
:10D97000C56E002C40F0FF80456EC5F804C0C56E32
:10D98000002D75D0D0E91C566E60002C70D0C56D8E
:10D99000019E05F01F0C3F2505FA0CF5B5601D68CA
:10D9A00025F480251D6085685F60402D00F0DF80D4
:10D9B0009960C3F80C8014B9002A00F095801968AA
:10D9C00021F01E0141F016011960196841F00801AB
:10D9D0001960B9E01C4DDFF874C0634518BFAB4255
:10D9E0000CF1140C0CBF01250025634508BF45F060
:10D9F00001050CF1140C634508BF45F001050CF15D
:10DA0000140C634508BF45F001050CF1140C634587
:10DA100008BF45F00105D3F800C02CF0010CC3F895
:10DA200000C0DFF848C0634508BF45F0010515B9DF
:10DA3000074DAB4258D1D0F868C09DE7006002584E
:10DA400000000024400D0300085402581C540258E2
:10DA500094540258F8ABFDA700093D004000024075
:10DA60005800024028000240100002408054025832
:10DA7000002A8CD14B4DDFF834C1634518BFAB424F
:10DA80000CF1140C0CBF01250025634508BF45F0BF
:10DA900001050CF1140C634508BF45F001050CF1BC
:10DAA000140C634508BF45F001050CF1140C6345E7
:10DAB00008BF45F001050CF1140C634508BF45F0A3
:10DAC000010515B9384DAB420ED1C56D019E05F06B
:10DAD0001F0C012505FA0CF5756085685F60402D07
:10DAE0004FD09960C3F80C8030492E4DAB4218BF1F
:10DAF0008B4205F128050CBF01210021AB4208BF74
:10DB000041F001011D6825F00E0545F00A051D6074
:10DB1000274DAB4208BF41F001011435AB4208BFAD
:10DB200041F001011435AB4208BF41F001011D680D
:10DB300045F004051D601F4DAB4208BF41F00101D7
:10DB400011B919498B420DD1016E0D68EA0303D555
:10DB50000D6845F480750D60C16E19B1086840F418
:10DB6000807008601A6842F001021A6077E5C3F815
:10DB70000880D9601FE7CEF804C0002D7FF402AF03
:10DB800005E7C3F80880D960AEE70B4B0B490344A7
:10DB90009B00FFF796BA4023C1F8C83081F8A970FE
:10DBA000FEF7C3BF08540258945402581C5402583C
:10DBB00044540258805402583F82001040090240E9
:10DBC00038B51446002944D0344B0D469FED344AF5
:10DBD00093ED4D7AD3ED506AB8EEC76AB3F9502190
:10DBE000B8EEE60AD3ED4E7A04EE902AB3F94C2152
:10DBF000C6EE046A93ED517A05EE902AB3F94E21F0
:10DC000005EE102AB3F94A21B3F94831F8EEE44A97
:10DC100006EE102AF8EEE55AF8EEE77AB8EEC55AA5
:10DC2000B8EEC77AC7EE843A07EE903AB8EEC66A05
:10DC3000E6EEA45AF8EEE77AA6EE856AA6EEA57A95
:10DC4000E6EE867AA6EE870AA3EEA70A77F068FCCE
:10DC500028600CB3114BF6EE005A9FED115AD3ED2C
:10DC60004E6AB3F93E21F8EEE66AB3F93C3107EEAD
:10DC7000102A9FED0C6A07EE903A86EE850AB8EE00
:10DC8000C77AF8EEE77A20EE070AA7EEA50A20EE9B
:10DC9000060A77F045FC2060012038BD206500248D
:10DCA0000000F04A0000C8420369416853EA0102DB
:10DCB000F0B43B4E5DD0C56A013390ED067A6A1C24
:10DCC000876830EE077A0361012AC26280ED067A26
:10DCD00042D090ED075A07EE902AD0ED096A70EE17
:10DCE000455A3468B8EEE76A611AC5EE867AB942D9
:10DCF00077EE857A30EE670AC0ED087AC0ED077AD4
:10DD0000F0EE667AE5EE807AC0ED0A7AC0ED097A27
:10DD100001D8F0BC7047012A28DD06EE905AF8EED3
:10DD2000E66A87EEA66AB5EEC06AF1EE10FA1DDB70
:10DD3000F1EEC67AF4EE677AF1EE10FA16D6D0ED6F
:10DD4000056AF4EEE76AF1EE10FA15D5037BFBB134
:10DD50000323F0BC03707047326880ED080A521A42
:10DD6000002180ED070ABA424162D2D9DFED0D7A77
:10DD7000E5E7316841609EE707EE903A0223F8EE4E
:10DD8000677A0370F0BCC7EE276AC0ED066A704779
:10DD9000316800220361C36241608261B9E700BF5C
:10DDA0004C3A00240000000010B5DFED4F4A8446D5
:10DDB00000F1480E0346DA6AB1EC017AD3ED067A37
:10DDC000013277EE877A012ADA62C3ED067A71D0E2
:10DDD00093ED075A07EE902A93ED096A77EE455ABC
:10DDE000F8EEE77AC5EEA76A76EE857AF0EE466A37
:10DDF00037EE677AC3ED087AE5EE876AC3ED0A6A03
:10DE0000C3ED077A1833C3ED036A7345D3D1374C9A
:10DE1000416822680369521A816801338A420361AA
:10DE200047D990ED056A0022DFED2F5ADCF82C105F
:10DE3000F0EE657ADCED0A6A012901F1FF3E11DDA1
:10DE400007EE90EAF8EEE77A86EEA77AB5EEC07AAA
:10DE5000F1EE10FA45DBF1EEC77AF4EE677AF1EEF7
:10DE600010FA3ED6B4EEE76A01320CF1180CF1EE6E
:10DE700010FA26D4022AD9DDB4EEE76AF1EE10FAE0
:10DE80001FD407EE903AD0ED066A90ED0C7A02238B
:10DE9000F8EE677AD0ED125A037086EEA76AC7EEE5
:10DEA000276A85EEA77A80ED066AC0ED0C6A80EDE0
:10DEB000127A10BDF0EE477A83ED087AF0EE646ACC
:10DEC0009EE7037B13B10323037010BD002221687A
:10DED0000361C36241608261026343648264C3651B
:10DEE00010BDDFED017ABDE7000000004C3A0024D0
:10DEF000B0EEC06AF0EEE05AF0EE407AF4EEC65AA8
:10DF0000F1EE10FA0EDCB5EE400AF1EE10FA4AD04E
:10DF1000F4EEC65AF0EE466AF1EE10FA4FD5B0EEC6
:10DF2000655A03E0F0EE656AB0EE465A85EE267A51
:10DF30009FED242A9FED243A9FED244ADFED244AE9
:10DF4000DFED242ADFED243AB7EE005ADFED236A35
:10DF5000F4EEC65AF1EE10FAA7EE023AE7EE223AD4
:10DF6000A7EE034AA7EE235AE7EE044AE7EE246A37
:10DF7000B1EE667A87EE050A10D4F5EEC00AF1EE2E
:10DF800010FA03D59FED167A37EE400AF5EEC07A07
:10DF9000F1EE10FA48BFB1EE400A70479FED117ADA
:10DFA00037EE400AE9E7F5EEC00ADFED0F7A9FEDA4
:10DFB0000F0AF1EE10FA58BFB0EE670A7047B0EEE4
:10DFC000465AB3E739094E3DE3B59EBE88FA16BE00
:10DFD00045FE7FBF99FB243F69A2163EA7DFA8B488
:10DFE000DB0F4940DB0FC93FA7DFA834DA0F4940F8
:10DFF000D1ED007AF7EE002AD0ED043A90ED054A13
:10E00000E7EEA73AD0ED064A90ED075AD0ED085A50
:10E0100090ED096AD0ED0A6A90ED0B7AC0ED043AF2
:10E0200091ED003AD1ED013AD0ED0C7AA3EE234AFE
:10E0300080ED054AD1ED003A91ED024AE3EE844AC3
:10E04000C0ED064AD1ED004A35EE245A80ED075A5C
:10E05000D1ED014A91ED005AE4EE855AC0ED085A1F
:10E06000D1ED015AA5EEA56A80ED096AD1ED015AFC
:10E0700091ED026AE5EE866AC0ED0A6AD1ED016AA9
:10E0800037EE267A80ED0B7AD1ED026A91ED007AB7
:10E09000E6EE877AC0ED0C7A91ED027AD1ED017A45
:10E0A00090ED0D3AD0ED0E3AA7EE273A90ED0F4ADB
:10E0B000D0ED104A90ED115AD0ED127AD0ED135AEE
:10E0C00090ED006A80ED0D3A75EEA25A91ED023A9C
:10E0D000D0ED016AE3EE033A90ED027AC0ED0E3A1C
:10E0E000D1ED023A34EE234A80ED0F4A91ED004A19
:10E0F00074EE844AC0ED104AD1ED014A35EE245A3F
:10E1000080ED115A91ED025AC0ED135A77EE857ADF
:10E11000C0ED127AD1ED017AD1ED005A67EEA77AFF
:10E1200091ED025AE5EEA57AE5EE057AA5EEA76A2D
:10E1300080ED006A91ED016AE6EE276AC0ED016AA2
:10E14000D1ED026AA6EEA77A80ED027A90ED037A0D
:10E1500077EE277AC0ED037A704700BF2DE9F04FC4
:10E160004FF00009864600F110050646034689B0C7
:10E1700000F13008074648462C468B469C46B2467E
:10E18000CDF80CE000283CD10CF1040CA445FBD1E7
:10E19000032800F1010151D09C46AA46029398B190
:10E1A000DCED047AAAEB0903B64601927246F3EC61
:10E1B000016A0EF1100E92ED007A5345E6EEC77A31
:10E1C000CCED047AF2D1019ADCED046A0CF1100C6A
:10E1D00015ED047A0AF1100AC445C6EE877ACCED33
:10E1E000007ADCD1029B0436084608F10408143397
:10E1F00014351034103709F104099C46B246002842
:10E20000C2D0DCED007AD646394601927246F1EC76
:10E21000016A0EF1100E92ED007A9942E6EEC77A8D
:10E22000CCED007AF2D10CF1040C019A0AF1040A47
:10E23000A445E6D1032800F10101ADD1DDF80CE0E1
:10E240000023594604AD7646774600200493059393
:10E2500006930793F2EC017AE5EC017AB0B104ACD5
:10E260003B46B4EC017AF3EC016AE6EEC77AB342BE
:10E2700045ED017AF5D1013004280BD0F2EC017A9A
:10E2800010371436E5EC017A0028E8D1103714363F
:10E290000120DFE708AD10310EF1400E042875EDC6
:10E2A000017AA1F10402744641ED017A1ED0734651
:10E2B000F3EC016AB1EC017AA342E6EEC77AC2ED53
:10E2C000007AF5D15EED016A013887EEA67A82ED1B
:10E2D000007A17D0AEF1140E103C114675ED017A9C
:10E2E0000428A1F1040241ED017AE0D15EED016A5A
:10E2F000103CAEF1140E032087EEA67A01ED017AF0
:10E300001146EBE709B0BDE8F08F00BF60EEA00A50
:10E31000E0EE000AF5EEC00AF1EE10FA07DBB1EE0E
:10E32000E00AB4EE400AF1EE10FA00D670479FED15
:10E33000010AFBE70000000060EEA00AE0EE000A20
:10E34000E1EE010AF5EEC00AF1EE10FA07DBB1EEDC
:10E35000E00AB4EE400AF1EE10FA00D670479FEDE5
:10E36000010AFBE700000000DFED297AB4EEE70ABE
:10E37000F1EE10FA28DD9FED277A30EE470AB4EE71
:10E38000E70AF1EE10FAF8DCDFED237AB4EEE70AE3
:10E39000F1EE10FA2FDD30EE670A37EEC00A60EEBC
:10E3A000007ADFED1E5A9FED1E6ADFED1E6AA7EEB2
:10E3B000A56A9FED1D7A60EE275AE7EE866AA7EE02
:10E3C000A67AA5EE870A7047DFED187AB4EEE70A61
:10E3D000F1EE10FAD8D59FED0F7A30EE070AB4EEC1
:10E3E000E70AF1EE10FAF8D4DFED0B7AB4EEE70AA3
:10E3F000F1EE10FACFDC9FED0E7AB4EEC70AF1EE23
:10E4000010FACCD530EE270A37EE400AC7E700BF36
:10E41000DB0F4940DB0FC940DB0FC93F9A7C2E362A
:10E42000FAAF4FB93587083CA4AA2ABEDB0F49C012
:10E43000DB0FC9BF10B5404CB4FBF2F4A14219D3B5
:10E44000DFED3E7AF7EE005AB0EE677AB0EE676A1B
:10E45000F0EE676A0023C0ED005AC0ED017A80ED4E
:10E46000027A80ED036AC0ED046A8361436103624E
:10E47000C36110BD07EE902ADFED315AB7EE006A96
:10E48000DFED306AB8EE677A07EE901AB0EE405AC8
:10E49000F8EE677A27EE257A67EEA67AC6EE076A67
:10E4A000C7EEA64AFDEEE47A17EE902A2032402A03
:10E4B0003FD8B0EE640AFFF757FFB0EE404ADFEDF9
:10E4C000227A34EEA70AFDEEC07A17EE902A2032A7
:10E4D000402A29D8FFF748FFF8EE006A60EE266A66
:10E4E000012B1CD0B7EE006AF6EE004A36EE406A09
:10E4F00066EE244A35EE055AF7EE007A84EE057A88
:10E5000077EE275A37EEC75A84EEA57AC6EE257AFB
:10E5100086EEA56AC5EE256AF0EE475A9AE7F7EE51
:10E52000004AB0EE666AE5E7DFED086A9FED030A90
:10E53000D6E79FED024AC2E720A1070000000000D5
:10E54000BD378635DB0FC940DB0FC93F00000080B7
:10E55000DFED077A30EE270AFDEEC07A17EE903A2B
:10E560002033402B00D8FFE69FED020A704700BF22
:10E57000DB0FC93F000000002DE9F84F9DF828404F
:10E580008946DDF82CB00546002C17461BF8011B08
:10E590000CBF4FF020084FF030081C1E08463ADB35
:10E5A00000295CD0002C53D04FF0000A5B4600E0FD
:10E5B00064B313F8016B013C002EF9D1BAF1000FDE
:10E5C0002FD1264644B14D454146284600D2B84792
:10E5D000013CF8D10B9B18780146A0B14FF0FF34F5
:10E5E0004FF0000A00E09B464D45284600D2B84750
:10E5F0005B4613F8011B0029F5D10B9BF61A5E440C
:10E60000BAF1000F10D13046BDE8F88FBAF1000F13
:10E610001BD15646E0E7634229B31C464FF0010A7E
:10E62000C4E70028E0D10646002C04F1FF3AEADDF9
:10E6300054464D454146284600D2B847013CF8D2E1
:10E64000013656443046BDE8F88F30B12646CBE758
:10E6500026464FF0FF34B246C6E70646D3E72646C5
:10E66000002CB0D1CFE76FEA040A0E46E0E700BF06
:10E670000FB430B583B00B4C06AB53F8042BD4E980
:10E68000550101936DF062FC0546206803685B69E3
:10E6900098470028F9D0284603B0BDE8304004B0C0
:10E6A000704700BF206500240EB410B583B0044647
:10E6B000084905AB01A853F8042BCDE900346DF0EF
:10E6C00045FC0022019B1A7003B0BDE8104003B066
:10E6D000704700BF25C004080CB4F0B53D4CADF543
:10E6E000277DD4F85C31002B6FD094F864319942C7
:10E6F0000BD90123D4F868218340134205D10DF5CD
:10E70000277DBDE8F04002B07047334B4FF47A717B
:10E71000324A1B68A2FB030206A8920901FB1233CE
:10E720002F49FFF7C1FF06ABAC9A064603442D49BB
:10E7300001A80193ADAB00936DF008FC019B0A2189
:10E7400000225D1C01951970019BD4F85C51591C85
:10E7500001911A70BDB12B685B6A2BB128469847AE
:10E760000028CCD0D4F85C519DF818100029C6D0F0
:10E770000DF119042B6828461B68984714F8011BF3
:10E780000029F7D1BBE7D4F86071002FB7D030442F
:10E7900026ABFD2206A9841C1846ADF8102022469F
:10E7A000CDF81250ADF8165078F046FF022203461D
:10E7B000044402A93846CDE9023432F0A3FA0DF53B
:10E7C000277DBDE8F04002B07047D4F86031002BDF
:10E7D0008BD194E7206500244C3A0024D34D62107D
:10E7E000A0290D0819C0040838B5184C0330D4F816
:10E7F0006C2102EB9003B3F5007F18D804EB810184
:10E8000004F5B87520F00300C4F86C3105EB8205FF
:10E81000D1F87029C3F5007310440D4A9B00C1F86C
:10E82000700904210020FFF757FF284638BD00215A
:10E83000084A00250846FFF74FFFD4F8F839284664
:10E8400043F00073C4F8F83938BD00BF20650024D8
:10E85000AC290D08D0290D0838B505680446EB69C8
:10E86000F3B1987800B938BDB3F90A20012007EE5A
:10E87000902AF8EEE77AC4ED057AB3F90C2007EE9A
:10E88000902AF8EEE77AF1EE677AC4ED047AB3F9EC
:10E890000E3007EE903AF8EEE77AC4ED067A38BD0E
:10E8A00009211420FFF7A0FF0346E861D9E700BF64
:10E8B00038B505680446EB69E3B1987800B938BD0E
:10E8C000B3F90420012007EE902AF8EEE77AC4EDB0
:10E8D000047AB3F9062007EE902AF8EEE77AC4ED41
:10E8E000057AB3F9083007EE903AF8EEE77AC4ED0E
:10E8F000067A38BD09211420FFF776FF0346E86148
:10E90000DBE700BF38B505680446EB69E3B19878EA
:10E9100000B938BD9A880120D2BA07EE902AF8EEE5
:10E92000E77AC4ED047ADA88D2BA07EE902AF8EED4
:10E93000E77AC4ED057A1B89DBBA07EE903AF8EE68
:10E94000E77AC4ED067A38BD09211420FFF74CFFA1
:10E950000346E861DBE700BF38B505680C46EB69A4
:10E960007BB1987800B938BD5B890120084ADBBAD1
:10E9700082FB0312DB17C3EB221303F26D13238018
:10E9800038BD09211420FFF72FFF0346E861E8E7AF
:10E99000797878782DE9F04103EB4306964686B006
:10E9A000034602EB4606754612F9067BA3EB070CFD
:10E9B00092F80080BCF1000FA3EB0804B8BFCCF1C3
:10E9C000000C002CB8BF6442644502DA15464FFAC9
:10E9D00088F70632B242E9D1688803E00EF1060EEC
:10E9E000764518D09EF800208446BA42F6D10A1A1D
:10E9F000BEF80280002AA1EB0804B8BF5242002CE6
:10EA0000B8BF64429442E9DA75460EF1060E4046FC
:10EA1000C4467645E6D16879CDF808C02A780490D6
:10EA2000287901920390012000910321034AFFF706
:10EA300053FE284606B0BDE8F08100BFE0290D086E
:10EA400003685A1C02601878704700BF03681A46B2
:10EA5000591C016012F8021B0260587841EA00203C
:10EA6000704700BF02681346511C016013F802CBC7
:10EA70000360D31C5178036093781B0443EA01239D
:10EA8000111D43EA0C030160D07843EA006070472F
:10EA900012B370B50446864604E0981B17D114EBF8
:10EAA0000C0C15D01EF8013BA3F14100A2EB0E0C9B
:10EAB000192811F8010BA0F1410598BF203300F18E
:10EAC0002006192DE9D91B1A04D10028E7D170BD01
:10EAD000604670BD184670BD10467047038800211F
:10EAE0001A4A30B503F0030E90F802C0184CA3F593
:10EAF000FA630EEB4E0E0CF1FF3C40F2B5550CEBF9
:10EB00008E0C04EB4C044FEA930CB4F8203184795A
:10EB100005FB0C3390F803C022444FF47A740CF1D7
:10EB2000FF3C634490F804C003EB43030CEBC30CBD
:10EB300043790089CCEB0C1C03EB8C03C3EB031370
:10EB400002EB8302C2FB040130BD00BF80436D387D
:10EB50006C7F0C08F8B516461F46404D04463946F2
:10EB600030464FF47A72002374F098F93C4B054418
:10EB70003C4F3D4E83FB0510E9172844C1EB601163
:10EB800083FB0103C8170B44C0EB631087FB003CF9
:10EB9000C317C3EBAC0386FB03764FEAE37ECEEBF1
:10EBA000E61EC1EB0116A5EB860CC0EB00154FEA83
:10EBB0008E0684F806C0A1EB8501617103EB430169
:10EBC000A0EBC10040F2B55101FB1E332071B3F53B
:10EBD000896F37DA40F2DA218B4239DCB3F5B77F3F
:10EBE0002249B4BF4FF0000E4FF0010E0EEB4E0065
:10EBF00075464FEA4E0701EBC001B1F836011C49DA
:10EC000007EB0E0C01EBCC0C0B210CF1160C01E008
:10EC10003CF8020D984212DD0139F9D177441349CD
:10EC200001EBC701B1F82001012106F5FA6E0133AD
:10EC3000A17075441B1A22812580E370F8BD013153
:10EC4000C9B2F2E7032540F296500627AE46D6E752
:10EC5000022540F229400427AE46D0E780BC92C787
:10EC600089888888ABAAAA2A73B06D166C7F0C08B5
:10EC70008C800C0830B5304C8DB086460D46EC4685
:10EC80001EF0030F0FCCACE80F000FCCACE80F0068
:10EC900094E80F008CE80F000FD1284B284A03FBA3
:10ECA0000EF3B2EBB30F44D3264AB2EB331F34BF9B
:10ECB00001220022C2F11D0200E01C220EF1FF33EE
:10ECC000019240F26D122048002B194602FB0EF211
:10ECD0001E4CB8BF0EF10201EE4602EBA10280FB12
:10ECE0000310DB17ADF1040101EB8501A3EB601507
:10ECF000C3EBE0132A441A44253284FB0230D317B5
:10ED00001044C3EBA003C3EBC303D31A5EF8040F94
:10ED1000C218714584FB023C4FEAE2739444C3EB92
:10ED2000AC03C3EBC303A2EB0303EFD1C01A0DB0D6
:10ED300030BD1D22C2E700BFEC800C08295C8FC2E9
:10ED4000285C8F020AD7A3001F85EB5193244992B8
:10ED50000E4B10B5D3F8004AD3F8043A54EA030234
:10ED60000AD10146002340F2011218460B80C1F877
:10ED700002208B710B8110BD054A1268121943F1F4
:10ED80000003FFF7E7FE012010BD00BF206500244F
:10ED90004C3A002430B5144D83B00446D5F8001A1F
:10EDA000D5F8043A51EA03020AD1002340F20112D5
:10EDB00018462380C4F80220A371238103B030BD1C
:10EDC0000A4A1268521843F10003FFF7C3FEB5F870
:10EDD000083A20460DF106022146ADF806306AF0E9
:10EDE0003FF9012003B030BD206500244C3A0024D7
:10EDF00088422DE9F04198464FF0010439D301FBD8
:10EE000004F4B0FBF4FC8C45F9D264B30025BCF1EA
:10EE1000000F04FB1C00B4FBF1F7D4BF0026012651
:10EE20006DB966B9A142354619D9C6460CF1300C08
:10EE30000EF801CB00238EF80030BDE8F081BCF164
:10EE4000090F18DD002A0CBF57233723C646634439
:10EE5000A14205F101050EF8013BF046EAD83C4617
:10EE6000B0FBF7FCD3E7C64600238EF80030BDE8C0
:10EE7000F0818446CAE73023E8E700BF2DE9F0417E
:10EE80000446154608469442B4FBF2F607D205FB49
:10EE90001644134B1B5D00F8013BBDE8F081964220
:10EEA000B6FBF2F70CD20E4B05FB176705FB1644B9
:10EEB000DA5D1B5D00F8012B00F8013BBDE8F08135
:10EEC000BA42B7FBF2F807D905FB1878044B13F8E0
:10EED000082000F8012BE7E74046FFF7CFFFF3E7F4
:10EEE0001C2A0D08B5EEC00ADFED357A0023F1EEDD
:10EEF00010FA30B5C8BF30EE270A87B0D8BF30EE61
:10EF0000670ADFED307A054603A9029320EE270A4F
:10EF1000CDE90033FDEEC07A17EE904A84EAE47042
:10EF2000A0EBE4706BF0C2F9002C03A8B4BF2D2352
:10EF300020238DF8003073F0F5F901282AD002283B
:10EF400034D003281ED003A9684678F09BFC68469D
:10EF500073F0E8F9044669462846033CE4B22246C9
:10EF600078F06AFB002328462B5573F0DBF92E223C
:10EF7000431C0DEB04012A54E81878F01DFD2846C7
:10EF800007B030BD302303A968468DF8013078F012
:10EF900079FCDCE743F23002302303A96846ADF880
:10EFA00001208DF8033078F06DFCD0E743F2300398
:10EFB00003A96846ADF8013078F064FCC7E700BFEC
:10EFC0006F12033A00007A440378202B03D110F823
:10EFD000013F202BFBD0092BF9D02D2B63D02B2BFD
:10EFE000B7EE000A08BF01300278A2F13003D9B2AF
:10EFF000092961D8F2EE046ADFED4D7A07EE103A86
:10F0000010F8012FB8EEC77AA2F13003D9B2A7EEFB
:10F01000A67A0929F0EE477AF0D92E2A50D0037843
:10F0200003F0DF03452B3BD110B442782D2A73D077
:10F030002B2A62D0A2F130030130092B63D80024BF
:10F04000002303EB830302EB430310F8012FA2F12B
:10F050003001303B0929F4D9B3F59A7F1A46B7EE4F
:10F06000007A28BF4FF49A72072B09D91346DFEDB7
:10F07000316A083B27EE267A072BFAD802F00702FE
:10F080002AB1F2EE046A013A27EE267AFBD1002C6F
:10F090003BD0C7EE877A5DF8044B20EE270A704715
:10F0A00020EE270A704742780130BFEE000AA2F135
:10F0B0003003D9B209299DD92E2ADFED1D7AAED1B0
:10F0C00043780130A3F13002D1B20929A8D8B2EEB9
:10F0D000047AF0EE475A06EE902A10F8013FB8EE97
:10F0E000E66AA3F13002D1B2C6EE076A092927EE1B
:10F0F000257A77EEA67AEED992E782780230A2F1ED
:10F100003003092B9BD9B7EE007A67EE877A5DF85A
:10F11000044B20EE270A704782780230A2F13003B8
:10F12000092B01D801248BE7B7EE007AB1E700BFC5
:10F130000000000020BCBE4C0378092B01D0202B1E
:10F1400005D110F8013F202BFBD0092BF9D02D2B36
:10F1500009D001784FF0010CA1F13002D3B2092B94
:10F160000AD900207047417801304FF0FF3CA1F1EF
:10F170003002D3B2092BF4D8002310F8011F03EB9F
:10F18000830302EB4303A1F13002D1B20929F4D980
:10F190000CFB03F0704700BFB14BB24A2DE9F04FB2
:10F1A00093F80C3A97B002EB430393F8B13113B1E3
:10F1B000012005F019FDAC4B4FF0000AAB4A41F2BB
:10F1C00021051F469E1A2C2200210DEB020078F02B
:10F1D00051FBA64AA64B0892CDE90976DA68D10719
:10F1E00007D5A44A5A6002F188325A60DB68DC070E
:10F1F0000DD49F4BD3F80C21D20708D59D4AC3F8F4
:10F20000042102F18832C3F80421D3F80C31002321
:10F21000012205A908A814937E238DF854208DF8A7
:10F220001430FDF7C7FB0028C0F22D8108214FF4F0
:10F23000FC4303E05B0001399BB207D01AB2002AFD
:10F24000F8DA85EA4202013993B2F7D18A4AADF879
:10F2500016308A4B934280F0628198460DF118096E
:10F26000CDE902A7B8F802204FF0000CB8F8003042
:10F27000C2F30B0B1004C3F30B014FEA13338DF8E9
:10F280001DC08DF81C300BF10603ADF81A10ADF857
:10F29000183000F191800622494608A8FDF78AFB44
:10F2A0000028C0F20E81BDF8164049460DF11E003F
:10F2B00011F8013B082284EA032403E06400013AC8
:10F2C000A4B207D023B2002BF8DA85EA4303013A4F
:10F2D0009CB2F7D18842EBD15A46D8F8041008A85E
:10F2E000FDF768FB0028C0F2EC80D8F8041001EBB1
:10F2F0000B00814215D00139013811F8013F082275
:10F3000084EA032403E06400013AA4B207D023B2E4
:10F31000002BF8DA85EA4303013A9CB2F7D1814227
:10F32000EBD1ADF8164008F11408534B984599D32A
:10F33000DDE902A700230222494608A8ADF81830EB
:10F34000FDF738FB0028C0F29E80BDF816300DF1A5
:10F350001A0041F2210119F8012B082483EA022343
:10F3600003E05B00013C9BB207D01AB2002AF8DA36
:10F3700081EA4202013C93B2F7D14845EBD1022227
:10F380000DF1160108A8ADF81630FDF713FB0028A3
:10F3900079DB1398002840F09A801498002872DBDB
:10F3A0009DF85420002A40F0A88000280DBF0124B9
:10F3B00000240123002368E0E246674601960137F6
:10F3C0000622494608A8FFB28DF81D70FDF7F2FA33
:10F3D000002855DBBDF8164049460DF11E0011F816
:10F3E000013B082284EA032403E06400013AA4B24A
:10F3F00007D023B2002BF8DA85EA4303013A9CB226
:10F40000F7D18842EBD1D8F804105A4608A801EB8E
:10F410000A063146FDF7CEFA002831DB06EB0B0079
:10F42000864215D0711E013811F8013F082284EA86
:10F43000032403E06400013AA4B207D023B2002BF6
:10F44000F8DA85EA4303013A9CB2F7D18142EBD165
:10F45000032FDA44ADF81640B1D1019E63E700BF37
:10F46000206500246C7F0C080000040800000208DE
:10F47000002000522301674598E50D08E4DF0D08E0
:10F48000DDE9016A039F012300240AF1010ABAF1B0
:10F49000020F02DC002B7FF496AE224B224A93F837
:10F4A0000C3A02EB430393F8B13133B914B1FCF7D2
:10F4B000C7FD48B9052007F0F3F8002005F094FBDC
:10F4C000F4E7DDE902A7DEE717B0BDE8F08F089B9F
:10F4D000099A03449342D6D80BABC0F120022146CF
:10F4E000184478F0C7F9149818B90BA908A8F4F7CC
:10F4F00037F900221490139250E70C4AD16841F07A
:10F500000101D160D168C9077FF54FAFD2F80C1166
:10F5100041F00101C2F80C11D2F80C2145E70DF1C0
:10F52000180907E7206500246C7F0C0800200052B2
:10F5300070B545880B4604460021C5F30B051846F7
:10F540002A4678F097F90A4A21690346914206D380
:10F55000084A914206D31846BDE870400847002982
:10F56000F9D170BD2A46BDE8704078F065B800BF9B
:10F5700098E50D08CBEA0D0810B50446C06900B146
:10F5800010BD09211420FFF72FF9E06110BD00BF65
:10F59000174B03EB8000806838B300EB400003EBAF
:10F5A000800292F9DDC0BCF1FF3F1FD092F8E50068
:10F5B000D8B103EB0C00002310B590F830E18C209B
:10F5C00092F8E410142200FB0CFC0A4C0CEB010036
:10F5D000013A714434F8100013FA80F3F6D1064A68
:10F5E000A2FB0320C0F30F1010BD7047002070472E
:10F5F0002065002400000030CDCCCCCC30B50023F9
:10F60000B0F80EE001250EF47F4419460EF00F0EFF
:10F61000C4814A1030F81220002A18BF002511F0CA
:10F62000010F1AD0D2B25340082213F4004F18BF72
:10F6300083F4C053013A4FEA4303F6D10131102954
:10F64000E7D14EEA0404C48155B9C3F30333B3EBE5
:10F650000E0018BF4FF0FF3030BD83EA1223E3E7FE
:10F660004FF0FF3030BD00BF036810B51A79044673
:10F67000022A03D000232360237110BD987A04F07E
:10F6800067FB0028F6D040F61A610022C1802021D5
:10F69000027204F019FB00232360237110BD00BF28
:10F6A0002DE9F04FBA4E85B0BA4CA64256D21D464F
:10F6B00002E00C36A64251D273798B42F9D13379EC
:10F6C000834201D00028F4D1F3799342F1D1346818
:10F6D000002C43D0002326606360A360E3602361B5
:10F6E0006361A361E36133792371012B96F806B05E
:10F6F000C4F808B0317AE16032D0022B2ED1F07A12
:10F7000004F026FB96F90970A061B07A277404F022
:10F710001FFB06466061F0B1DFF8948207EB4701FA
:10F720007B0058F8319008EBC1010193B9F1000F4B
:10F7300011D0887DE8B10E2200230D213046F271F0
:10F740003372B57104F0C0FA3368B2889A6120460A
:10F7500005B0BDE8F08F2046FFF786FF0024F6E7EE
:10F76000F07A04F0F5FA727AB37AA06122746374C5
:10F77000EDE7B1F808A0504669F06CFD01214FEAB1
:10F780005A100AF01F0A023801FA0AF1092812D8A1
:10F79000DFE810F0F6001100EE0018011001E6009D
:10F7A000E000D800D0000A007B4BD3F89C0020EA90
:10F7B0000101C3F89C107B00D91908EBC1014879FD
:10F7C00004F0C6FA791CCBB20146019318B103725A
:10F7D00040F60A30C8807B000291D81908EBC000BF
:10F7E000C07904F0B5FA02990346039020B1019A5A
:10F7F000027240F60A50D8807B000291D81908EBBB
:10F80000C000807904F0A4FA0299824628B1019BD5
:10F81000037240F60A40AAF806007B00D8191BF0D4
:10F82000040308EBC0000293807A0246084614BF26
:10F830004E212E2104F06AFA03987B002E2103EB5F
:10F84000070B08EBCB0B9BF80B2004F05FFA50463C
:10F850009BF80C200E2104F059FA9BF804A0BAF191
:10F86000000F40F0ED80D9F8002022F00102C9F825
:10F8700000204A4A914500F0C180494A914540F034
:10F88000AC80454AD2F8901041F48041C2F8901003
:10F89000D2F8901021F48041C2F89010029B002B06
:10F8A00040F098804FF000714FF08072D9F80C0052
:10F8B00040F00040C9F80C00D9F8080020F4F070BE
:10F8C000C9F80800D9F80000C00727D4D9F8080003
:10F8D000344B034034481843C9F80800D9F80C00E9
:10F8E000C30005D4D9F8000040F48050C9F80000E6
:10F8F000D9F80C0011432D4A02400A4342F08862B5
:10F90000C9F80C20D9F8002022F40062C9F80020C0
:10F91000D9F8502022F00102C9F85020BAF1000FA6
:10F9200040F09B807B003B4408EBC308012388F830
:10F93000163000E7184BD3F8880020EA0101C3F81D
:10F94000881038E7144BD3F88C0020EA0101C3F883
:10F950008C1030E7104BD86F20EA0101D9672AE7F5
:10F960000D4BD3F8940020EA0101C3F8941022E76C
:10F97000094BD3F8800020EA0101C3F880101AE790
:10F98000054BD3F8980020EA0101C3F8981012E75C
:10F99000A00200089804000800440258003001400A
:10F9A00000380040E0FFBF8F07000020FFFF39D87C
:10F9B0002C0200243E4BD3F8900020EA0101C3F84A
:10F9C0009010F8E63A4BD3F8840020EA0101C3F81E
:10F9D0008410F0E600210A4668E7364A91451BD1BB
:10F9E000334AD2F8901041F40041C2F89010D2F896
:10F9F000901021F40041C2F890104FE72C4AD2F841
:10FA0000981041F48051C2F89810D2F8981021F45F
:10FA10008051C2F8981041E7274A914527D0274ADC
:10FA2000914532D1224AD2F8981041F48011C2F89F
:10FA30009810D2F8981021F48011C2F898102DE790
:10FA4000504604F085F920B1019B40F60A6203722A
:10FA5000C2800D2104F038F905E7504604F078F92A
:10FA600000283FF45FAF0268838893615AE7104A29
:10FA7000D2F8981041F40051C2F89810D2F89810BA
:10FA800021F40051C2F8981008E70D4A91457FF41F
:10FA900005AF02F50C32D2F89C1041F02001C2F8FB
:10FAA0009C10D2F89C1021F02001C2F89C10F5E6C1
:10FAB00000440258003C0040003401400050014026
:10FAC00000140058104B70B5104CA34219D20546D3
:10FAD00002E00C33A34214D293F805C08C45F8D150
:10FAE00093F804C00DB1AC45F3D1D8799042F0D170
:10FAF000186890F804E0E645EBD106689E42E8D12C
:10FB000070BD002070BD00BFA0020008980400086E
:10FB10000379022B00D0704790F9102008311C485F
:10FB200002EB420210B41B4C83B050F83220009418
:10FB30006944194C11F808CCA24224D017498A42D2
:10FB400023D001F580618A4205D0154B9A420CBF43
:10FB500003234FF0FF33116803EB430321F001014E
:10FB600000EBC30011600169936851F82C1023F079
:10FB7000E0430B439360136843F00103136003B049
:10FB80005DF8044B70470023E5E70123E3E700BF7E
:10FB90002C02002400010203003001400038004024
:10FBA0000034014090F91030F0B503EB4303294EC7
:10FBB000154683B056F83360044683689A0719D512
:10FBC00001230DF106028DF8061030460DF10701F4
:10FBD000F4F7D2FD01230DF106020DF107013046C5
:10FBE0008DF80650F4F7C8FDA3689B0717D50120D0
:10FBF00003B0F0BD43691BB19A8818681204826192
:10FC0000154B164AD3F8100A154BC0005768A3FBD2
:10FC1000003080095368DB1B9842FBD2D0E70E4AC4
:10FC20004FF4FA700E4BD2F8102A0C4900FB02F286
:10FC30004868A3FB023292094B681B1A9A42FBD216
:10FC40006369002BD3D01A6801209B88936103B0AD
:10FC5000F0BD00BF2C02002420650024001000E04D
:10FC6000D34D621010B5037984B084468E46012BC3
:10FC70000DD0022B02D0002004B010BD8368DB073A
:10FC800058BF01F07F0104B0BDE810408AE78168E9
:10FC90000DF10F001446724601F001018DF80F407E
:10FCA000CDE900019CF811109CF91000F4F768F8F8
:10FCB00004B010BD2DE9F0410768642682B0B62279
:10FCC0007E2180463846FFF7CDFF06F00BF804464C
:10FCD0000D4606F007F8001B61EB0501B0F57A7FD1
:10FCE00071F10001F5D3013EEFD102213846FFF753
:10FCF0000FFF7B691BB19A88196812048A6105F0AD
:10FD0000F1FF04460D4605F0EDFF001B61EB050118
:10FD1000B0F57A7F71F10001F5D37B6913B11A68F0
:10FD20009B8893610A2605F0DDFF04460D4605F029
:10FD3000D9FF001B61EB0501B0F57A7F71F100017D
:10FD4000F5D3013EEFD132467C213846FFF78AFFDA
:10FD500005F0C8FF04460D4605F0C4FF001B61EB2B
:10FD60000501B0F57A7F71F10001F5D30022592128
:10FD70003846FFF777FF05F0B5FF04460D4605F05E
:10FD8000B1FF001B61EB0501B0F57A7F71F1000155
:10FD9000F5D397F910305E218E4A03EB43038DF8BB
:10FDA000071052F83340BB689A0740F1E480012302
:10FDB0000DF1070200212046F4F7DEFC4FF4A47396
:10FDC000854A20460021F4F7D7FCBB689B0740F129
:10FDD000E7800A2605F086FF04460D4605F082FFFF
:10FDE000001B61EB0501B0F57A7F71F10001F5D3DD
:10FDF000013EEFD1012259213846FFF733FF05F0CC
:10FE000071FF04460D4605F06DFF001B61EB050117
:10FE1000B0F57A7F71F10001F5D38C22402138468C
:10FE2000FFF720FF05F05EFF04460D4605F05AFF80
:10FE3000001B61EB0501B0F57A7F71F10001F5D38C
:10FE4000032241213846FFF70DFF05F04BFF044622
:10FE50000D4605F047FF001B61EB0501B0F57A7F09
:10FE600071F10001F5D35D4C0323D8F8382098F8E0
:10FE70003500B4FBF2F291B2594AFEF78BFD43888C
:10FE80004221B4FBF3F4C8F840400279384642F00E
:10FE9000C002FFF7E7FE05F025FF04460D4605F01A
:10FEA00021FF001B61EB0501B0F57A7F71F10001C4
:10FEB000F5D3082243213846FFF7D4FE05F012FFA0
:10FEC00004460D4605F00EFF001B61EB0501B0F581
:10FED0007A7F71F10001F5D3042258213846FFF7EB
:10FEE000C1FE05F0FFFE04460D4605F0FBFE001BBB
:10FEF00061EB0501B0F57A7F71F10001F5D30A22BB
:10FF000053213846FFF7AEFE05F0ECFE04460D46E1
:10FF100005F0E8FE001B61EB0501B0F57A7F71F199
:10FF20000001F5D300227C213846FFF79BFE05F047
:10FF3000D9FE04460D4605F0D5FE001B61EB050118
:10FF4000B0F57A7F71F10001F5D306227D213846A4
:10FF5000FFF788FE05F0C6FE04460D4605F0C2FE1A
:10FF6000001B61EB0501B0F57A7F71F10001F5D35B
:10FF700002B0BDE8F0817B691BB11A689B881B0445
:10FF80009361184B1849D3F8102A184BD2004868CF
:10FF9000A3FB023292094B681B1A9A42FBD206E776
:10FFA000104A4FF4FA70114BD2F8102A0E4900FB98
:10FFB00002F24868A3FB023292094B681B1A9A426C
:10FFC000FBD27B69002B3FF404AF1A689B889361D6
:10FFD000FFE600BF2C0200242C810C0840420F00D9
:10FFE00074820C0820650024001000E0D34D6210DC
:10FFF0002DE9F041816B0623654D044607686426B0
:020000040805ED
:10000000644A90F83500B5FBF1F189B2FEF7C2FC05
:100010004388002180463846B5FBF3F52564FFF799
:1000200077FD80226B213846FFF71CFE05F05AFE53
:1000300004460D4605F056FE001B61EB0501B0F5C8
:100040007A7F71F10001F5D3013EEFD164260722DA
:1000500068213846FFF706FE05F044FE04460D46CB
:1000600005F040FE001B61EB0501B0F57A7F71F1F0
:100070000001F5D3013EEFD1324664266B213846AC
:10008000FFF7F0FD05F02EFE04460D4605F02AFEB2
:10009000001B61EB0501B0F57A7F71F10001F5D32A
:1000A000013EEFD10F2601226B213846FFF7DAFD22
:1000B00005F018FE04460D4605F014FE001B61EB2A
:1000C0000501B0F57A7F71F10001F5D3013EEFD162
:1000D0000F2618221B213846FFF7C4FD05F002FE4B
:1000E00004460D4605F0FEFD001B61EB0501B0F571
:1000F0007A7F71F10001F5D3013EEFD10F2618226E
:100100001C213846FFF7AEFD05F0ECFD04460D4618
:1001100005F0E8FD001B61EB0501B0F57A7F71F198
:100120000001F5D3013EEFD10F2698F804201A21E3
:100130003846FFF797FD05F0D5FD04460D4605F05E
:10014000D1FD001B61EB0501B0F57A7F71F1000173
:10015000F5D3013EEFD1642698F8052019213846E1
:10016000FFF780FD05F0BEFD04460D4605F0BAFD23
:10017000001B61EB0501B0F57A7F71F10001F5D349
:10018000013EEFD138460321BDE8F041C0E400BF95
:1001900040420F0088820C082AE700BF00680379FC
:1001A000012B09D0022B01D0002070478368F02278
:1001B000DB0717D5FF21F5E4826890F910C002F043
:1001C0000102417C60464FF0F00C10B584B00DF197
:1001D0000F040192FF228DF80FC00094F3F7D0FDB9
:1001E00004B010BD7F21DDE40068CA43037941EA11
:1001F0000211012BCAB208D0022B01D00020704797
:100200008368DB0715D5D221CCE410B584B08468AF
:1002100090F910C08DF80F200DF10F0204F00104C9
:10022000417C0092D22260460194F3F7A9FD04B00C
:1002300010BD5221B6E400BF00680379012B09D03C
:10024000022B01D0002070478368B422DB0717D54A
:10025000FF21A7E4826890F910C002F00102417CFE
:1002600060464FF0B40C10B584B00DF10F0401924C
:10027000FF228DF80FC00094F3F782FD04B010BD8B
:100280007F218FE400680379012B09D0022B01D074
:100290000020704783680A46DB0715D5A52181E455
:1002A00010B584B0846890F910C00DF10F0204F00D
:1002B00001048DF80F10417C60460092A522019444
:1002C000F3F75EFD04B010BD25216BE400680379EF
:1002D000012B09D0022B01D00020704783689622A1
:1002E000DB0717D5FF215DE4826890F910C002F0AA
:1002F0000102417C60464FF0960C10B584B00DF1C0
:100300000F040192FF228DF80FC00094F3F738FD1F
:1003100004B010BD7F2145E400680379012B09D0AA
:10032000022B01D00020704783680A46DB0715D5F1
:10033000872137E410B584B0846890F910C00DF1BE
:100340000F0204F001048DF80F10417C604600920A
:1003500087220194F3F714FD04B010BD072121E4B6
:100360000068C9010379CAB2012B05D0022B01D064
:1003700000207047782115E410B584B0846890F9A6
:1003800010C08DF80F200DF10F0204F00104417C24
:100390000092782260460194F3F7F2FC04B010BD9D
:1003A00000680379012B0AD0022B01D0002070478E
:1003B00083685522DB0718D5A521FFF7F3BB8268B8
:1003C00090F910C002F00102417C60464FF0550CDC
:1003D00010B584B00DF10F040192A5228DF80FC065
:1003E0000094F3F7CDFC04B010BD2521FFF7DABB74
:1003F00000680379012B0AD0022B01D0002070473E
:1004000083682E22DB0718D5F421FFF7CBBB826867
:1004100090F910C002F00102417C60464FF02E0CB2
:1004200010B584B00DF10F040192F4228DF80FC0C5
:100430000094F3F7A5FC04B010BD7421FFF7B2BB24
:10044000154B00681A8F03799201012B02F13402D7
:10045000D2B209D0022B01D0002070478368DB079D
:1004600016D5F421FFF79EBB10B584B0846890F9CF
:1004700010C08DF80F200DF10F0204F00104417C33
:100480000092F42260460194F3F77AFC04B010BDA8
:100490007421FFF787BB00BF20650024006810B5FA
:1004A000037984B0012B0FD0022B02D0012004B0BD
:1004B00010BD83683122DB074CBFF4217421FFF7A4
:1004C00071FB012004B010BD82680DF10F0490F99A
:1004D00010C002F00102417C60464FF0310C0192E5
:1004E000F42200948DF80FC0F3F74AFC012004B009
:1004F00010BD00BF00680379012B07D0022B01D08B
:100500000020704713221B21FFF74CBB826890F933
:1005100010C002F00102417C60464FF0130C10B590
:1005200084B00DF10F0401921B228DF80FC00094CE
:10053000F3F726FC04B010BD00680379012B07D047
:10054000022B01D00020704701225821FFF72ABB5F
:100550008268417C02F0010210B590F9104084B02D
:1005600020460DF10F040192582200948DF80F30AF
:10057000F3F706FC04B010BD00680379012B07D027
:10058000022B01D00020704701224821FFF70ABB4F
:100590008268417C02F0010210B590F9104084B0ED
:1005A00020460DF10F040192482200948DF80F307F
:1005B000F3F7E6FB04B010BD00680379012B07D008
:1005C000022B01D0002070471A460821FFF7EABA33
:1005D000826890F910C002F00102417C60464FF041
:1005E000020C10B584B00DF10F04019208228DF8B1
:1005F0000FC00094F3F7C4FB04B010BD006803798A
:10060000012B07D0022B01D00020704701220821C6
:10061000FFF7C8BA8268417C02F0010210B590F978
:10062000104084B020460DF10F040192082200947E
:100630008DF80F30F3F7A4FB04B010BD2DE9F041A5
:1006400005461F462948164695F9103082B003EB3F
:10065000430350F83380AB689A0716D501230DF198
:1006600006028DF8061040460DF10701F4F784F8F4
:100670003B46324600214046F4F77EF8AB689B07C4
:1006800019D5012002B0BDE8F0816B691BB19A88D1
:10069000186812048261164BD3F8100A154BC0007B
:1006A000A3FB0030144B80095A685C68A4EB020C71
:1006B0006045FAD2D2E70E4A4FF4FA700D4BD2F8E9
:1006C000102A0D4900FB02F24868A3FB023292098E
:1006D0004B681B1A9A42FBD26B69002BD1D01A6867
:1006E00001209B88936102B0BDE8F0812C020024B8
:1006F00020650024D34D6210001000E030B505796C
:1007000083B084468E46012D0DD0022D02D00020EC
:1007100003B030BD8468E40758BF01F07F0103B027
:10072000BDE830408AE7806814460A46009400F02D
:1007300001049CF811109CF910000194F3F720FBC0
:1007400003B030BD2DE9F04105461F462948164645
:1007500095F9103082B003EB430350F83380AB6857
:100760009A0716D501230DF106028DF806104046B2
:100770000DF10701F4F700F83B46002231464046F0
:10078000F3F7FAFFAB689B0719D5012002B0BDE86B
:10079000F0816B691BB19A88186812048261164B4C
:1007A000D3F8100A154BC000A3FB0030144B80098E
:1007B0005A685C68A4EB020C6045FAD2D2E70E4A94
:1007C0004FF4FA700D4BD2F8102A0D4900FB02F2DB
:1007D0004868A3FB023292094B681B1A9A42FBD26B
:1007E0006B69002BD1D01A6801209B88936102B0FD
:1007F000BDE8F0812C02002420650024D34D621056
:10080000001000E030B5057983B084468E46012D96
:100810000DD0022D02D0002003B030BD8468E40763
:1008200058BF41F0800103B0BDE830408AE78068DE
:1008300014460A46009400F001049CF811109CF93B
:1008400010000194F3F7ACFC03B030BD2DE9F04388
:10085000816B85B0804C0623076880467F4A9626C8
:1008600090F83500B4FBF1F189B2FEF793F84388B4
:10087000002181463846B4FBF3F4C8F84040FFF746
:1008800047F980226B213846FFF7ECF905F02AFA88
:1008900004460D4605F026FA001B61EB0501B0F594
:1008A0007A7F71F10001F5D3013EEFD19626032244
:1008B00068213846FFF7D6F905F014FA04460D46CC
:1008C00005F010FA001B61EB0501B0F57A7F71F1BC
:1008D0000001F5D3013EEFD103226B213846FFF72B
:1008E000C1F905F0FFF904460D4605F0FBF9001BC0
:1008F00061EB05010F2871F10001F6D310226A2186
:100900003846FFF7AFF905F0EDF904460D4605F05E
:10091000E9F9001B61EB05010F2871F10001F6D325
:1009200000226C213846FFF79DF905F0DBF90446FB
:100930000D4605F0D7F9001B61EB05010F2871F199
:100940000001F6D399F8052019213846FFF78AF9F6
:1009500005F0C8F904460D4605F0C4F9001B61EB2B
:1009600005010F2871F10001F6D318221B2138462A
:10097000FFF778F905F0B6F904460D4605F0B2F92F
:10098000001B61EB05010F2871F10001F6D318225D
:100990001C213846FFF766F905F0A4F904460D4618
:1009A00005F0A0F9001B61EB05010F2871F10001B2
:1009B000F6D399F804201A213846FFF753F905F0C9
:1009C00091F905460C4605F08DF98C4208BF854229
:1009D000F9D003213846FFF79BF8062302AA4321EA
:1009E000D8F80000FFF70EFF28B3BDF80810BDF8D7
:1009F0000A30BDF80C20C9BADBBA07EE901AD2BA99
:100A0000F8EEE76A07EE102A07EE903AB8EEC77ADA
:100A1000F8EEE77AC8ED076A88ED097AC8ED087A3A
:100A2000FDEEE77ACDED017A9DF90430013305D072
:100A300005B0BDE8F083D8ED087AF1E7D8ED077A84
:100A4000FDEEE77ACDED017A9DF904300133EFD167
:100A5000062005F025FE00BF40420F0088820C08EA
:100A6000006808B50379022B20D00623124A04211E
:100A7000FFF7C8FE114B012093F8171A93F816CA16
:100A8000090493F81A2A41EA0C2193F815CA1204B2
:100A900041EA0C0193F819CA42EA0C2293F818CAE9
:100AA000C3F8881042EA0C025A6608BD0723044ABC
:100AB0000421FFF7A7FEDDE7356F00242065002441
:100AC000346F002470B5066882B00546F469002CC6
:100AD0003ED03379221D012B2DD0022B26D1B368B5
:100AE000304613F0010F4FF00C030CBF8C21194658
:100AF000FFF728FEA070D8B1B4F9043007EE903AA1
:100B0000F8EEE77AC5ED077AB4F9063007EE903AC9
:100B1000F8EEE77AC5ED087AB4F9083007EE903AB6
:100B2000F8EEE77AC5ED097A02B070BD0023A37034
:100B3000002002B070BDB368717C03F0010396F928
:100B40001000009201930C231A46F3F729FBD1E71A
:100B500009211420FDF748FEF06104462E68B8E72D
:100B600070B5066882B00546F469002C3ED0337932
:100B7000E21C012B2DD0022B26D1B368304613F096
:100B8000010F4FF00D0314BF0C218C21FFF7DAFD8C
:100B9000A070D8B1B4F90A3007EE903AF8EEE77ACF
:100BA000C5ED077AB4F90C3007EE903AF8EEE77A23
:100BB000C5ED087AB4F90E3007EE903AF8EEE77A10
:100BC000C5ED097A02B070BD0023A370002002B009
:100BD00070BDB368717C03F0010396F910000092B8
:100BE0000C2201930D23F3F7DBFAD1E7092114203E
:100BF000FDF7FAFDF06104462E68B8E7006810B50D
:100C0000037984B00C46012B1AD0022B02D00020AD
:100C100004B010BD836803AA13F0010F4FF0030363
:100C200014BF2221A221FFF78DFD0028EFD0BDF9CE
:100C30000D3003EB83031B12E633238004B010BD99
:100C4000836803AA417C03F0010390F9100000922D
:100C5000222201930323F3F7A3FAE6E770B50668AF
:100C600082B00546F469002C3ED03379221D012B59
:100C70002DD0022B26D1B368304613F0010F4FF070
:100C80000E0314BF3B21BB21FFF75CFDA070D8B160
:100C9000A389DBBA07EE903AF8EEE77AC5ED077A5A
:100CA000E389DBBA07EE903AF8EEE77AC5ED087A09
:100CB000238ADBBA07EE903AF8EEE77AC5ED097AB7
:100CC00002B070BD0023A370002002B070BDB368F5
:100CD000717C03F0010396F9100000923B2201930E
:100CE0000E23F3F75DFAD1E709211420FDF77CFD0F
:100CF0000446F061B9E700BF006810B5037984B01D
:100D0000012B10D0022B01D000200AE003AAF6210B
:100D1000FFF718FD0028F7D0BDF80C30094A5BBA80
:100D2000138304B010BD826803AC417C022302F03F
:100D3000010290F91000CDE90042F622F3F730FAF3
:100D4000E8E700BF20650024006810B5037984B08F
:100D5000012B1DD0022B01D0002017E0032303AA92
:100D6000F621FFF7EFFC0028F6D09DF80D309DF836
:100D70000CC01B020D499DF80E2043EA0C4313439F
:100D8000B1F93820C2F10802D340CB6304B010BDE2
:100D9000826803AC417C032302F0010290F9100049
:100DA000CDE90042F622F3F7FBF9DCE720650024E9
:100DB000006810B5037984B0012B31D0022B09D023
:100DC0001E490020D1F81C3AD1F8202A0B660A648B
:100DD00004B010BD062302AAF721FFF7B3FC0028D8
:100DE000EED09DF809309DF80C209DF808C01B013D
:100DF0009DF80BE012019DF80A1043EA0C3342EA19
:100E00000E329DF80DC043EA11130C4942EA1C1240
:100E1000C1F81C3AC1F8202A0A640B6604B010BD60
:100E2000826802AC417C062302F0010290F91000B6
:100E3000CDE90042F722F3F7B3F9D0E720650024AB
:100E4000006810B5037984B0012B1DD0022B0FD0A0
:100E50009DF80D3001209DF80CC01B029DF80E106E
:100E6000104A43EA0C430B43C2F8B03004B010BD43
:100E7000836803AA13F0010F4FF0030314BF00218E
:100E80008021FFF75FFCE3E7826803AC417C03232A
:100E900002F0010290F91000CDE900420022F3F7C0
:100EA0007FF9D5E720650024006810B5037984B088
:100EB000012B1DD0022B0FD09DF80D3001209DF885
:100EC0000CC01B029DF80E10104A43EA0C430B4362
:100ED000C2F8C43004B010BD836803AA13F0010F38
:100EE0004FF0030314BF00218021FFF72BFCE3E741
:100EF000826803AC417C032302F0010290F91000E8
:100F0000CDE900420022F3F74BF9D5E72065002434
:100F1000006810B5037984B0012B28D0022B01D0D2
:100F2000002022E0836803AA13F0010F4FF00303AF
:100F30000CBF83211946FFF705FC0028F0D09DF86F
:100F40000C309DF90C109DF80D201B0400299DF814
:100F50000EC043EA02230D4AACBF00214FF07F418F
:100F600043EA0C030B43C2F8383104B010BD826869
:100F700003AC0323417C02F0010290F91000CDE99B
:100F800000421A46F3F70CF9D7E700BF20650024AA
:100F9000006810B5037984B0012B28D0022B01D052
:100FA000002022E0836803AA13F0010F4FF003032F
:100FB00014BF00218021FFF7C5FB0028F0D09DF869
:100FC0000C309DF90C109DF80D201B0400299DF894
:100FD0000EC043EA02230D4AACBF00214FF07F410F
:100FE00043EA0C030B43C2F8343104B010BD8268ED
:100FF00003AC417C032302F0010290F91000CDE91B
:1010000000420022F3F7CCF8D7E700BF20650024A8
:1010100090F91030F0B503EB4303274E154683B02B
:1010200056F83360044683689A0715D501230DF1FD
:1010300006028DF8061030460DF10701F3F79CFB10
:101040000123002229463046F3F796FBA3689B074D
:1010500017D5012003B0F0BD43691BB19A88186809
:1010600012048261154B164AD3F8100A154BC000C2
:101070005768A3FB003080095368DB1B9842FBD202
:10108000D4E70E4A4FF4FA700E4BD2F8102A0C49EE
:1010900000FB02F24868A3FB023292094B681B1A5C
:1010A0009A42FBD26369002BD3D01A6801209B8837
:1010B000936103B0F0BD00BF2C0200242065002422
:1010C000001000E0D34D621010B5037982B08E4657
:1010D000012B0DD0022B02D0002002B010BD83687E
:1010E000DB0758BF41F0800102B0BDE810408FE738
:1010F000816814467246009401F00104417C90F925
:1011000010000194F3F74CF802B010BD70B50568FB
:1011100084B004460E462B79012B15D0022B02D049
:10112000002004B070BDAB68E122DB071CD5284667
:101130001146FEF737FD0028F2D03246FF21206825
:1011400004B0BDE87040BFE7AA68697C02F0010204
:1011500095F910000DF10F050192E12200958DF82F
:101160000F20F2F70DFEE6E761212846FEF71AFD93
:10117000E1E700BF70B5056884B004460E462B79E0
:10118000012B16D0022B02D0002004B070BDAB683A
:10119000C3222846DB074CBFE1216121FEF702FD97
:1011A0000028F1D03246FF21206804B0BDE870402D
:1011B0008AE7AA6895F9100002F00102697C0192A1
:1011C0000DF10F020092C3228DF80F20E122F2F7F9
:1011D000D7FDE5E770B5056884B004460E462B7967
:1011E000012B1BD0022B02D0002004B070BDAB68D5
:1011F000F0222846DB074CBFE1216121FEF7D2FC3B
:101200000028F1D02246FF2152F8040BFFF75CFFC3
:101210000028E9D02379337004B070BDAA6895F92D
:10122000100002F00102697C01920DF10F020092A0
:10123000F0228DF80F20E122F2F7A2FDE0E700BFD7
:10124000F0B5046883B00021074664262046FEF707
:101250005FFC15227E212046FEF704FD04F042FDCE
:1012600004460D4604F03EFD001B61EB0501B0F5A0
:101270007A7F71F10001F5D3013EEFD105261122ED
:101280007E213868FEF7EEFC04F02CFD04460D4686
:1012900004F028FD001B61EB0501B0F57A7F71F1C8
:1012A0000001F5D3013EEFD10DF1070203213868AB
:1012B000FFF70AFF9DF8073003F03C03142B40F0C2
:1012C0009B800C2240213868FEF7CCFC04F00AFD1C
:1012D00004460D4604F006FD001B61EB0501B0F568
:1012E0007A7F71F10001F5D3454C0923B96B454A6A
:1012F00097F83500B4FBF1F189B2FDF74BFB0346DB
:10130000422138685A88B4FBF2F43C641A79FEF73B
:10131000A9FC04F0E7FC04460D4604F0E3FC001BC6
:1013200061EB0501B0F57A7F71F10001F5D3082278
:1013300041213868FEF796FC04F0D4FC04460D46C3
:1013400004F0D0FC001B61EB0501B0F57A7F71F170
:101350000001F5D3002243213868FEF783FC04F036
:10136000C1FC04460D4604F0BDFC001B61EB050109
:10137000B0F57A7F71F10001F5D310225121386860
:10138000FEF770FC04F0AEFC04460D4604F0AAFC27
:10139000001B61EB0501B0F57A7F71F10001F5D317
:1013A0000A2253213868FEF75DFC04F09BFC0446DA
:1013B0000D4604F097FC001B61EB0501B0F57A7F48
:1013C00071F10001F5D3802256213868FEF74AFCFE
:1013D00004F088FC04460D4604F084FC001B61EB1D
:1013E0000501B0F57A7F71F10001F5D3032138686A
:1013F000FEF78EFB03B0F0BD062005F051F900BFEB
:1014000040420F00F0860C08F0B583B015461C462C
:1014100006460DF107020F46FFF756FE9DF807201E
:1014200005EA0203A34201D103B0F0BD22EA05029E
:1014300039463046224303B0BDE8F040FEF712BC07
:1014400010B582B00821044600686A46FFF73CFEEA
:101450009DF80030DB0602D4002002B010BD062348
:101460006A4600212068FFF7CDF90028F4D09DF8E6
:1014700001209DF8001012029DF80230DFED4A6A4B
:1014800002EB01429DF8041014024FEA01219DF87D
:10149000034013449DF8052001EB044148BF03F1CC
:1014A0007F430A44090207EE903A404B48BF02F1DD
:1014B0007F42F8EEE77A93ED256A07EE102AB3F93A
:1014C0009820F8EEC65AB3F99E10B8EEC77A04EE2B
:1014D000901AB3F9A210C7EE263A87EEA67A06EE66
:1014E000902A334AD3ED247A92F85C41B3F99A20DA
:1014F000F8EEE66A112C06EE102AB3F99C20F8EEFD
:10150000E77A05EE102AB3F9A020B8EEC66A04EE19
:10151000102AB8EEC55AF8EEE44AB3F9A420B8EEA2
:10152000C44A66EEA36A27EE232A23D0A7EE045A04
:10153000A7EE246AE5EE075AE5EE877A77EEA67AFB
:10154000E6EE027AB3F98E20F6EE006AC3ED2A7A4F
:1015500007EE902AB3F98C10F8EEE77A07EE101A2E
:10156000B8EEC77A67EEA37AE7EE267AC3ED2B7A58
:1015700002B010BD03EE102AF8EEC32A03EE101AD3
:10158000B8EEC33AA7EE224AE7EE034AA4EE075AA2
:10159000A4EE876AE5EE075AE5EE877A77EEA67A3B
:1015A000E6EE027ACEE700BF00007848206500240E
:1015B000F8B90024F0B5044683B00D461746061D61
:1015C00020680379012B19D0022B02D0002003B030
:1015D000F0BD83683246FF21DB075CBF3246FF2146
:1015E000FFF716FD0028F1D015B12379DB07E7D40A
:1015F000002FECD023793B7003B0F0BD8268417CB2
:1016000002F0010C90F91000FF22CDE9006CF2F716
:10161000C7FDE7E770B50446051D82B02068037971
:10162000012B16D0022B02D0002002B070BD8368BF
:101630002A46FF21DE075CBF2A46FF21FFF7E8FCB0
:101640000028F1D02379DB07EFD520680379012B3F
:10165000E8D18668FF22417C06F0010690F910006F
:10166000CDE90056F2F79CFDEAE700BF024630B52F
:10167000044652F8040B83B00379012B0ED0022BE1
:1016800001D0002008E0FF21FFF7C2FC0028F8D0BD
:101690002079C04300F0010003B030BD8568417C73
:1016A00005F0010590F910000092FF220195F2F774
:1016B00077FDEBE770B5B42282B00446FF210068E5
:1016C000FEF7D0FA10B9002002B070BD2068251DC9
:1016D0000379012B13D0022BF5D183682A46FF2111
:1016E000DE075CBF2A46FF21FFF792FC0028EAD004
:1016F0002379DB07E8D520680379012BEBD18668D5
:10170000FF22417C06F0010690F91000CDE9005659
:10171000F2F746FDEAE700BF70B50A4682B004461C
:10172000A5210068FEF79EFA10B9002002B070BD36
:101730002068251D0379012B13D0022BF5D1836876
:101740002A46FF21DE075CBF2A46FF21FFF760FC27
:101750000028EAD02379DB07E8D520680379012B3C
